:100000000C949A1B0C94C41B0C94C41B0C94C41B1E
:100010000C94C41B0C94C41B0C94C41B0C94C41BE4
:100020000C94C41B0C94C41B0C94C41B0C94C41BD4
:100030000C94C41B0C94CC670C94C41B0C94C41B70
:100040000C94C41B0C9411A10C9457AE0C94C41BBB
:100050000C94143D0C94C41B0C94C41B0C94C41B32
:100060000C94C41B0C94C41B0C94C41B0C94C41B94
:100070000C94C41B0C94C41B0C94C41B0C94C41B84
:100080000C94C41B0C94C41B0C94C41B8BAC8EAC82
:1000900081AC85ACA5ACA5AC92AC96AC9CACA0AC4C
:1000A000C6ADCBADD0ADDAAD08AE08AEE4ADECADCB
:1000B000F4ADFEAD76D54FD486D4B2D586D486D4F1
:1000C00086D486D486D486D486D486D486D486D460
:1000D00086D486D486D486D486D486D486D486D450
:1000E00086D486D486D486D486D486D486D486D440
:1000F000ACD586D486D486D486D486D486D486D409
:1001000086D485D586D486D486D486D486D486D41F
:1001100086D486D486D486D4C9D583D4084AD73B1E
:100120003BCE016E84BCBFFDC12F3D6C74319ABDC6
:1001300056833DDA3D00C77F11BED9E4BB4C3E91EA
:100140006BAAAABE000000803F05A84CCDB2D44ED9
:10015000B93836A9020C50B9918688083CA6AAAADB
:100160002ABE000000803F004E414E494E4954597E
:10017000494E46CDCCCC3D0AD7233C17B7D1387772
:10018000CC2B329595E6241FB14F0A000020410088
:1001900000C84200401C4620BCBE4CCA1B0E5AAED2
:1001A000C59D7400407A10F35A00A0724E180900E1
:1001B00010A5D4E80000E87648170000E40B5402CC
:1001C0000000CA9A3B000000E1F505000080969807
:1001D00000000040420F000000A086010000001057
:1001E0002700000000E80300000000640000000099
:1001F000000A00000000000100000000002C76D87A
:1002000088DC674F0823DFC1DFAE59E1B1B796E55F
:10021000E3E453C63AE651997696E8E6C28426EBC3
:10022000898C9B62ED407C6FFCEFBC9C9F40F2BAD6
:10023000A56FA5F490055A2AF75C936B6CF9676D6E
:10024000C11BFCE0E40D47FEF520E6B500D0ED90C3
:100250002E0300943577050080841E080000204E90
:100260000A000000C80C333333330F986E12831129
:1002700041EF8D2114893BE65516CFFEE6DB18D100
:10028000844B381BF77C1D901DA4BBE424203284D2
:10029000725E228100C9F124ECA1E53D27434F4D58
:1002A0004D554E49434154494F4E004452595255C1
:1002B0004E004552524F525300494E464F0045435F
:1002C000484F0020746F6F206C6F6E6720657874E4
:1002D000727573696F6E2070726576656E74656491
:1002E0000A0020636F6C6420657874727573696F9F
:1002F0006E2070726576656E7465640A0047322FF1
:1003000047332062616420706172616D657465724B
:10031000730A00536C6565702E2E2E00456E646561
:10032000722D332072656164792E00526573756D8C
:10033000696E67207072696E7400436C69636B202C
:10034000746F20726573756D652E2E2E004E6F20B2
:100350006D6F76652E00456E642066696C65206C55
:100360006973740A00426567696E2066696C65206E
:100370006C6973740A005446207072696E74696EF9
:1003800067206279746520004E6F74205446207097
:1003900072696E74696E670A0046696C65206465EF
:1003A0006C657465643A0044656C6574696F6E20B1
:1003B0006661696C65642C2046696C653A20006F43
:1003C00070656E206661696C65642C2046696C6599
:1003D0003A20002569730025696D20256973002581
:1003E00069682025696D20256973002569642025C9
:1003F00069682025696D20256973002569792025A4
:100400006964202569682025696D2025697300507D
:1004100072696E742074696D653A200050726F7451
:1004200065637465642050696E0A0045787472755E
:1004300064657220257300456E6465722D332072E9
:10044000656164792E00BE02B902B202AB029D0260
:100450006F66660044454255473A004B494C4C454F
:10046000442E20004D3131332053006F6B00456E18
:100470006465722D33204F66662E004361703A45E5
:100480004D455247454E43595F5041525345523AAC
:10049000300A004361703A434153455F4C49474835
:1004A000545F4252494748544E4553533A300A002C
:1004B0004361703A544F47474C455F4C4947485455
:1004C000533A300A004361703A534F4654574152F1
:1004D000455F504F5745523A300A004361703A4CDD
:1004E0004556454C494E475F444154413A300A0015
:1004F0004361703A5A5F50524F42453A300A0043C6
:1005000061703A4155544F4C4556454C3A300A00BB
:100510004361703A5052494E545F4A4F423A310A51
:10052000004361703A50524F47524553533A300A94
:10053000004361703A4155544F5245504F52545FF9
:1005400054454D503A310A004361703A4545505286
:100550004F4D3A310A004649524D574152455F4E80
:10056000414D453A4D61726C696E20437265616C14
:1005700069747920334420534F555243455F434FAC
:1005800044455F55524C3A68747470733A2F2F6724
:1005900069746875622E636F6D2F4D61726C696E40
:1005A0004669726D776172652F4D61726C696E205C
:1005B00050524F544F434F4C5F56455253494F4E44
:1005C0003A312E30204D414348494E455F545950F1
:1005D000453A456E6465722D332045585452554452
:1005E00045525F434F554E543A3120555549443A90
:1005F00063656465326132662D343161322D343782
:1006000034382D396231322D6335356336326633F5
:10061000363766660A002F2F20004D3134352053BF
:100620003C696E6465783E206F7574206F66207239
:10063000616E67652028302D31290A005365747476
:10064000696E672054726176656C20416363656CE6
:1006500065726174696F6E3A200053657474696ED7
:1006600067205265747261637420416363656C65D1
:10067000726174696F6E3A200053657474696E67B5
:10068000205072696E7420416363656C6572617499
:10069000696F6E3A200053657474696E67205072FA
:1006A000696E7420616E642054726176656C2041BD
:1006B0006363656C65726174696F6E3A2000205ADD
:1006C00000205900580020204D61783A2000205A1F
:1006D00000205900580020204D696E3A20004F6ECE
:1006E00020004F666600536F667420656E647374F5
:1006F0006F70733A200000010F150E12FF16170ECF
:1007000013FF03021A14FFFFFF0C04FFFFFF010099
:100710000EFFFF0C190DFF18FFFFFFFFFFFF206406
:100720003A0020693A0020703A0043290A006162C9
:100730006C656420286D696E2074656D70200043BF
:100740006F6C64206578747275646573206172657E
:1007500020004F666673657473206170706C696504
:1007600064004572723A20546F6F206661722100F6
:10077000546F6F206661722066726F6D20726566BD
:100780006572656E636520706F696E740A004E6FE6
:100790002063617365206C696768740A0041637443
:1007A0006976652045787472756465723A200055E3
:1007B0006E6B6E6F776E20636F6D6D616E643A2045
:1007C000220062696E004D31313720494E56414C4E
:1007D000494420444154412E004D3131372050725C
:1007E000696E74696E672E2E2E004730205A25736D
:1007F00000473238205830205930004730205A25E1
:100800007300473932205A257320452573006269E9
:100810006E002020506C616E6E6572427566666572
:100820007242797465733A20002046726565204DE6
:10083000656D6F72793A2000436F6D70696C656405
:100840003A204A616E20323720323031390A002096
:100850007C20417574686F723A2028456E64657219
:100860002D33290A00323031382D31312D32380004
:10087000204C61737420557064617465643A200083
:10088000312E312E360A004D61726C696E00205394
:100890006F6674776172652052657365740A002013
:1008A0005761746368646F672052657365740A00EA
:1008B0002042726F776E206F757420526573657475
:1008C0000A002045787465726E616C20526573650C
:1008D000740A00506F77657255700A007374617204
:1008E000740A006572726F722077726974696E673C
:1008F00020746F2066696C650A00456E6473746FBE
:100900007073202563202563202563202563002044
:100910005A3A0020593A0020583A00656E647374C0
:100920006F7073206869743A2000446F6E6520739D
:100930006176696E672066696C652E0A004D3239F2
:10094000004B494C4C45442E200053544F505045C9
:10095000442E20005072696E7465722073746F703B
:100960007065642064756520746F206572726F72A3
:10097000732E2046697820746865206572726F72E4
:1009800020616E6420757365204D39393920746F8C
:1009900020726573746172742E202854656D7065C1
:1009A0007261747572652069732072657365742E47
:1009B00020536574206974206166746572207265C5
:1009C0007374617274696E67290A004E6F204C69F6
:1009D0006E65204E756D626572207769746820635C
:1009E0006865636B73756D2C204C617374204C6962
:1009F0006E653A20004E6F20436865636B73756DBA
:100A00002077697468206C696E65206E756D62650B
:100A1000722C204C617374204C696E653A2000631F
:100A20006865636B73756D206D69736D6174636860
:100A30002C204C617374204C696E653A20004C691F
:100A40006E65204E756D626572206973206E6F74DD
:100A5000204C617374204C696E65204E756D626523
:100A6000722B312C204C617374204C696E653A20D6
:100A7000004D313130004D3331004D383420582095
:100A800059205A20450054462072656164206572E1
:100A9000726F720A00446F6E65207072696E7469BD
:100AA0006E672066696C650A0020496E76616C6924
:100AB000642065787472756465722000000000001F
:100AC000000000000000000000006B4300006B43CA
:100AD00000007A434D36303020486F74656E6420D4
:100AE000746F6F20636F6C6420746F206368616E35
:100AF00067652066696C616D656E740A0020746FAD
:100B00006F206C6F6E6720657874727573696F6E95
:100B10002070726576656E7465640A0020636F6C80
:100B20006420657874727573696F6E207072657673
:100B3000656E7465640A00FFFFFFFFFFFFFFFFFFA4
:100B4000FFFFFFFFFFFFFFFFFFFFFFFFFFFFFFFFB5
:100B5000FFFFFFFFFFFFFFFFFFFFFFFFFFFFFFFFA5
:100B6000FFFFFFFFFFFFFFFFFFFFFFFFFFFFEFFFA5
:100B7000FFFFFFFFFFFFFFFFFFFFFFFFFFFFEFEFA5
:100B8000FFFFFFFFFFFFFFFFFFFFFFFFFFFFE7DFAD
:100B9000FFFFFFFFFFFFFFFFFFFFFFFFFFFFE7DF9D
:100BA000FFFFFFFFFFFFFFFFFFFFFFFFFFFFE3DF91
:100BB000FFFFFFFFFFFFFFFFFFFFFFFFFFFFF3CF81
:100BC000FFFFFFFFFFFFFFFFFFFFFFFFFFE1E1CFA1
:100BD000FFFFFFFFFFFFFFFFFFFFFFFE78000003A7
:100BE000DDFFFFFFFFFFFFFFFFFFFEFF807E000135
:100BF000EEFFFFFFFFFFFFFFFFFFFE7DCFFC0000CA
:100C0000F77FFFFFFFFFFFFFFFFFFF8E06000000E3
:100C10007BBFFFFFFFFFFFFFFFFFFFC000000000E3
:100C20007DDFFFFFFFFFFFFFFFFFFFFC01FE000076
:100C30003EE7FFFFFFFFFFFFFFFFFFFFFFFC00039B
:100C40001F73FFFFFFFFFFFFFFFFFFFFFFF8000124
:100C50008F81FFFFFFFFFFFFFFFFFFFFFFE00000AF
:100C600083F9FFFFFFFFFFFFFFFFFFFFFF00FC0017
:100C700000F0FFFFFFFFFFFFFFFFFFFFE00FFFC0E0
:100C80000000FFFFFFFFFFFFFFFFFFFE03FFFFC0AE
:100C90000000FFFFFFFFFFFFFFFFFFFFFFFFF90067
:100CA0000000FFFFFFFFFFFFFFFFFFFFFFFFFC0054
:100CB00007C0FFFFFFFFFFFFFFFFFFFFFFFFFF007A
:100CC00007E0FFFFFFFFFFFFFFFFFFFFFFFFFFE06A
:100CD00007F1FFFFFFFFFFFFFFFFFFFFFFFFFFFC2D
:100CE00007F9FFFFFFFFFFFFFFFFFFFFFFFFFFFF12
:100CF00003F9FFFFFFFFFFFFFFFFFFFFFFFFFFFF06
:100D000083F9FFFFFFFFFFFFFFFFFFFFFFFFFFFF75
:100D1000C3FFFFFFFFFFFFFFFFFFFFFFFFFFFFFF1F
:100D2000E1FFFFFFFFFFFFFFFFFFFFFFFFFFFFFFF1
:100D3000F0BFFFFFFFFFFFFFFFFFFFFFFFFFFFFB16
:100D4000F83FFFFFFFFFFFFFFFFFFFFFFFFFFFF980
:100D5000F83FFFFFFFFFFFFFFFFFFFFFFFFFFF7EEB
:100D6000F0FFFFFFFFFFFFFFFFFFFFFFFFFFFF8E13
:100D700003FFFFFFFFFFFFFFFFFFFFFFFFFFFFE09E
:100D80001FFFFFFFFFFFFFFFFFFFFFFFFFFFFFFF53
:100D9000FFFFFFFFFFFFFFFFFFFFFFFFFFFFFFFF63
:100DA000FFFFFFFFFFFFFFFFFFFFFFFFFFFFFFFF53
:100DB000FF7FFFFFFFFFFFFFFFFFFF00007FFFFF41
:100DC000F87FFFFFFFFFFFFFFFFFFF80007FFFFFB8
:100DD000E07FFFFFFFFFFFFFFFFFFFC3FCFFFFFF01
:100DE000F8FFFFFFFFFFFFFFFFFFFFC3FCFFFFFF59
:100DF000F8FFFFFFFFFFFFFFFFFFFF87FDFFFFFF84
:100E0000F1FFFFFFFFFFFFFFFFFFFF87FFFFFFFF78
:100E1000F1FFFFFFFFFFFFFFFFFFFF0FE7F30FFCF7
:100E200023FC3FFFFFFFFFFFFFFFFF0FEF8007F0F7
:100E300003F01E007FFFFFFFFFFFFE1FCF8187C76C
:100E400087C70C007FFFFFFFFFFFFE001FC7C78F94
:100E5000C79F0F0CFFFFFFFFFFFFFE001F878F1FC5
:100E60008F1F0F1FFFFFFFFFFFFFFC3F9F8F8F1F95
:100E70008E001E3FFFFFFFFFFFFFFC7F3F0F1E3F67
:100E80001E3FFE3FFFFFFFFFFFFFF87FFF1F1C3FDE
:100E90001C7FFC7FFFFFFFFFFFFFF8FFFF1E1C7E94
:100EA0001C7FFC7FFFFFFFFFFFFFF0FFCE3E3C7E7D
:100EB0003C7FB8FFFFFFFFFFFFFFF0FF9E3C387C49
:100EC000387E78FFFFFFFFFFFFFFE1FF3C7C787C6F
:100ED000783CF1FFFFFFFFFFFFFFE1F83878781063
:100EE0001801F1FFFFFFFFFFFFFF000060203C0043
:100EF0007C07807FFFFFFFFFFFFFFFFFFFFFFE1F5D
:100F0000FE1FFFFFFFFFFFFFFFFFFFFFFFFFFFFFD2
:100F1000FFFFFFFFFFFFFFFFFFFFFFFFFFFFFFFFE1
:100F2000FFFFFFFFFFFFFFFFFFFFFFFFFFFFFFFFD1
:100F3000FFFFFFFFFFFFFF25753A253032750025C3
:100F40003032753A253032750025756420253032EF
:100F5000753A25303275005A0059005800092000B2
:100F6000000000000000000000000000003FFFF053
:100F700000000000000000000000000000380070C9
:100F80000000000000000000000000000030FC3005
:100F90000000000000000000000000000020FC1025
:100FA0000000000000000000000000000020781099
:100FB00000000000000000000000000000203010D1
:100FC000000000000000000000000000002C00D025
:100FD000F80180000C1FE00000104100002E31D00D
:100FE00048008000123FF00000082080002F7BD0D6
:100FF00043C38CD0023FF00000082080002F7BD03C
:1010000071249267CC3FF00000104100002E31D0D7
:1010100041249E40021FE00000208200002C00D0EE
:1010200049249040121FE0000041040000203010CD
:10103000FBB3CEE00C3FF00000410400002078102C
:1010400000000000003FF000002082000020FC10A3
:1010500000000000003FF000001041000030FC30B4
:1010600000000000000FC000000000000038007009
:10107000000000000007800000FFFFC0003FFFF0FD
:10108000000000000003000000FFFFC0000000009F
:10109000000000000000000000000000003FFFF022
:1010A0000000000000000000000000000038007098
:1010B0000000000000000000000000000033873046
:1010C00000000000000000000000000000278790E2
:1010D000000000000000000000000000002F87D08A
:1010E000000000000000000000000000002F87D07A
:1010F000000000000000000000000000002F03D0EE
:10110000F80180000C1FE000000820800020301053
:1011100048008000123FF0000004104000207810CA
:1011200043C38CD0023FF000000410400020781030
:1011300071249267CC3FF00000082080002030101E
:1011400041249E40021FE00000104100002F03D008
:1011500049249040121FE00000208200002F87D019
:10116000FBB3CEE00C3FF00000208200002F87D0C0
:1011700000000000003FF0000010410000278790B1
:1011800000000000003FF00000082080003387309E
:1011900000000000000FC0000000000000380070D8
:1011A000000000000007800000FFFFC0003FFFF0CC
:1011B000000000000003000000FFFFC0000000006E
:1011C0005072696E742070617573656400473120D8
:1011D000463132303020583020593000004730201E
:1011E0005A2573004D31303920532569004D313473
:1011F0003020532569004D313036205332353500CB
:101200004D31303920532569004D31393020532577
:1012100069005072696E742061626F727465640057
:10122000526573756D65207072696E740053746FCA
:1012300070207072696E7400506F7765722D4C6FFC
:101240007373205265636F7665727900496E6974B5
:101250002E2054462063617264004D3231004E6F7F
:101260002054462063617264004368616E676520A4
:1012700054462063617264004D3231005072696ED1
:10128000742066726F6D2054460053746F70207026
:1012900072696E740041626F7574205072696E7469
:1012A000657200526573756D65207072696E7400A9
:1012B0005061757365207072696E740053746F703D
:1012C000207072696E7400526573756D652070725E
:1012D000696E74005061757365207072696E740078
:1012E000436F6E74726F6C0050726570617265004E
:1012F00054756E6500496E666F2073637265656E26
:10130000004261627973746570205A004D36303046
:10131000204230004368616E67652066696C616DCC
:10132000656E74004261627973746570205A00467C
:101330006C6F7700466C6F7700466C6F7700466184
:101340006E2073706565640046616E20737065651C
:10135000640046616E2073706565640042656400D8
:1013600042656400426564004E6F7A7A6C65004E97
:101370006F7A7A6C65004E6F7A7A6C65005370658F
:101380006564005370656564005370656564004D65
:1013900061696E0057726974696E6720746F2066A8
:1013A000696C653A20006F70656E206661696C65D6
:1013B000642C2046696C653A20006F70656E20666B
:1013C00061696C65642C2046696C653A2000466949
:1013D0006C652073656C65637465640A00205369ED
:1013E0007A653A200046696C65206F70656E6564A9
:1013F0003A20006F70656E206661696C65642C2010
:1014000046696C653A20002066696C653A20004E9A
:101410006F7720002220706F730022207061726548
:101420006E743A2200535542524F5554494E45204E
:1014300043414C4C207461726765743A22004B49F9
:101440004C4C45442E2000747279696E6720746F8D
:101450002063616C6C207375622D67636F64652017
:1014600066696C6573207769746820746F6F206D8E
:10147000616E79206C6576656C732E204D41582025
:101480006C6576656C2069733A0043616E6E6F74AB
:10149000206F70656E207375626469722000544617
:1014A0002063617264206F6B0A006F70656E526F0B
:1014B0006F74206661696C65640A00766F6C756D87
:1014C000652E696E6974206661696C65640A004501
:1014D00072726F723A00544620696E6974206661B8
:1014E000696C0A006175746F25692E67004D32348E
:1014F000004D32332025730024F4D43050C38E20A5
:10150000C2A24017828B7011127A910D816CD90A98
:10151000A861E108C7586607615143061E4B5D0587
:10152000C145A7041A411104093D980371393103DB
:101530004036DB0265339102D4305402802E1D0206
:10154000632CEE01752AC501B028A0011027810186
:101550008F2564012B244B01E0223401AC211F01B3
:101560008D200D01801FFC00841EED00971DDF0003
:10157000B81CD200E61BC600201BBC00641AB200D7
:10158000B219A8000A19A0006A189900D117910091
:1015900040178B00B516840031167E00B315790014
:1015A0003A157300C7146F0058146A00EE136600F2
:1015B0008813630025135E00C7125B006C1257008E
:1015C00015125400C111510070114F0021114B0030
:1015D000D61049008D10470046104400021042000A
:1015E000C00F4000800F3E00420F3C00060F3B0042
:1015F000CB0E3800930E37005C0E3500270E3400FA
:10160000F30D3200C10D3100900D3000600D2E0041
:10161000320D2D00050D2C00D90C2B00AE0C29002D
:10162000850C29005C0C2700350C27000E0C2600C9
:10163000E80B2400C40B2400A00B23007D0B230027
:101640005A0B2100390B2100180B2000F80A1F004B
:10165000D90A1E00BB0A1E009D0A1D00800A1D003B
:10166000630A1C00470A1B002C0A1B00110A1A00FF
:10167000F7091A00DD091900C4091900AB0919009E
:10168000920917007B091800630917004C0916001E
:1016900036091600200916000A091500F50815007C
:1016A000E0081400CC081400B8081400A4081400C2
:1016B000900813007D0812006B08130058081200F0
:1016C0004608120034081100230811001208110006
:1016D00001081100F0071000E0071000D00710000B
:1016E000C0071000B0070F00A107100091070E00FF
:1016F00083070F0074070F0065070E0057070E00E1
:1017000049070E003B070D002E070E0020070D00B5
:1017100013070D0006070D00F9060C00ED060D007D
:10172000E0060C00D4060C00C8060C00BC060C0039
:10173000B0060C00A4060B0099060C008D060B00E9
:1017400082060B0077060B006C060B0061060A0090
:1017500057060B004C060A0042060A0038060A002B
:101760002E060A0024060A001A060A0010060900BE
:1017700007060A00FD050900F4050900EB0509004C
:10178000E2050900D9050900D0050900C7050900CF
:10179000BE050900B5050800AD050800A50509004E
:1017A0009C050800940508008C05080084050800C5
:1017B0007C050800740508006C0507006505080035
:1017C0005D050700560508004E05070047050700A0
:1017D0004005080038050700310507002A05070005
:1017E000230507001C050600160507000F05070066
:1017F0000805060002050700FB040600F5040700C3
:10180000EE040600E8040600E2040700DB0406001C
:10181000D5040600CF040600C9040600C304060070
:10182000BD040600B7040600B1040500AC040600C0
:10183000A6040600A00405009B040600950405000C
:10184000900406008A040500850405008004060053
:101850007A04050075040500700405006B0405009A
:1018600066040500610405005C04050057040500DA
:10187000520405004D04050048040500430405001A
:101880003E0404003A040500350405003004040059
:101890002C04050027040400230405001E04040092
:1018A0001A04040016040500110404000D040400C9
:1018B000090405000404040000040400FC030400FF
:1018C000F8030400F4030400F0030400EC03040034
:1018D000E8030400E4030400E0030400DC03040064
:1018E000D8030400D4030400D0030400CC03040094
:1018F000C8030300C503030024F404D9201BC40C4F
:101900005C0E9804C4095F0265077101F405F900D3
:10191000FB04B30048048700C10369005803550065
:1019200003034500BE023A008402310053022A003C
:101930002902250004022000E4011C00C80119004E
:10194000AF01170098011400840113007101100009
:101950006101100051010E0043010D0036010B0022
:101960002B010B0020010B00150109000C010900DF
:1019700003010800FB000800F3000800EB0007006B
:10198000E4000600DE000600D8000600D2000600D3
:10199000CC000500C7000500C2000500BD00040022
:1019A000B9000400B5000400B1000400AD0004005B
:1019B000A9000400A5000300A20003009F0004008A
:1019C0009B000300980003009500020093000300B1
:1019D000900003008D0002008B00030088000200CD
:1019E0008600020084000300810002007F000200E4
:1019F0007D0002007B0002007900020077000100F8
:101A00007600020074000200720001007100020002
:101A10006F0002006D0001006C0002006A0001000E
:101A20006900020067000100660001006500010016
:101A3000640002006200010061000100600001001A
:101A40005F0002005D0001005C0001005B0001001E
:101A50005A00010059000100580001005700010020
:101A60005600010055000100540001005300000021
:101A7000530001005200010051000100500001001C
:101A80004F0001004E0000004E0001004D0001001B
:101A90004C0001004B0000004B0001004A00010017
:101AA0004900010048000000480001004700010013
:101AB000460000004600010045000000450001000E
:101AC0004400010043000000430001004200000008
:101AD00042000100410000004100010040000100FF
:101AE0003F0000003F0001003E0000003E000100FA
:101AF0003D0000003D0001003C0000003C000000F3
:101B00003C0001003B0000003B0001003A000000E7
:101B10003A000100390000003900010038000000DF
:101B200038000000380001003700000037000100D5
:101B300036000000360000003600010035000000CD
:101B400035000000350001003400000034000000C2
:101B500034000100330000003300000033000100B6
:101B600032000000320000003200010031000000AD
:101B700031000000310001003000000030000000A2
:101B8000300001002F0000002F0000002F00000097
:101B90002F0001002E0000002E0000002E0001008A
:101BA0002D0000002D0000002D0000002D00010080
:101BB0002C0000002C0000002C0000002C00010074
:101BC0002B0000002B0000002B0000002B00010068
:101BD0002A0000002A0000002A0000002A0001005C
:101BE0002900000029000000290000002900000051
:101BF0002900010028000000280000002800000043
:101C00002800000028000100270000002700000035
:101C10002700000027000000270001002600000028
:101C2000260000002600000026000000260001001B
:101C30002500000025000000250000002500000010
:101C40002500000025000100240000002400000001
:101C500024000000240000002400010023000000F4
:101C600023000000230000002300000023000000E8
:101C700023000000230001002200000022000000D9
:101C800022000000220000002200000022000100CB
:101C900021000000210000002100000021000000C0
:101CA00021000000210000002100010020000000B0
:101CB00020000000200000002000000020000000A4
:101CC0002000000020000000200001001F00000094
:101CD0001F0000001F0000001F0000001F00000088
:101CE0001F0000001F0001001E0000001E00000079
:101CF0001E0000001E0000004D38342058205920DE
:101D00005A2045006265640A002C2073797374655B
:101D10006D2073746F70706564212048656174650F
:101D2000725F49443A200048656174696E672066B5
:101D300061696C65640048656174696E67206661FD
:101D4000696C65640048656174696E6720666169E5
:101D50006C65640048656174696E67206661696CD2
:101D60006564005072656865617420504C4120457F
:101D70006E64005072656865617420504C41204269
:101D80006564005072656865617420504C41005074
:101D9000726570617265005072656865617420419A
:101DA000425320456E64005072656865617420413D
:101DB0004253204265640050726568656174204139
:101DC0004253005072657061726500473238004DB1
:101DD000343238005072656865617420504C41009F
:101DE000436F6F6C646F776E004368616E67652048
:101DF00066696C616D656E740044697361626C65DF
:101E0000207374657070657273004D3834005365CB
:101E10007420686F6D65206F66667365747300501B
:101E200072656865617420414253004175746F208A
:101E3000686F6D65004D6F76652061786973004D40
:101E400061696E004D6F76652058004D6F76652094
:101E500059004D6F7665205A004578747275646537
:101E600072004D6F766520302E316D6D004D6F76AE
:101E70006520316D6D004D6F76652031306D6D00E0
:101E80004D6F76652061786973004578747275646A
:101E90006572004D6F7665205A004D6F766520594A
:101EA000004D6F76652058004578747275646572D0
:101EB000004D6F7665205A004D6F76652059004DB4
:101EC0006F76652058005072657061726500F4018C
:101ED0000000F401000064000000E80300000000BE
:101EE000FA430000FA430000A0400000C84100008F
:101EF000A0420000A0420000C8430000BA422044B3
:101F00000020490020204D333031205000504944FA
:101F10002073657474696E67733A0A002046002066
:101F2000420020480020204D3134352053004D61BF
:101F300074657269616C2068656174757020706188
:101F400072616D65746572733A0A00205A002059F7
:101F50000020204D323036205800486F6D65206FCC
:101F600066667365743A0A00204500205A002059BD
:101F70000020580020420020540020204D323035EF
:101F8000205300416476616E6365643A20533C6D72
:101F9000696E5F66656564726174653E20543C6D70
:101FA000696E5F74726176656C5F666565647261A7
:101FB00074653E20423C6D696E5F7365676D656E4A
:101FC000745F74696D655F6D733E20583C6D617818
:101FD0005F78795F6A65726B3E205A3C6D61785F0D
:101FE0007A5F6A65726B3E20453C6D61785F655F24
:101FF0006A65726B3E0A0020540020520020204D7A
:10200000323034205000416363656C6572617469DD
:102010006F6E2028756E6974732F7332293A2050C1
:102020003C7072696E745F616363656C3E20523C04
:10203000726574726163745F616363656C3E2054A2
:102040003C74726176656C5F616363656C3E0A0027
:10205000204500205A0020590020204D32303120E8
:1020600058004D6178696D756D20416363656C65DD
:10207000726174696F6E2028756E6974732F733284
:10208000293A0A00204500205A0020590020204DFE
:102090003230332058004D6178696D756D2066656A
:1020A000656472617465732028756E6974732F732B
:1020B000293A0A00204500205A0020590020204DCE
:1020C0003932205800537465707320706572207522
:1020D0006E69743A0A0020204D3230302044300AB4
:1020E0000020204D3230302044002044697361626A
:1020F0006C65640A0046696C616D656E7420736579
:102100007474696E67733A0020204D31343920436E
:10211000203B20556E69747320696E2043656C7393
:102120006975730A002020473231202020203B208F
:10213000556E69747320696E206D6D0A007A5F6D4B
:10214000696E3A2000795F6D696E3A2000785F6DA4
:10215000696E3A20005265706F7274696E6720650F
:102160006E6473746F70207374617475730A004CBD
:102170006F61642073657474696E677300496E697A
:102180007469616C697A6520454550524F4D005322
:10219000746F72652073657474696E677300466945
:1021A0006C616D656E74004D6F74696F6E0054657F
:1021B0006D7065726174757265004D61696E005075
:1021C0007265686561742041425320636F6E6600DA
:1021D0005072656865617420504C4120636F6E6673
:1021E0000046616E2073706565640046616E207301
:1021F000706565640046616E2073706565640042B9
:1022000065640042656400426564004E6F7A7A6CD2
:1022100065004E6F7A7A6C65004E6F7A7A6C650055
:10222000436F6E74726F6C0053746F7265207365C8
:102230007474696E677300426564004265640042AD
:102240006564004E6F7A7A6C65004E6F7A7A6C65C1
:10225000004E6F7A7A6C650046616E20737065651A
:10226000640046616E2073706565640046616E208F
:1022700073706565640054656D7065726174757224
:1022800065005654726176206D696E005654726115
:1022900076206D696E005654726176206D696E000D
:1022A000566D696E00566D696E00566D696E00560A
:1022B0006D6178204500566D6178204500566D614E
:1022C00078204500566D6178205A00566D6178205F
:1022D0005A00566D6178205A00566D617820590079
:1022E000566D6178205900566D6178205900566D01
:1022F0006178205800566D6178205800566D6178DD
:102300002058004D6F74696F6E00416D61782045F3
:1023100000416D6178204500416D6178205A00418F
:102320006D6178205A00416D6178205900416D61DE
:1023300078205900416D6178205800416D61782006
:102340005800412D74726176656C00412D74726184
:1023500076656C00412D7265747261637400412D65
:102360007265747261637400416363656C004163FC
:1023700063656C004D6F74696F6E00202F00204202
:10238000403A0020403A0048656174696E672064F5
:102390006F6E652E0020573A00457874727564653B
:1023A0007220257300456E6465722D33207265615D
:1023B00064792E0042656420646F6E652E0020579C
:1023C0003A004265642048656174696E672E00209A
:1023D0005A3A0020593A0020436F756E7420583ADB
:1023E0000020453A00205A3A0020593A00583A0055
:1023F00023646566696E65202044454641554C540A
:102400005F4B64200023646566696E652020444547
:102410004641554C545F4B69200023646566696EE4
:1024200065202044454641554C545F4B7020005078
:102430004944204175746F74756E652066696E69D4
:1024400073686564212050757420746865206C6120
:102450007374204B702C204B6920616E64204B6498
:1024600020636F6E7374616E74732066726F6D207B
:1024700062656C6F7720696E746F20436F6E66695A
:102480006775726174696F6E2E680A005049442046
:102490004175746F74756E65206661696C65642141
:1024A0002074696D656F75740A0050494420417548
:1024B000746F74756E65206661696C656421205463
:1024C000656D706572617475726520746F6F2068D8
:1024D0006967680A00204B643A2000204B693A2063
:1024E00000204B703A20000A20436C6173736963CB
:1024F00020504944200A002054753A2000204B7592
:102500003A2000206D61783A2000206D696E3A20F3
:102510000020643A200020626961733A2000566509
:102520002D6A65726B0056652D6A65726B00566583
:102530002D6A65726B00567A2D6A65726B00567A49
:102540002D6A65726B0056792D6A65726B0056793B
:102550002D6A65726B0056792D6A65726B0056782C
:102560002D6A65726B0056782D6A65726B0056781D
:102570002D6A65726B004D6F74696F6E00457374E0
:102580006570732F6D6D004573746570732F6D6D7D
:10259000005A73746570732F6D6D005A7374657093
:1025A000732F6D6D005973746570732F6D6D0059C5
:1025B00073746570732F6D6D005873746570732F2D
:1025C0006D6D005873746570732F6D6D004D6F7471
:1025D000696F6E0053746570732F6D6D004A65727C
:1025E0006B00416363656C65726174696F6E005660
:1025F000656C6F6369747900436F6E74726F6C0001
:1026000046696C2E204469612E0046696C2E204478
:1026100069612E004F6666004F6E20004520696E8E
:10262000206D6D3300436F6E74726F6C0043616E8A
:102630006E6F7420656E7465722073756264697262
:102640003A2000022E2E0001526566726573680002
:102650004D61696E00426175643A20313135323026
:1026600030004D656C7A692028437265616C69742D
:102670007929004578747275646572733A20310067
:102680007777772E637265616C69747933642E6332
:102690006E00456E6465722D3300312E312E36008A
:1026A000437265616C6974792033440041626F75CF
:1026B00074205072696E7465720020204E6F7A7AB1
:1026C0006C653A200020004261636B004D696E69C1
:1026D0006D756D2054656D70206973203137302E13
:1026E0000048656174696E67206661696C656400A5
:1026F00045787472756465206D6F726500526573FC
:10270000756D65207072696E7400524553554D4564
:10271000204F5054494F4E533A0020204E6F7A7A42
:102720006C653A20006368616E6765006F662074AF
:1027300068652066696C616D656E740057616974C7
:1027400020666F72207374617274005052494E5447
:10275000205041555345440020204E6F7A7A6C65D5
:102760003A2000200066696C616D656E7420756E9C
:102770006C6F6164005761697420666F720050521B
:10278000494E54205041555345440020204E6F7A05
:102790007A6C653A20002000506C65617365207783
:1027A0006169742E2E2E0048656174696E67206E13
:1027B0006F7A7A6C65005052494E542050415553FF
:1027C00045440020204E6F7A7A6C653A2000200044
:1027D00068656174206E6F7A7A6C652E0050726540
:1027E000737320627574746F6E20746F0050524959
:1027F0004E54205041555345440020204E6F7A7A64
:102800006C653A2000746F20636F6E74696E756535
:102810002E2E2E00616E64207072657373206275B7
:1028200074746F6E00496E736572742066696C61B2
:102830006D656E74005052494E54205041555345B9
:10284000440020204E6F7A7A6C653A2000200066A2
:10285000696C616D656E74206C6F616400576169AD
:102860007420666F72005052494E542050415553A7
:1028700045440020204E6F7A7A6C653A2000200093
:1028800066696C616D656E742065787472756465D7
:10289000005761697420666F72005052494E54208F
:1028A00050415553454400746F20726573756D65D2
:1028B000005761697420666F72207072696E7400CF
:1028C0005052494E54205041555345440070012CFC
:1028D0000190012701B0012201C0011D01F0011882
:1028E000011002130130020E01600209019002047E
:1028F00001C002FF000003FA004003F5008003F06E
:1029000000D003EB002004E6007004E100E004DCEA
:10291000004005D700C005D2004006CD00D006C853
:10292000008007C3003008BE00F008B900C009B439
:1029300000B00AAF00B00BAA00D00CA500000EA09A
:1029400000500F9B00C01096005012910000148C94
:1029500000C0158700B0178200B0197D00D01B7829
:1029600000001E730040206E0090226900F0246475
:102970000040275F0090295A00E02B5500102E5090
:102980000020304B0010324600E033410090353CCF
:10299000001037370070383200A0392D00B03A28C7
:1029A00000A03B2300603C1E00103D1900903D1428
:1029B00000103E0F00703E0A00C03E0500003F00C0
:1029C00000403FFBFF803FF6FFC03FF1FF5448450A
:1029D000524D414C2052554E415741590054686563
:1029E000726D616C2052756E61776179004572720B
:1029F0003A204D494E54454D5020424544004572C1
:102A0000723A204D494E54454D50004D494E544563
:102A10004D50207472696767657265640045727213
:102A20003A204D415854454D50204245440045728E
:102A3000723A204D415854454D50004D415854452F
:102A40004D5020747269676765726564007C3C3E16
:102A50005E2B3D3F2F5B5D3B2C2A225C000006096C
:102A600000FE070192032120FFFF08FF07FF00007F
:102A700000060000010707060200808080808000B9
:102A800080030202060105A0A0050707060000500A
:102A900050F850F850500507070600002078A07045
:102AA00028F020050707060000C0C810204098182D
:102AB0000507070600006090A040A8906802030385
:102AC000060104C040800307070601002040808003
:102AD000804020030707060100804020202040801E
:102AE00005050506000120A870A8200505050600BB
:102AF000012020F820200203030602FFC0408005C9
:102B00000101060003F8020202060200C0C005052A
:102B10000506000108102040800507070600007028
:102B200088888888887003070706010040C04040F5
:102B30004040E0050707060000708808708080F8B4
:102B4000050707060000F81020100808F005070721
:102B500006000010305090F810100507070600001E
:102B6000F880F0080888700507070600007080806C
:102B7000F0888870050707060000F808102020205C
:102B80002005070706000070888870888870050790
:102B9000070600007088887808087002050506029C
:102BA00000C0C000C0C00206060602FFC0C000C0D0
:102BB00040800407070600001020408040201005D8
:102BC0000303060002F800F804070706010080402E
:102BD000201020408005070706000070880810209C
:102BE000002005070706000070880868A8A870057F
:102BF0000707060000708888F88888880507070698
:102C00000000F08888F08888F0050707060000704B
:102C1000888080808870050707060000F088888813
:102C20008888F0050707060000F88080F08080F8AB
:102C3000050707060000F88080F080808005070700
:102C4000060000708880B8888870050707060000B5
:102C5000888888F8888888010707060200808080B5
:102C60008080808005070706000038101010109043
:102C7000600507070600008890A0C0A0908805079F
:102C800007060000808080808080F8050707060026
:102C90000088D8A8888888880507070600008888E3
:102CA000C8A8988888050707060000708888888863
:102CB0008870050707060000F08888F0808080058E
:102CC000070706000070888888A89068050707062F
:102CD0000000F08888F0A0908805070706000078BB
:102CE0008080700808F0050707060000F820202003
:102CF00020202005070706000088888888888870BB
:102D0000050707060000888888888850200507077F
:102D10000600008888888888A850050707060000F4
:102D20008888502050888805070706000088888812
:102D300050202020050707060000F80810204080DA
:102D4000F8030707060100E08080808080E0050529
:102D5000050600018040201008030707060100E077
:102D60002020202020E005030306000420508805D1
:102D70000101060000F80202020602058040050576
:102D800005060000700878887805070706000080AF
:102D900080B0C88888F0050505060000708080882E
:102DA00070050707060000080868988888780505F8
:102DB000050600007088F8807005070706000030DF
:102DC00048E0404040400506060600FF70888878CD
:102DD00008700507070600008080B0C88888880151
:102DE00007070602008000808080808003080806B4
:102DF00001FF200020202020A0400407070600003B
:102E0000808090A0C0A090030707060100C040404A
:102E1000404040E0050505060000D0A8A8A8A80588
:102E20000505060000B0C88888880505050600006D
:102E300070888888700506060600FFF08888F08094
:102E4000800506060600FF788888780808050505CD
:102E5000060000B0C880808005050506000070806F
:102E60007008F00407070600004040E04040403092
:102E70000505050600008888889868050505060090
:102E80000088888850200505050600008888A8A8C5
:102E900050050505060000885020508805060606E6
:102EA00000FF888888780870050505060000F8107E
:102EB0002040F803070706010020404080404020E2
:102EC000010707060200808080808080800307075A
:102ED00006010080404020404080050202060002BA
:102EE00068900000000600000000000600000000DE
:102EF00000060000000000060000000000060000C0
:102F000000000006000000000006000000000006AF
:102F100000000000000600000000000600000000A5
:102F2000000600000000000600000000000600008F
:102F3000000000060000000000060000000000067F
:102F40000000000000060000000000060000000075
:102F5000000600000000000600000000000600005F
:102F6000000000060000000000060000000000064F
:102F70000000000000060000000000060000000045
:102F8000000600000000000600000000000600002F
:102F9000000000060000000000060000000000061F
:102FA000000000000006000000000006000001070D
:102FB00007060200800080808080800507070600E9
:102FC000002070A8A0A87020050707060000304068
:102FD00040E04050A8050505060000887050708844
:102FE000050707060000885020F820F82001070791
:102FF00006020080808000808080050808060000AE
:103000003048205050209060030101060107A005C0
:103010000707060000F888B8B8B888F8050707065B
:103020000001700878887800F80505050600012879
:1030300050A05028050303060001F8080802020208
:103040000602064080050707060000F888A8889851
:10305000A8F8050101060006F80404040600036050
:103060009090600507070600002020F8202000F857
:1030700004050506000360902040F00305050600E6
:1030800003E020E020E0020202060206408005087C
:10309000080600FF8888888898E88080050707066A
:1030A000000078989878181818020202060202C0E8
:1030B000C00202020602FF4080030505060003402D
:1030C000C04040E00507070600017088888870004E
:1030D000F8050505060001A0502850A005070706C1
:1030E00000008890A858B80808050707060000885F
:1030F00090B848982038050808060000C040C0482D
:10310000D8380808050707060000200020408088FE
:10311000700508080600004020007088F8888805BF
:1031200008080600001020007088F8888805080844
:103130000600002050007088F888880508080600FE
:10314000006890007088F88888050808060000501C
:1031500000708888F888880508080600002050203C
:103160007088F888880507070600003860A0B8E076
:10317000A0B80508080600FF70888080887020606D
:10318000050808060000402000F880F080F80508D7
:1031900008060000081000F880F080F8050808060E
:1031A0000000205000F880F080F8050707060000B6
:1031B0005000F880F080F803080806010080400005
:1031C000E0404040E0030808060100204000E040E5
:1031D0004040E003080806010040A000E0404040F5
:1031E000E0030707060100A000E0404040E00507BB
:1031F00007060000704848E84848700508080600BF
:103200000068900088C8A898880508080600004053
:1032100020708888888870050808060000102070D3
:10322000888888887005080806000020500070888B
:1032300088887005080806000068900070888888F3
:10324000700508080600005000708888888870059E
:10325000050506000188502050880508080600FF73
:103260001070A8A8A8A87040050808060000402013
:1032700088888888887005080806000010208888DB
:103280008888887005080806000020500088888813
:1032900088700508080600005000888888888870B3
:1032A000050808060000102088502020202005096D
:1032B000090600FFC040704848704040E00408081C
:1032C0000601FF609090A09090E08005080806003D
:1032D0000040200070087888780508080600001073
:1032E0002000700878887805080806000020500043
:1032F0007008788878050808060000689000700853
:1033000078887805070706000050007008788878EC
:103310000508080600002050207008788878050607
:1033200006060000D02878A0A8500506060600FF73
:10333000708088702060050808060000402000703A
:1033400088F880700508080600001020007088F8D2
:1033500080700508080600002050007088F8807012
:1033600005070706000050007088F8807003080801
:1033700006010080400040C04040E003080806010C
:103380000020400040C04040E00308080601004023
:10339000A00040C04040E0030707060100A0004035
:1033A000C04040E0050707060000A040A010788854
:1033B00070050808060000689000B0C88888880575
:1033C00008080600004020007088888870050808FA
:1033D0000600001020007088888870050808060024
:1033E0000020500070888888700508080600006872
:1033F00090007088888870050707060000500070EC
:10340000888888700505050600012000F800200561
:1034100007070600FF1070A8A8A870400508080656
:103420000000402000888888986805080806000089
:103430001020008888889868050808060000205039
:10344000008888889868050707060000500088886B
:103450008898680509090600FF102000888888F808
:1034600008700407070601FFC04060506040E00597
:1034700008080600FF50008888887808700000213E
:1034800000240027002A0000002200250028002B2D
:103490000000002000230026002900020202020290
:1034A00002020204040404040404040303030303E7
:1034B00003030301010101010101010102040810DC
:1034C00020408001020408102040800102040810FE
:1034D000204080804020100804020100000001020A
:1034E00000090A00000000040308070000000000B3
:1034F0000000000000000000000000656E717565AE
:103500007565696E672022006563686F3A002E0A50
:10351000006F70656E206661696C65642C20466979
:103520006C653A200057726974696E6720746F2069
:1035300066696C653A2000526573656E643A2000D6
:103540006F6B00627573793A2070617573656420E2
:10355000666F7220696E7075740A00627573793ACD
:103560002070617573656420666F72207573657273
:103570000A00627573793A2070726F6365737369BC
:103580006E670A004B494C4C45442E20004B494C79
:103590004C2063617573656420627920746F6F20BD
:1035A0006D75636820696E616374697665207469FE
:1035B0006D65202D2063757272656E7420636F6D6A
:1035C0006D616E643A2000506C65617365207265B0
:1035D000736574005052494E5445522048414C5432
:1035E0004544005072696E7465722068616C746540
:1035F000642E206B696C6C28292063616C6C656497
:10360000210A00000000000000000000000000008F
:10361000004842000048420000804000000000577F
:1036200061726E696E673A20486F6D696E672042FD
:10363000756D702044697669736F72203C20310A81
:10364000000202040000A0400000A0400000004072
:1036500000006B4300006B4300007A43FFFFFF2E26
:103660000A0046696C652862696E292064656C658C
:103670007465640044656C6574696F6E2862696E78
:1036800029206661696C6564004572726F722077EB
:10369000726974696E6720746F20454550524F4DB2
:1036A000210A0000060900FE0000000000010900D8
:1036B00008FE000005080806000040F0C888889849
:1036C0007810050808060000C0F88888888888F8FF
:1036D0000505050600012030F83020050808060021
:1036E000002070F820202020E00509090600FF20B6
:1036F00070A8A8B8888870200509090600FFE08036
:10370000C0B0A8283028280509090600FFF8A888B5
:1037100088888888A8F8050A0A0600FE20505050BC
:103720005088A8A8887003030306000340A0400047
:1037300048E105E211241FBECFEFD0E4DEBFCDBFCC
:1037400013E0A0E0B1E0EEE1F8EE01E00BBF02C053
:1037500007900D92AE37B107D9F729E1AEE7B3E094
:1037600001C01D92A23AB207E1F71BE1C9E9DBE112
:1037700004C02197FE010E9472F3C839D107C9F72E
:103780000E946CD60C9402F40C9400002F923F928D
:103790004F925F926F927F928F929F92AF92BF9261
:1037A000CF92DF92EF92FF920F931F93CF93DF930D
:1037B000CDB7DEB7C056D1090FB6F894DEBF0FBE45
:1037C000CDBF0091CD0820E6029F80011124035B4C
:1037D000184F8091C10980FF1AC0E8E0F5E3849199
:1037E0007F013FEFE31AF30A811102C0780104C0A0
:1037F0000E949238F701F3CFD7018D917D01882384
:1038000019F00E949238F8CF8AE00E94923881E045
:1038100090E09093BE158093BD151092A90310926D
:10382000A8038FE38093AC031092AB031092AA031A
:1038300084E0E8E9F3E0DF011D928A95E9F7F801F9
:1038400080810F5F1F4F8032D1F38E34C9F48181A4
:1038500090ED980F9A3020F08D3211F08B3281F478
:10386000DF0112969D012F5F3F4F8C9180538A306C
:1038700010F4D901F7CFFD01119680818032D9F380
:10388000F093C615E093C5157F01BFEFEB1AFB0A55
:1038900010816AE270E0C7010E94CAF3009731F01C
:1038A000FC01319780818032E1F311821D3431F1C6
:1038B000143521F1173411F1E8E0F5E384918F011B
:1038C0000F5F1F4F882321F00E949238F801F6CF36
:1038D0006091C5157091C6158FEA97E00E944D4121
:1038E00082E20E9492388AE00E9492381092BE15BD
:1038F0001092BD150E94B0CA0C944133C701FC015F
:10390000208101962032D9F320532A30A8F6109353
:10391000AC0380E090E06AE03196DF0111972C91D2
:10392000022E000C330B20533109689FA001699FC0
:10393000500D1124C901840F951F208120532A3076
:1039400058F39093AB038093AA03DF0131962C9137
:103950002032D9F31D34A9F48E319105D1F03CF415
:1039600087319105B1F08C31910559F412C085373A
:1039700091053CF08737910564F0803AE3E09E07BB
:1039800041F00091C51560E070E0EE24E394F12C65
:1039900043C0B093A903A093A8037FC0213209F4C8
:1039A00045C03FEBB32EB20E49E1A42EAB1408F490
:1039B0005FC0AF01FA0130814F5F5F4F3032D1F30A
:1039C00040ED430F4A3008F047C0AF018B2C912CDB
:1039D000640123E0D594C7942A95E1F7960128560F
:1039E0003C4F69012B2D2770D70102C0AA0FBB1FC6
:1039F0002A95E2F79D01D6013C91232B2C9341158A
:103A00005105A1F1401BD401A258BC4F4C93208119
:103A100021542A3190F5DF01FD0131962C912111BD
:103A2000BDCF7093A9036093A80337C01D3409F07C
:103A3000B8CF8032910509F0B4CFF093A903E09399
:103A4000A80363E270E0CF010E94CAF3009709F473
:103A50007FC7DC011C9221C043ED430F423008F4C4
:103A6000B4CF3B3211F00C94D232AFCF40E0CBCF89
:103A70006115710561F6BD01CACFDF01AD014F5F70
:103A80005F4F2C9120532A3010F4DA01F7CFFD015B
:103A9000119620812032D9F3BECF8091AC038D34B2
:103AA00009F456C7843511F40C948F32873409F029
:103AB00003CF2090AA033090AB03B4E02B1631045F
:103AC00009F4E2C554F437FC11CF80912101F2E0F2
:103AD0002F1631040CF0F4C017C02AE52216310469
:103AE00009F4CDC634F44CE12416310409F411C6AE
:103AF000FDCE5BE52516310409F4C4C68CE5281615
:103B0000310409F4C3C6F2CE882309F4EFCE0E9433
:103B10000F3880912E01882321F083EE95E10E94D9
:103B200054C60E9487388091C10983FD79C0C09036
:103B3000EF15D090F015E090F115F090F21520916E
:103B40008718309188184091891850918A18C701B8
:103B5000B6010E9483E9882309F462C00E9468418B
:103B6000882309F1C0928718D0928818E0928918AA
:103B7000F0928A18E8E0F5E384918F010F5F1F4F00
:103B8000811103C0E2EEF2E004C00E949238F80115
:103B9000F3CF84918F010F5F1F4F882321F00E9484
:103BA0009238F801F6CFC090EF15D090F015E09064
:103BB000F115F090F21520918718309188184091F6
:103BC000891850918A18C701B6010E943CF020E084
:103BD00030E048E453E40E949DF218160CF5C092C0
:103BE0008718D0928818E0928918F0928A18E8E035
:103BF000F5E384918F010F5F1F4F811103C0E3EC48
:103C0000F2E004C00E949238F801F3CF84918F0152
:103C10000F5F1F4F882321F00E949238F801F6CFE2
:103C20002091E3153091E4154091E5155091E6158A
:103C300060917B1870917C1880917D1890917E180E
:103C40000E9483E981111DC02091E7153091E8158C
:103C50004091E9155091EA1560917F187091801894
:103C600080918118909182180E9483E9811109C086
:103C700060910601709107018091080190910901FE
:103C80001AC060911A0170911B01072E000C880B5D
:103C9000990B0E948AE92091060130910701409119
:103CA0000801509109010E94E9E92AE037ED43E259
:103CB0005CE30E94E9E90E94D2350E94C83516CE25
:103CC000882309F413CE0E940F3882E50E9402383F
:103CD000882309F43CC10E94A0374B015C0120E01D
:103CE00030E0A9010E9483E9882309F45CC1209196
:103CF0007B1830917C1840917D1850917E182DA72B
:103D00003EA74FA758AB80917F1890918018A09143
:103D10008118B091821889AB9AABABABBCAB209148
:103D2000E3153091E4154091E5155091E61529AF62
:103D30003AAF4BAF5CAF8091E7159091E815A09139
:103D4000E915B091EA158DAB9EABAFABB8AF6DA5E1
:103D50007EA58FA598A90E9483E981110DC02DA988
:103D60003EA94FA958AD69A97AA98BA99CA90E941F
:103D700083E9882309F417C111E092E02916310480
:103D800009F010E020E030E0A901C501B4010E9473
:103D900083E9881F8827881F181759F020E030E032
:103DA00040E85FEB29962CAF3DAF4EAF5FAF299750
:103DB0000AC080E090E0A0E8BFE329968CAF9DAFF9
:103DC000AEAFBFAF29972DA53EA54FA558A969ADA8
:103DD0007AAD8BAD9CAD0E943CF025966CAF7DAF6B
:103DE0008EAF9FAF259729A93AA94BA95CA96DA9C8
:103DF0007EA98FA998AD0E943CF06B017C012596AD
:103E00002CAD3DAD4EAD5FAD2597CA01B9010E9405
:103E1000E9E92B013C01A7019601C701B6010E9407
:103E2000E9E99B01AC01C301B2010E943DF00E948F
:103E3000EBF221966CAF7DAF8EAF9FAF219720E064
:103E400030E040E05FE30E94E9E92B013C01A5017D
:103E50009401C501B4010E94E9E94B015C01A30191
:103E60009201C301B2010E94E9E99B01AC01C501C5
:103E7000B4010E943CF00E94EBF229962CAD3DADBE
:103E80004EAD5FAD29970E94E9E94B015C01C70186
:103E9000B601905821962CAD3DAD4EAD5FAD21974A
:103EA0000E9437F1A50194010E94E9E96B017C01B0
:103EB00029AD3AAD4BAD5CAD6DA57EA58FA598A99A
:103EC0000E943DF020E030E040E05FE30E94E9E93D
:103ED0009B01AC01C701B6010E943DF02DA53EA596
:103EE0004FA558A90E943CF06B017C012DA93EA969
:103EF0004FA958AD69A97AA98BA99CA90E943DF048
:103F000020E030E040E05FE30E94E9E92B013C0162
:103F100021962CAD3DAD4EAD5FAD219725966CAD94
:103F20007DAD8EAD9FAD25970E9437F1A50194011F
:103F30000E94E9E99B01AC01C301B2010E943DF07E
:103F400029A93AA94BA95CA90E943CF014C089E4B4
:103F50000E940238882329F00E94A0376B017C015F
:103F600003C0C12CD12C76018AE40E940238882338
:103F7000E9F00E94A03769AF7AAF8BAF9CAF20E029
:103F800030E0A901C701B6010E9483E981111BC07D
:103F900020E030E0A90169AD7AAD8BAD9CAD0E9407
:103FA00083E9811110C0EFECF4E15BC320E030E065
:103FB000A901C701B6010E9483E98823A1F319AEC4
:103FC0001AAE1BAE1CAEA701960150582DA73EA7F6
:103FD0004FA758AB89AD9AADABADBCADB05889AB6E
:103FE0009AABABABBCABCA01B9010E94E9E94B018A
:103FF0005C0129A93AA94BA95CA9CA01B9010E948F
:10400000E9E99B01AC01C501B4010E943DF00E94A9
:10401000EBF265966CAF7DAF8EAF9FAF6597209149
:104020007B1830917C1840917D1850917E182DABF3
:104030003EAB4FAB58AFA70196016DA97EA98FA9E2
:1040400098AD0E943DF029966CAF7DAF8EAF9FAFCB
:10405000299780917F1890918018A0918118B09134
:10406000821821968CAF9DAFAEAFBFAF21979C0158
:10407000AD0169AD7AAD8BAD9CAD0E943DF0699606
:104080006CAF7DAF8EAF9FAF69972091E3153091F4
:10409000E4154091E5155091E6152D962CAF3DAFF6
:1040A0004EAF5FAF2D9729962CAD3DAD4EAD5FADB8
:1040B00029972D966CAD7DAD8EAD9FAD2D970E944D
:1040C0003CF06B017C018091E7159091E815A0917F
:1040D000E915B091EA1561968CAF9DAFAEAFBFAF59
:1040E000619769962CAD3DAD4EAD5FAD6997BC0152
:1040F000CD010E943CF04B015C012091831830916E
:10410000841840918518509186186D962CAF3DAF5C
:104110004EAF5FAF6D976091EB157091EC1580918C
:10412000ED159091EE150E943CF025966CAF7DAF99
:104130008EAF9FAF2597A70196016DA57EA58FA590
:1041400098A90E94E9E92B013C01A501940169A904
:104150007AA98BA99CA90E94E9E99B01AC01C30142
:10416000B2010E943DF02B013C01A50194016DA517
:104170007EA58FA598A90E94E9E94B015C01A701E2
:10418000960169A97AA98BA99CA90E94E9E99B01DA
:10419000AC01C501B4010E943CF0A30192010E9450
:1041A000BCF06B017C0120E030E0A9010E9483E9B2
:1041B00087FF0AC02BED3FE049EC50E4C701B60190
:1041C0000E943DF06B017C0132E02316310451F472
:1041D0002BED3FE049EC50E4C701B6010E943CF0F2
:1041E0006B017C0120E030E0A901C701B6010E940B
:1041F00083E9811126C02D962CAD3DAD4EAD5FAD4E
:104200002D976DA97EA98FA998AD0E9483E9811190
:1042100018C061962CAD3DAD4EAD5FAD6197219656
:104220006CAD7DAD8EAD9FAD21970E9483E981116C
:1042300008C01BEDC12E1FE0D12E19ECE12E10E4B9
:10424000F12EA701960165966CAD7DAD8EAD9FAD4B
:1042500065970E94E9E99B01AC010E94E9E94B01E5
:104260005C0125962CAD3DAD4EAD5FAD2597CA01E5
:10427000B9010E94E9E99B01AC01C501B4010E94AA
:104280003DF00E94EBF24B015C012FE632E143E886
:104290005AE30E9483E987FDDEC1C501B4010E9493
:1042A000DFF10E94B0F17EAF6DAF672B21F421E00A
:1042B00030E03EAF2DAF4090871850908818609046
:1042C000891870908A18ADACBEACB50180E090E062
:1042D0000E9488E94B015C019B01AC01C701B6015A
:1042E0000E9437F16DAB7EAB8FAB98AFA501940107
:1042F00025966CAD7DAD8EAD9FAD25970E9437F1B3
:1043000065966CAF7DAF8EAF9FAF6597A3019201AD
:104310006091EF157091F0158091F1159091F21563
:104320000E943CF0A50194010E9437F1A1966CAF68
:104330007DAF8EAF9FAFA1972DA93EA94FA958ADD4
:10434000CA01B9010E94E9E920E030E040E05FE302
:104350000E94E9E99B01AC0160E070E080E89FE326
:104360000E943CF025966CAF7DAF8EAF9FAF259736
:104370006D962CAD3DAD4EAD5FAD6D9729873A87FB
:104380004B875C874D865E866F86788A60911A01BE
:1043900070911B01072E000C880B990B0E948AE973
:1043A00020910601309107014091080150910901C7
:1043B0000E94E9E92AE037ED43E25CE30E94E9E983
:1043C0002D966CAF7DAF8EAF9FAF2D970E944BAEF9
:1043D0009B01AC0128533F4F4F4F5F4F61962CAF6D
:1043E0003DAF4EAF5FAF61974DA45EA46FA478A8B8
:1043F00022242394312CB9E1DB2EADACBEACA21447
:10440000B30409F414C10E949B640E944BAEDC010A
:10441000CB0161962CAD3DAD4EAD5FAD6197821B7A
:10442000930BA40BB50BB7FD11C00E944BAE9B01C3
:10443000AC0128533F4F4F4F5F4F61962CAF3DAFBC
:104440004EAF5FAF619780E00E9444C8DA94DD20F0
:1044500009F441C029A93AA94BA95CA925966CADDC
:104460007DAD8EAD9FAD25970E94E9E94B015C01C2
:104470009201A3016DA97EA98FA998AD0E94E9E9D7
:10448000A50194010E943DF07B018C019201A301E2
:1044900025966CAD7DAD8EAD9FAD25970E94E9E967
:1044A0004B015C0129A93AA94BA95CA96DA97EA978
:1044B0008FA998AD0E94E9E99B01AC01C501B40147
:1044C0000E943CF02B013C01C701D80189AB9AAB9B
:1044D000ABABBCAB4DC0B10180E090E00E9488E97D
:1044E0002DA93EA94FA958AD0E94E9E94B015C01F5
:1044F0000E9432F16B017C01C501B4010E94DDF222
:104500004B015C01A70196016DA57EA58FA598A919
:104510000E94E9E92B013C01A501940169AD7AAD46
:104520008BAD9CAD0E94E9E9A30192010E943DF090
:104530002B013C01A50194016DA57EA58FA598A92D
:104540000E94E9E94B015C01A701960169AD7AADD2
:104550008BAD9CAD0E94E9E99B01AC01C501B401A2
:104560000E943CF069AB7AAB8BAB9CABF9E1DF2EE0
:104570009201A30129966CAD7DAD8EAD9FAD2997BB
:104580000E943DF069837A838B839C8329A93AA991
:104590004BA95CA969966CAD7DAD8EAD9FAD699759
:1045A0000E943DF06D837E838F83988765962CAD46
:1045B0003DAD4EAD5FAD659769857A858B859C85F0
:1045C0000E943DF069877A878B879C87A1962CADE6
:1045D0003DAD4EAD5FADA1976D857E858F85988988
:1045E0000E943DF06D877E878F87988B80912E018A
:1045F000882321F0CE0101960E9454C6C090730911
:104600002D96ECACFDAC0EAD1FAD2D979E01235F3A
:104610003F4FAE01475F5F4FBE016B5F7F4FCE01E3
:1046200001960E9402433FEF231A330AE6CEC09060
:1046300073092D96ECACFDAC0EAD1FAD2D972FEE92
:1046400035E14BEE55E167EE75E183EE95E10E94B1
:1046500002430E94C8350E94873848C90E94923898
:10466000F80184918F010F5F1F4F8111F7CFEDEF9C
:10467000F2E084918F010F5F1F4F882309F436C940
:104680000E949238F801F5CF80E50E940238882315
:1046900029F00E945C376B017C0103C0C12CD12C36
:1046A000760183E50E940238882361F00E94A037DA
:1046B00020E030E04AE754E40E94E9E90E94B0F1CA
:1046C0006B017C010E94876780913701811105C0D1
:1046D00060E083E193E00E9407B30E9487388091F5
:1046E000290790912A07A0912B07B0912C07C80E9B
:1046F000D91EEA1EFB1E0E944BAEDC01CB018C19B9
:104700009D09AE09BF09B7FFF1C880E00E9444C807
:10471000F2CF0E9487678091060190910701A091D6
:104720000801B09109018093A4039093A503A0937D
:10473000A603B093A70380911A0190911B01909357
:10474000A3038093A20384E690E090931B018093DF
:104750001A010E94873881E08093B30388E50E94A4
:10476000D337E82E89E50E94D337082F8AE50E94C7
:10477000D337F82EE11005C0011105C011E018274C
:1047800005C0011102C010E001C0182F0E94BE3503
:10479000111105C0E11003C0002309F444C020E05A
:1047A00030E040EA50E46091D3157091D4158091C7
:1047B000D5159091D6150E943DF06093EB1570933E
:1047C000EC158093ED159093EE15209183183091A0
:1047D000841840918518509186180E949DF21816F1
:1047E0007CF419821A821B821C829E012F5F3F4F2C
:1047F0004BEE55E16FE778E18BE798E10E94CC340E
:10480000111105C0E11003C0011107C00CC080E008
:1048100090E00E94E6C61123B9F381E090E00E9487
:10482000E6C6111102C0FF2021F082E090E00E9454
:10483000E6C60E94F436809115118093B3038091EF
:10484000A4039091A503A091A603B091A703809320
:10485000060190930701A0930801B093090180918C
:10486000A2039091A30390931B0180931A010E94CD
:10487000873883E080938F010E94868737C8109223
:10488000A10334C881E08093A10330C885E40E946D
:104890000238B82E811102C00E94876764E9862E13
:1048A00061E0962E7BE7C72E78E1D72EE7EDEE2E5E
:1048B000E5E1FE2E00E010E0A12C33243394D40176
:1048C0008D914D010E940238882359F1F6014080F4
:1048D0005180628073800E94A037D6016D937D93D2
:1048E0008D939C9313970330E1F0023011F43092D2
:1048F000B603A30192010E943CF09B01AC01F701B9
:1049000060817181828193810E943DF0D7016D9316
:104910007D938D939C931397C8010E94EB35AA2435
:10492000A3940F5F1F4FB4E0CB0ED11CE4E0EE0E5A
:10493000F11C0430110519F6AA2019F00E94F43672
:1049400003C0B1100E9425CC0E9486870C94761C6F
:104950008091AA039091AB038137910509F41EC69B
:104960000CF0D0C08B34910509F436C50CF05FC053
:104970008831910509F494C2B4F58231910509F4A6
:10498000E0C6BCF497FF02C00C94761C82309105FF
:104990000CF4A7C1419711F00C94761C60E08DE4F3
:1049A00093E00E9407B35E985E9815985E980C9409
:1049B000761C8531910509F45CC23CF4449711F0F2
:1049C0000C94761CE5E6F3E014C28631910509F4F7
:1049D00054C2479711F00C94761C8091A8039091D3
:1049E000A903FC0154C28C31910509F4C2C264F4DC
:1049F0008A31910509F461C20CF07EC210928C12CA
:104A00000E94D2CC0C94761C8F31910509F4EEC330
:104A10002CF44E9709F4B7C20C94761C80329105A1
:104A200009F49AC38A9709F497C40C94761C8836C3
:104A3000910509F4DDC40CF046C08235910509F4F6
:104A400077C644F58D34910509F4CEC40CF4C8C47E
:104A50008135910511F00C94761C0E9427A40E94C8
:104A600087670E94D1C710921116109210160E94EB
:104A7000A3CC1092B8031092B70368EE73E080E005
:104A800090E00E94ECB160E08EE694E00E9407B3F3
:104A90000C94761C8435910509F453C60CF44CC66D
:104AA0008535910509F480C68C35910511F00C947B
:104AB000761C24E9C22E21E0D22E3BE8E32E38E119
:104AC000F32E10E08CC68C36910509F463C53CF4D6
:104AD0008A36910509F4FBC50CF4ABC517C68E36B2
:104AE000910509F4D1C40CF4EAC58F36910509F497
:104AF000DEC48037910511F00C94761C8BE594E0B0
:104B00000E94DBC7833D910509F4E4C00CF06BC043
:104B10008139910511F40C944C2D5CF58637910583
:104B200009F472C7A4F48337910509F4D7C00CF4D3
:104B3000D6C68537910511F00C94761C60E0809103
:104B4000A8039091A9030E9425B30C94761C883782
:104B5000910511F40C943F2D0CF48DC78937910504
:104B600011F40C94462D8C38910509F444C50C942D
:104B7000761C893C910511F40C941B2E7CF48E3B21
:104B8000910509F4A0C5883C910511F40C94C72D3A
:104B90008B39910511F00C94761C68C58C3C9105FD
:104BA00011F40C94572E6CF48B3C910511F00C947D
:104BB000761C74E9E72E71E0F72E0CE211E10C94FB
:104BC000472E8D3C910511F40C94C32E8E3C91051B
:104BD00011F00C94761C64E9E62E61E0F62E00E0FC
:104BE00010E00C94302F8039F1E09F0711F40C9401
:104BF0005F3184F58C3231E0930711F40C943B3033
:104C00008CF48D3D910511F40C94F02F823E9105AA
:104C100011F40C940C308C3D910511F00C94761C21
:104C20000C94E12F8E3251E0950711F40C9404316D
:104C300014F40C9465308F32B1E09B0711F40C949E
:104C40005B318336914011F00C94761CEFECF4E16B
:104C50000C946732863FF1E09F0711F40C944D32BB
:104C6000FCF48C3A31E0930711F40C9463314CF46A
:104C70008A39914011F00C94761C0E942D870C9477
:104C8000761C843FA1E09A0711F40C944932853FC9
:104C9000914011F00C94761C0E94A9BD0C94761CD6
:104CA0008835E2E09E0711F40C9460323CF4873FB3
:104CB000914011F40C9451320C94761C803A33E0FC
:104CC000930709F486C2873E934011F40C947B321B
:104CD0000C94761CE8E0F5E30C94492FE6E5F5E04A
:104CE00007C6A090A803B090A90380E50E940238EF
:104CF000882359F00E945C376B017C0111E0672B1F
:104D0000682B692B31F410E004C010E0C12CD12CC9
:104D1000760183E50E9402388823F1F00E94A037D3
:104D200020E030E04AE754E40E94E9E90E94B0F153
:104D30006B017C01111112C0672B682B692B71F478
:104D4000A114B10459F0D5018C91882339F061E0A8
:104D5000C5010E9425B307C0112391F360E08AE3E7
:104D600093E00E9407B383E090E09093BE15809398
:104D7000BD1581E08093E5110E9487670E94873806
:104D8000C114D104E104F104E1F08091290790916C
:104D90002A07A0912B07B0912C07C80ED91EEA1E36
:104DA000FB1E0E944BAEDC01CB018C199D09AE09A4
:104DB000BF09B7FF1AC08091E51181110C94DC3254
:104DC00014C08091E511882321F080E00E9444C83E
:104DD000F8CF80918C1260E0882319F08BE293E089
:104DE00002C08CE193E00E9407B31092E5110C948D
:104DF000761C84918F010F5F1F4F882321F00E9442
:104E00009238F801F6CF10923115109230158DEBD3
:104E100092E10E941AA78BE1EDEBF2E1DE0115961B
:104E200001900D928A95E1F78091BB129091BC128E
:104E30009C838B838CE991E09A83898340E050E0E6
:104E4000BE016F5F7F4F8BE792E00E944F60CE0103
:104E500001960E94C9C7E6E5F3E084918F010F5FD8
:104E60001F4F882311F40C94761C0E949238F8018D
:104E7000F4CF0E94CF5E0C94761C10928C1210928C
:104E80008D120C94761C203209F410823196208108
:104E90002111F9CF40E061E00E945A620C94761C27
:104EA0000E94A3CC80918D12882319F081E0809319
:104EB0008C120E9463CC0C94761C80918D128823F6
:104EC00011F40C94761C83E50E940238882311F4B7
:104ED0000C94761C0E946C37AB01BC0140932715E3
:104EE000509328156093291570932A1587E594E14E
:104EF0000E9485D10C94761C80918D12811103C083
:104F0000E8E8F3E02AC0E6E7F3E084918F010F5F61
:104F10001F4F882321F00E949238F801F6CF60914C
:104F20002715709128158091291590912A154AE02E
:104F30000E9499388FE20E949238609123157091F7
:104F4000241580912515909126154AE00E949938E4
:104F50008AE00E9492380C94761C84918F010F5F36
:104F60001F4F882311F40C94761C0E949238F8018C
:104F7000F4CF40E060E08091A8039091A9030E94E3
:104F80005A620C94761C80918D12882311F40C9433
:104F9000761C87E594E10E9452D187E594E10E9456
:104FA000BCA510928B1210928A12E090A803F09088
:104FB000A90380918D12882311F40C94761C109211
:104FC0008C1280915A14882321F087E594E10E9485
:104FD000BCA5FE0131966F01CF010E94F2CE89EB94
:104FE00092E19093D9128093D812D7018C918F328D
:104FF00009F060C06FE270E0C7010E94CAF38C0143
:105000000F5F1F4F09F45CC06FE270E0C8010E949F
:10501000CAF35C01009709F454C00817190708F097
:1050200050C04C01801A910AA401B801CE018096AB
:105030000E94F3F3E0E2F0E0EC0FFD1FE80DF91D34
:1050400010828E01005E1F4FF80181918F0188232D
:1050500019F00E949238F8CF8AE00E94923860914D
:10506000D8127091D9126115710511F06C5F7F4FE4
:1050700021E0AE01405E5F4FCE0105960E946BAB12
:10508000811112C0BE01605E7F4F8FEB93E00E94E2
:105090004D418EE20E9492388AE00E949238C60109
:1050A0000E94C9C70C94761CD092D912C092D81213
:1050B0008501A6CF8AED92E19093D9128093D81200
:1050C00087018091D8129091D912009709F0049627
:1050D000B8010E94B0D3811103C0E7EAF3E021C018
:1050E000E9E9F3E084917F012FEFE21AF20A8823C5
:1050F00021F00E949238F701F5CFD8018D918D01F2
:10510000882319F00E949238F8CF8AE00E949238E2
:1051100010922715109228151092291510922A1511
:1051200016C084917F01BFEFEB1AFB0A882321F0A0
:105130000E949238F701F5CFF80181918F01882301
:1051400019F00E949238F8CF8EE20E949238C60180
:105150000E94C9C70C94761C80918C1281110E9408
:105160008767E090A803F090A90380E50E94D337F9
:10517000182F882319F00E949037182F80918D12D4
:10518000882311F40C94761C412F61E0C7010E9422
:105190005A6283E50E940238882381F00E946C37AE
:1051A000AB01BC0140932715509328156093291536
:1051B00070932A1587E594E10E9485D180918D1224
:1051C000882319F081E080938C1211110C94761CC5
:1051D00070CE8091A8039091A90321E020938B12B7
:1051E00040E060E00E945A620C94761C0E941960B4
:1051F0007B018C0120E831E541E050E00E94D9EFCD
:10520000C9016DE671E00E944AF34B015C01C801DF
:10521000B70120E13EE040E050E00E94D9EFCA0132
:10522000B90128E130E040E050E00E94D9EF762E4D
:10523000672EC62ED72E5CE3252E312C412C512C07
:10524000C801B701A20191010E94D9EFF62EE72E05
:10525000CA01B901A20191010E94D9EFCB018E01CF
:105260000F5F1F4F8114910499F0EF92FF927F938B
:105270006F936F927F92BF92AF929F928F928BEFBC
:1052800093E09F938F931F930F930E941BE913C08A
:10529000A114B104B1F0EF92FF927F936F936F92DC
:1052A0007F92BF92AF928BEE93E09F938F931F9369
:1052B0000F930E941BE90FB6F894DEBF0FBECDBF5F
:1052C00030C0CD2879F0EF92FF927F936F936F9269
:1052D0007F928FED93E09F938F931F930F930E9484
:1052E0001BE9E9CF892B69F0EF92FF927F936F93CF
:1052F00087ED93E09F938F931F930F930E941BE979
:10530000DACFEF92FF9283ED93E09F938F931F93F9
:105310000F930E941BE90F900F900F900F900F902A
:105320000F9060E0C8010E9425B3E8E0F5E38491A6
:105330007F01BFEFEB1AFB0A882321F00E9492380D
:10534000F701F5CFB8018FE094E00E944D418AE06B
:105350000E9492380C94761C83E50E9402388823C0
:1053600011F40C94761C0E947C37E82E80E50E9494
:105370000238882311F40C94761C0E946C37162F87
:10538000C62ED72ED7FE02C00C94761CE6EFF6E0B0
:105390008491181303C0EFECF4E10AC0319627E0C2
:1053A000EE31F207A9F70C94E1320E949238F8012D
:1053B00084918F010F5F1F4F8111F7CFECE1F4E073
:1053C00084918F010F5F1F4F882311F40C94761C7A
:1053D0000E949238F801F4CF0E9463CC0C94761CA2
:1053E0000E94D2CC0C94761C0E94EEBB0C94761CCE
:1053F00088E690E00E94063981110C94761C809119
:10540000C10983FF02C00C94761C83E50E94023818
:105410008823B1F10E94A0370E94A9F1CB010E941C
:105420008CB20E94A03720E030E04AEA52E40E94A9
:1054300083E918163CF00E94EEBB60E087E394E03D
:105440000E9407B30E94A0372091C5113091C61168
:105450004091C7115091C8110E949DF2181684F412
:105460008AE092E09F938F938BE294E09F938F93D7
:105470001F920E940ACC0F900F900F900F900F90E8
:105480000E9488410C94761C8EE40E940238882386
:1054900011F40C94761C0E946C376093B9157093CC
:1054A000BA158093BB159093BC150C94761C83E5BC
:1054B0000E94D337882359F083E50E94023888235D
:1054C00019F00E947C3701C080E08093C109E8E0B8
:1054D000F5E384918F010F5F1F4F811103C0E4E555
:1054E000F4E004C00E949238F801F3CF84918F0158
:1054F0000F5F1F4F882321F00E949238F801F6CFEA
:105500008091C109811103C0E0E5F4E034C046E4B4
:10551000C42E44E0D42EE12CF12C20E08091C1096E
:1055200090E00E2C02C0959587950A94E2F780FFD3
:1055300017C0BB24B394B20E222319F08CE20E9450
:105540009238F60185919491FC0184918F010F5F4F
:105550001F4F882321F00E949238F801F6CF2B2D9F
:105560003FEFE31AF30A42E0C40ED11C55E0E51602
:10557000F104A1F60AC084918F010F5F1F4F8823A9
:1055800021F00E949238F801F6CF8AE00E9492380A
:105590000C94761C109217010C94761C83E50E94E3
:1055A0000238811103C0E8E0F5E30DC00E947C37AA
:1055B00080937A018D3310F40C94761C8CE38093E5
:1055C0007A010C94761C84918F010F5F1F4F882302
:1055D00021F00E949238F801F6CF40917A0150E014
:1055E00060E070E084E694E00E94FA408AE00E9465
:1055F00092380C94761C8091C10983FF02C00C94F0
:10560000761C83E50E940238882311F40C94761CE2
:105610000E94A0370E94A9F16739710514F066E96C
:1056200070E070930F1660930E160E94DBA30C942B
:10563000761C89E690E00E940639811111C0EBE6E4
:10564000F4E084918F010F5F1F4F882321F00E94A7
:105650009238F801F6CF0E9445888AE00E9492387D
:105660001092BE151092BD150C94413383E50E9433
:105670000238882311F40C94761C0E947C378093A6
:10568000C3158D3318F08CE38093C3150E944BAE85
:105690006B017C012091C31530E0A8EEB3E00E94BD
:1056A0002DF0C60ED71EE81EF91EC092BF15D0926F
:1056B000C015E092C115F092C2150C94761C0E94A0
:1056C0004A8E0C94761C0E94A38C0C94761C83E565
:1056D0000E940238882339F00E946C378B016F3F9B
:1056E000710519F010F00FEF10E080E50E9402380C
:1056F000811106C010931116009310160C94761C9D
:105700000E947C3781110C94761CF4CF80E50E94B6
:105710000238811106C010921116109210160C94C6
:10572000761C0E946C37672B11F00C94761CF3CF1B
:105730001092A0030C94761C81E08093A0030C943B
:10574000761C83E50E9402388823A1F00E94A037CE
:1057500020E030E04AE754E40E94E9E90E94B0F119
:1057600060937B0170937C0180937D0190937E0117
:105770000C94761C88E50E94D33781113BC789E5DC
:105780000E94D337811136C78AE50E94D337811131
:1057900031C785E40E94D33781112CC70E948767E7
:1057A0000E94D1C70C94761C83E50E94D3378823CE
:1057B00011F40C94761C0E94A03720E030E04AE7F8
:1057C00054E40E94E9E90E94B0F16093C715709318
:1057D000C8158093C9159093CA150C94761CD601F0
:1057E0008D916D010E94D337882309F46DC0133069
:1057F00009F063C00E94A0374B015C0120E030E05B
:1058000040EA51E40E9483E987FF4EC0A50194015C
:1058100060919718709198188091991890919A18A2
:105820000E9437F12B013C019B01AC016091751185
:105830007091761180917711909178110E94E9E929
:10584000609375117093761180937711909378110E
:10585000A3019201609138117091391180913A1130
:1058600090913B110E94E9E96093381170933911CE
:1058700080933A1190933B1160916609709167098A
:1058800080916809909169090E9488E9A3019201B9
:105890000E94E9E90E94B0F160936609709367097C
:1058A000809368099093690980929718909298184C
:1058B000A0929918B0929A1807C00E94A037F701D9
:1058C00060837183828393831F5FF4E0EF0EF11C8A
:1058D000143009F084CF0E94D6420C94761C0E94AA
:1058E00087670E9486870C94761C0E949238F80184
:1058F00084918F010F5F1F4F8111F7CFE8E4F5E02E
:1059000003C00E949238F80184918F010F5F1F4FEE
:105910008111F7CFE1E3F5E003C00E949238F8016E
:1059200084918F010F5F1F4F8111F7CFE1E2F5E006
:1059300003C00E949238F80184918F010F5F1F4FBE
:105940008111F7CFE0E1F5E003C00E949238F80141
:1059500084918F010F5F1F4F8111F7CFEFEFF4E0BC
:1059600003C00E949238F80184918F010F5F1F4F8E
:105970008111F7CFE0EFF4E003C00E949238F80104
:1059800084918F010F5F1F4F8111F7CFEBEDF4E092
:1059900003C00E949238F80184918F010F5F1F4F5E
:1059A0008111F7CFE5ECF4E003C00E949238F801D2
:1059B00084918F010F5F1F4F8111F7CFE0EBF4E06F
:1059C00003C00E949238F80184918F010F5F1F4F2E
:1059D0008111F7CFE3E9F4E003C00E949238F801A7
:1059E00084918F010F5F1F4F8111F7CFEBE7F4E038
:1059F00084918F010F5F1F4F882311F40C94761C44
:105A00000E949238F801F4CF85E40E94D3378823AE
:105A100081F00E949037882361F0E8E0F5E38491FB
:105A20008F010F5F1F4F882321F00E949238F801E9
:105A3000F6CF81E40E94D337882381F00E9490370B
:105A4000882361F0E6E1F6E084918F010F5F1F4F3C
:105A5000882321F00E949238F801F6CF0091A80324
:105A60001091A903D8018D918D01882309F48DCD62
:105A70000E949238F7CF0E9439790C94761C81E00D
:105A80008093B303809315110C94761C1092B3038A
:105A9000109215110C94761C83E50E94023888231D
:105AA00019F00E946C3702C060E070E08B01112792
:105AB00002301105DCF0EFECF4E184918F010F5F0F
:105AC0001F4F811103C0EAE1F6E004C00E94923842
:105AD000F801F3CF84918F010F5F1F4F882311F4DA
:105AE0000C94761C0E949238F801F4CF88E40E944E
:105AF00002388823A9F00E946C376A3A71053CF09D
:105B00006530B1E07B072CF064E071E002C06AEA26
:105B100070E0F801EE0FFF1FE45EFE4E71836083BC
:105B200086E40E9402388823A9F00E946C37F801AD
:105B3000EE0FFF1FE05EFE4E718360836F3F7105C5
:105B400019F014F06FEF70E077FF02C060E070E0D2
:105B50007183608382E40E940238882311F40C94DC
:105B6000761C0E946C376530710534F06838710519
:105B70002CF067E870E002C065E070E0000F111FD4
:105B8000F801E85EFE4E718360830C94761C88EC0D
:105B900090E00E94063981110C94761C84E40E94E6
:105BA000D337882309F443C00E94A0376B017C01DE
:105BB00011E020E030E0A9010E9483E9811101C0D9
:105BC00010E010937D1120E030E0A901C701B6017B
:105BD0000E9483E9882359F100919C0310E00E9400
:105BE000A037000F111F000F111FF801E758FE4EDC
:105BF000608371838283938320E030E0A901609108
:105C0000791170917A1180917B1190917C110E9491
:105C100083E981110CC080E090E0A0EEBFE38093A7
:105C2000791190937A11A0937B11B0937C110E940B
:105C300008C60C94761CE4E9EE2EE1E0FE2E0CE39F
:105C400011E1FCE4CF2EF1E1DF2EF70181917F011C
:105C50000E94D337882351F00E94A0370E94B0F1F0
:105C6000D8016D937D938D939C9313970C5F1F4F79
:105C7000C016D10651F70E94B8410C94761C0C5FF7
:105C80001F4FB1E10C331B0711F40C94761CF70184
:105C900081917F010E94D337882389F30E94A03726
:105CA000D8016D937D938D939C931397E8CF83E5F3
:105CB0000E94D3378823D9F00E94A037AB01BC01E2
:105CC000409354115093551160935611709357118E
:105CD00040934C1150934D1160934E1170934F119E
:105CE00086E996E00E9417418AE00E94923880E59A
:105CF0000E94D337882399F00E94A037AB01BC01E2
:105D0000409354115093551160935611709357114D
:105D100089E796E00E9417418AE00E94923882E566
:105D20000E94D337882399F00E94A037AB01BC01B1
:105D3000409350115093511160935211709353112D
:105D40008AE596E00E9417418AE00E94923884E535
:105D50000E94D337882311F40C94761C0E94A0373C
:105D6000AB01BC0140934C1150934D1160934E1107
:105D700070934F118CE396E00E9417418AE00E94D5
:105D800092380C94761C83E50E94D337882351F017
:105D90000E94A037609328117093291180932A11D3
:105DA00090932B1184E50E94D337882351F00E94F1
:105DB000A03760932411709325118093261190933E
:105DC000271182E40E94D337882351F00E945C3768
:105DD0006093520970935309809354099093550925
:105DE00088E50E94D337882351F00E94A037609342
:105DF000691170936A1180936B1190936C1189E50E
:105E00000E94D337882351F00E94A03760936D1110
:105E100070936E1180936F11909370118AE50E94B8
:105E2000D337882351F00E94A0376093711170938B
:105E30007211809373119093741185E40E94D3378B
:105E4000882311F40C94761C0E94A037609375117E
:105E50007093761180937711909378110C94761C3F
:105E6000F70181917F010E94D337882339F00E9486
:105E7000A037AB01BC01C8010E9441360F5F1F4F24
:105E80000330110569F70E94F4360E9486870C944E
:105E9000761C84918F010F5F1F4F882321F00E9491
:105EA0009238F801F6CF83E50E94D337882321F09A
:105EB0000E94903780932E01E6EEF6E084918F01E8
:105EC0000F5F1F4F882321F00E949238F801F6CF10
:105ED00080912E01882319F0EEEDF6E002C0E2EE8B
:105EE000F6E084918F010F5F1F4F811103C0E6ED33
:105EF000F6E004C00E949238F801F3CF84918F013C
:105F00000F5F1F4F882321F00E949238F801F6CFCF
:105F10004091FE105091FF1060910011709101119D
:105F200084ED96E00E9417414091021150910311B7
:105F3000609104117091051181ED96E00E94174166
:105F4000409106115091071160910811709109114B
:105F50008EEC96E00E941741E6ECF6E084918F010A
:105F60000F5F1F4F882321F00E949238F801F6CF6F
:105F700040912201509123016091240170912501EB
:105F800084EC96E00E941741409126015091270130
:105F9000609128017091290181EC96E00E941741DF
:105FA00040912A0150912B0160912C0170912D019B
:105FB0008EEB96E00E9417418AE00E9492380C9482
:105FC000761C83E50E940238882311F40C94761C19
:105FD0000E946C3770931B0160931A010C94761C1D
:105FE0008DED90E00E94063981110C94761C83E5BA
:105FF0000E940238882311F40C94761C00919C03B3
:1060000010E00E946C37000F111FF801E85EFE4F90
:10601000718360830C94761C80E50E94D3378823BB
:1060200011F40C94761C0E946C37F62EC62ED72ED7
:1060300083E50E940238882321F00E946C378B018F
:1060400002C00FEF1FEFC8010196039710F00C94E8
:10605000761CD7FE02C00C94761CE6EFF6E08EE1CB
:1060600097E02491F21611F40C94761C31968E1759
:106070009F07B9F7DDC283E50E940238882319F033
:106080000E946C3702C064E071E079A368A380E5E8
:106090000E940238882339F00E946C376938F3E196
:1060A0007F0730F402C068EE73E07A83698304C02E
:1060B00088E893E19A838983BE01605E7F4FCE01B9
:1060C00001960E94D6CB0C94761C85E40E9402387F
:1060D000811110C080E50E94D337882391F00E947F
:1060E000A0376093AF107093B0108093B11090936D
:1060F000B21007C00E947C37882361F3EFECF4E113
:1061000072C089E40E94D337882381F00E94A037AF
:106110002CEA35EC47E25EE30E94E9E96093AB10BC
:106120007093AC108093AD109093AE1084E40E94F5
:10613000D337882381F00E94A0372CEA35EC47E260
:106140005EE30E9437F16093B3107093B4108093B4
:10615000B5109093B610E8E0F5E384918F010F5FDE
:106160001F4F882321F00E949238F801F6CF40910A
:10617000AF105091B0106091B1107091B21086E2E2
:1061800097E00E9417412CEA35EC47E25EE360910C
:10619000AB107091AC108091AD109091AE100E9438
:1061A00037F1AB01BC0182E297E00E9417412CEA73
:1061B00035EC47E25EE36091B3107091B4108091CA
:1061C000B5109091B6100E94E9E9AB01BC018EE1D7
:1061D00097E00E9417418AE00E9492380C94761C46
:1061E0000E949238F80184918F010F5F1F4F811137
:1061F000F7CF05E112E0D8018D918D01882309F4D4
:10620000C4C90E949238F7CF83E50E94D337182F74
:10621000882371F00E94A0370E94A9F17093340185
:106220006093330121E0672B09F020E02093C9112E
:1062300080E50E94D337882361F0209133013091AB
:106240003401232B11F00E9490378093C9110C94D4
:10625000761C11110C94761CE8E0F5E384918F0113
:106260000F5F1F4F882321F00E949238F801F6CF6C
:106270008091C911882319F060E373E002C066E0E1
:1062800072E08FE397E00E944D416091330170917D
:1062900034018EE297E00E943441EAE2F7E0849113
:1062A0008F010F5F1F4F882311F40C94761C0E94FE
:1062B0009238F801F4CF0E94CA880C94761C0E9490
:1062C00087670C94761CE4E7F9E0FEA7EDA78BEC5A
:1062D000882E85E1982E9BE7A92E98E1B92E2EEF06
:1062E000C22E20E1D22E32E2232E31E0332E43E0C3
:1062F000E42E46E3F42E00E010E0ADA5BEA58D919E
:10630000BEA7ADA7882309F488C0F501408051805D
:1063100062807380D1012D913D914D915C91F60188
:1063200060817181828193810E943DF020E030E0A4
:1063300040E05FE30E94E9E99B01AC01C301B201C7
:106340000E949DF2181654F4F70185919591A5913C
:10635000B49189AB99AFADABBDAF04C019AA19AE6A
:106360001DAA1DAED4012D913D914D915C91C301AB
:10637000B2010E943CF09B01AC0169A979AD8DA9E5
:106380009DAD0E943CF02B013C0120E030E040EA52
:1063900051EC0E949DF287FD0AC020E030E040EA07
:1063A00051E4C301B2010E9483E918161CF4EFEC1A
:1063B000F4E109C0B301A201C8010E9441362DC019
:1063C0000E949238F80184918F010F5F1F4F811155
:1063D000F7CFE0E7F7E084918F010F5F1F4F88232D
:1063E00021F00E949238F801F6CF61E082E697E052
:1063F0000E9407B30E94FD4F88E290E09A83898350
:1064000088EC90E099A388A3BE016F5F7F4FCE0117
:1064100080960E94D6CB0C94761C0F5F1F4FB4E081
:106420008B0E911CE4E0AE0EB11CF4E0CF0ED11C3B
:1064300024E0220E311C34E0E30EF11C0330110580
:1064400009F05BCF0E94F4360E94868760E082E507
:1064500097E00E9407B383E992E099A388A304E63A
:1064600010E01A830983BE01605E7F4FCE01019662
:106470000E94D6CB8AEB92E099A388A31A83098362
:10648000BE01605E7F4FCE0101960E94D6CB0C9478
:10649000761C0E94CEC10C94761C0E9499790C94B3
:1064A000761C83E50E94D337882319F00E94903729
:1064B00001C081E091E089270E94957A0C94761CB6
:1064C0000E943D3D0C94761C0E949238F801849104
:1064D0008F010F5F1F4F8111F7CFEEE8F7E0849136
:1064E0008F010F5F1F4F882311F40C94761C0E94BC
:1064F0009238F801F4CF81E08093210110929B182B
:1065000083E50E94D337811104C00E94CFCA0C9446
:10651000761C0E94903781110C94761CF6CFF09077
:10652000AA03FF2029F1E8E0F5E384918F010F5FD2
:106530001F4F882321F00E949238F801F6CF84E59E
:106540000E9492386F2D70E080E090E04AE00E9457
:10655000993880E20E94923805E112E0D8018D91CD
:106560008D01882311F40C94C52A0E949238F6CF2D
:1065700010927309E8E0F5E384918F010F5F1F4FDC
:10658000882321F00E949238F801F6CF60917309B8
:1065900070E08DE997E00E9434418AE00E949238D1
:1065A0000C94761C6115710519F4BF0161507109D5
:1065B00040E050E00C94E61C80E00E9444C80C943B
:1065C000D12661E0812F0E9463AD6E2D812F0E9444
:1065D00034ADF12CB701812F0E949FADB4E0CB16F2
:1065E000D10411F00C94761CF0921116E092101662
:1065F0000C94761C0E94876788E50E94D337882315
:1066000019F05E9A1092B40389E50E94D33788236B
:1066100019F05E9A1092B5038AE50E94D337882359
:1066200011F40C94761C159A1092B6030C94761CF7
:106630000E94876760E08F2D0E9463AD0F3FEFEFF0
:106640001E0759F48F2D0E940BAD31E020E0892BFD
:1066500009F030E0032F122F05C00130110571F44D
:1066600001E010E08F2D0E940BAD8017910711F40F
:106670000C94761C80E00E9444C8F4CF00E010E047
:10668000F1CFC05ADF4F0FB6F894DEBF0FBECDBFBB
:10669000DF91CF911F910F91FF90EF90DF90CF90FE
:1066A000BF90AF909F908F907F906F905F904F9032
:1066B0003F902F90089590912D07E92FF0E0EB5D2A
:1066C000F84F80839F5F943018F490932D0702C099
:1066D00010922D078091CE088F5F8093CE08089589
:1066E000089580E090E008958FB7F8949091B815E0
:1066F0002091B715921759F0E92FF0E0E95CFA4EB6
:10670000208130E09F5F9F779093B81502C02FEFF4
:106710003FEF8FBFC90108950F931F93CF93DF936E
:10672000EC010E944BAE0E811F8128853985011531
:1067300011052105310559F52C852223A9F13A854A
:1067400021502C8721E0230F2A874D85241301C077
:106750001A86FE0124E0329FE00DF11D112406850A
:106760001785208931890A831B832C833D83DC01B3
:10677000CB01800F911FA11DB11D8E839F83A88720
:10678000B9878C819D81892B79F0149A0DC0DC0129
:10679000CB01801B910BA20BB30BB7FD05C0149866
:1067A0001E821F8218861986DF91CF911F910F914B
:1067B0000895CF92EF92FF920F931F93E0900601FE
:1067C000F09007010091080110910901C090730930
:1067D00027E838E143E858E16FE778E18BE798E193
:1067E0000E9402431F910F91FF90EF90CF90089568
:1067F000CF92DF92EF92FF92CF9381E080931701C7
:10680000C1E081E090911701992309F449C08823E0
:1068100009F446C080E00E9444C860912E07709140
:106820002F076115710581F1072E000C880B990B5C
:106830000E948AE99B01AC016091C5117091C6115B
:106840008091C7119091C8110E943CF06B017C01AE
:1068500020E030E0A9010E949DF218165CF020E0D3
:1068600030E040E450ECC701B6010E9483E987FDA7
:106870000DC00AC020E030E040E450E4C701B6019A
:106880000E949DF2181614F080E0BCCFC093DD1179
:1068900040E050E0BA018AE09BE90E94DA4FB1CFB4
:1068A000CF91FF90EF90DF90CF900895CF92DF923D
:1068B000EF92FF920F931F93CF93DF9300D000D0FE
:1068C000CDB7DEB7182F662351F010924009109211
:1068D0003C0910923D0910923E0910923F090E9416
:1068E0004BAEC0903C09D0903D09E0903E09F0903D
:1068F0003F099B01AC012C193D094E095F0957FD69
:106900003EC017FD16C040914009212F012E000CFA
:10691000330B2C5F3F4FE42F042E000CFF0B2E1780
:106920003F076CF141172CF000E911E020E030E066
:1069300004C004EC19E020E030E0DC01CB01800F62
:10694000911FA21FB31F80933C0990933D09A09310
:106950003E09B0933F0980ED97E09C838B838CE2E6
:1069600091E09A838983BE016D5F7F4FCE010196CE
:106970000E94D6CB809140098F5F809340090F9091
:106980000F900F900F90DF91CF911F910F91FF907B
:10699000EF90DF90CF9008954F925F926F927F9229
:1069A0008F929F92AF92BF92CF92DF92EF92FF921F
:1069B0000F931F93CF93DF935C014B018A01E90191
:1069C0004090060150900701609008017090090105
:1069D000FA01208131814281538160918318709145
:1069E000841880918518909186180E9483E987FF0A
:1069F0002EC0C880D980EA80FB8020E030E0A90169
:106A0000B601C7010E9483E9811108C0E7E1F6E3FE
:106A100085919591A591B4916C017D01C601D70135
:106A20008093060190930701A0930801B093090198
:106A3000F80180819181A281B38180938318909322
:106A40008418A0938518B09386180E94D933C88003
:106A5000D980EA80FB8020E030E0A901C701B601BF
:106A60000E9483E9811106C0C12CD12C88E4E82E54
:106A700082E4F82EC0920601D0920701E09208014C
:106A8000F0920901F50180819181A281B381809307
:106A90007B1890937C18A0937D18B0937E18F40116
:106AA00080819181A281B38180937F189093801817
:106AB000A0938118B09382180E94D933F8012081E5
:106AC0003181428153816091831870918418809143
:106AD0008518909186180E949DF21816A4F5D8800A
:106AE000E980FA80CB8120E030E0A9016D2D7E2D78
:106AF0008F2D9C2F0E9483E981110AC0E7E1F6E304
:106B000085919591A591B491D82EE92EFA2ECB2F8F
:106B10008D2D9E2DAF2DBC2F8093060190930701E4
:106B2000A0930801B0930901F80180819181A281AD
:106B3000B3818093831890938418A0938518B093A1
:106B400086180E94D9330E948767409206015092AE
:106B500007016092080170920901DF91CF911F91A6
:106B60000F91FF90EF90DF90CF90BF90AF909F90EC
:106B70008F907F906F905F904F90089580E1EBE74A
:106B8000F8E1A3EEB5E101900D928A95E1F7089541
:106B900080E1E3EEF5E1ABE7B8E101900D928A9573
:106BA000E1F70895CF92EF92FF920F931F93C09059
:106BB00073097B018C012FEE35E14BEE55E167EE59
:106BC00075E183EE95E10E9402431F910F91FF90C2
:106BD000EF90CF900895CF92DF92EF92FF920F93B4
:106BE0001F93CF93DF93EC01CC0FDD1FCC0FDD1F84
:106BF000FE01E75EF84F20E030E0A901608171817D
:106C0000828193810E943DF0FE01E952FA4E20817B
:106C10003181428153810E943DF06B017C01FE0174
:106C2000E553FA4E6083718382839383FE01E454BB
:106C3000F54F25913591459154918E0102501F4E8B
:106C40000E943DF0F8016083718382839383FE018B
:106C5000E853F54F2591359145915491CE5DDE4F26
:106C6000C701B6010E943DF0688379838A839B83C4
:106C7000DF91CF911F910F91FF90EF90DF90CF9018
:106C800008958F929F92AF92BF92EF92FF920F93CF
:106C90001F93CF93DF938C014A015B01EC01CC0F72
:106CA000DD1FCC0FDD1FCE018558974E7C01C75EDE
:106CB000D84F288139814A815B81C501B4010E9486
:106CC0003CF0F70120813181428153810E943DF0E7
:106CD000F701608371838283938388829982AA8279
:106CE000BB82C801DF91CF911F910F91FF90EF9070
:106CF000BF90AF909F908F900C94EB35CF93FC0199
:106D000020812B33A9F02091CE08243088F4C62F9F
:106D1000BC0180912D07F0E68F9FC0011124835B99
:106D2000984F0E94DEF38C2F0E945B3381E001C0FC
:106D300080E0CF910895DF92EF92FF920F931F931F
:106D4000CF93DF93CDB7DEB76E970FB6F894DEBF63
:106D50000FBECDBF6091D40B7091D50B611571053D
:106D600049F14DE150E0CE0101967C010E94F2E82C
:106D70001E8EF7018F010E191F09D190DD2019F029
:106D80009AE0D912F7CFF701E00FF11F1082C70187
:106D90000E9480BD882371F0DD20A9F00F5F1F4F96
:106DA0008091D40B9091D50B080F191F1093D50B20
:106DB0000093D40B81E02091D40B3091D50B232B81
:106DC00029F480E003C000E010E0F0CF6E960FB62B
:106DD000F894DEBF0FBECDBFDF91CF911F910F9111
:106DE000FF90EF90DF90089527E838E143E858E1FD
:106DF0006FE778E18BE798E10C9413428F929F92B2
:106E0000AF92BF92CF92DF92EF92FF920F931F93B8
:106E1000CF93DF934A015B017901EC01CC0FDD1FB9
:106E2000CC0FDD1FCE018558974E6C01FC011082FE
:106E30001182128213820E94F436F60180829182BE
:106E4000A282B382C090730920E030E0A901B801AA
:106E5000C7010E9483E981110CC0FE01E15FF94C7A
:106E60004591559165917491342F252F962F872F39
:106E700004C0302F212F9E2D8F2DE32EF22E092FAF
:106E8000182F27E838E143E858E16FE778E18BE70E
:106E900098E10E9402430E94876710924C07DF919D
:106EA000CF911F910F91FF90EF90DF90CF90BF9007
:106EB000AF909F908F9008958091CF089091D008C7
:106EC000009731F04AE050E060E070E00C94C4E7D5
:106ED00060E070E0CB0108958091CF089091D008D8
:106EE000009731F04AE050E060E070E00C9496E6E4
:106EF00060E070E0CB0108950E946C3797FD0CC0F4
:106F00000E946C376F3F71058105910509F034F4DB
:106F10000E946C37862F089580E008958FEF0895C2
:106F20008091CF089091D008892B39F00E947C374E
:106F300091E0811103C090E001C091E0892F089594
:106F40000F931F93CF938091CF089091D008009713
:106F5000F1F0FC018F01C1912C2F2F7D89F0C534F8
:106F600011F0C536B9F7F801108260E070E00E94B8
:106F70003AE5F801C083562F472F382F292F0BC031
:106F800060E070E0CF911F910F910C943AE550E0D2
:106F900040E030E020E0652F742F832F922FCF91B7
:106FA0001F910F91089581548A3150F5482F50E078
:106FB000FA0193E0F595E7959A95E1F7E856FC4FCD
:106FC000208130E0877002C0359527958A95E2F7D9
:106FD000822F817020FF15C0FA01E258FC4F90818A
:106FE000992339F02091C5153091C615290F311D0F
:106FF00002C020E030E03093D0082093CF080895FD
:1070000080E008950E94D337882341F081E02091E9
:10701000CF083091D008232B09F480E00895CF9257
:10702000DF92EF92FF920F931F93CF93DF9384E948
:10703000E82E81E0F82E03EE15E1CBE7D8E19DE9DB
:10704000C92E93E0D92EF70181917F010E94D33799
:107050008823E1F00E94A0379B01AC01F6018081FA
:10706000811104C08091A103882329F0688179816E
:107070008A819B8103C060E070E0CB010E943DF0FB
:10708000F801608371838283938309C08881998129
:10709000AA81BB81F80180839183A283B3830C5FB3
:1070A0001F4F2496FFEFCF1ADF0A88E9E81681E028
:1070B000F80649F686E40E9402388823C9F00E9447
:1070C000A03720E030E0A9010E949DF2181684F458
:1070D0000E94A03720E030E040E752E40E9437F100
:1070E0006093060170930701809308019093090152
:1070F000DF91CF911F910F91FF90EF90DF90CF9094
:107100000895FC01238121110C94BCA508950E94CF
:107110004BAE6093290770932A0780932B079093B7
:107120002C0708959091C00095FFFCCF8093C60076
:1071300008958F929F92AF92BF92EF92FF920F931A
:107140001F93CF93DF93CDB7DEB7A0970FB6F89418
:10715000DEBF0FBECDBF611571058105910591F1AF
:1071600000E0842E912CA12CB12C102FEE24E3945E
:10717000F12CEC0EFD1EE00EF11C07FDFA94A501AA
:1071800094010E94D9EFF7016083B901CA010F5F32
:10719000611571058105910541F71F3F31F1E1E06E
:1071A000F0E0EC0FFD1FE10FF11D17FDFA95808156
:1071B0008A3010F097E301C090E3890F0E94923863
:1071C0001150EBCF80E3A0960FB6F894DEBF0FBE50
:1071D000CDBFDF91CF911F910F91FF90EF90BF90A6
:1071E000AF909F908F900C949238A0960FB6F89421
:1071F000DEBF0FBECDBFDF91CF911F910F91FF90EA
:10720000EF90BF90AF909F908F900895EF92FF9274
:107210000F931F93CF93DF937C0184E50E94023884
:10722000D82F882349F10E947C37C82F181604F5FF
:10723000E8E0F5E384918F010F5F1F4F882321F071
:107240000E949238F801F6CF8DE40E949238B7017F
:1072500080E090E04AE00E9499386C2FCC0F770BC9
:1072600089EA9AE00E9434418AE00E94923808C07C
:1072700080939C03D0E004C08091730980939C03A9
:107280008D2FDF91CF911F910F91FF90EF90089577
:10729000CF92DF92EF92FF926B017C0197FF0BC0C0
:1072A0008DE20E949238F094E094D094C094C11C76
:1072B000D11CE11CF11C4AE0C701B601FF90EF9020
:1072C000DF90CF900C949938FF920F931F93CF9338
:1072D000DF93F82E092F162FEFECF4E18491EF01E4
:1072E0002196882321F00E949238FE01F7CFEF2DDE
:1072F000F02F8491EF012196882321F00E9492388B
:10730000FE01F7CF6091B9157091BA158091BB1548
:107310009091BC150E9448398AE00E949238111160
:107320000E94CFCA1092360910923509DF91CF9191
:107330001F910F91FF9008952F923F924F925F926D
:107340006F927F928F929F92AF92BF92CF92DF9275
:10735000EF92FF920F931F93CF93DF931F92CDB7BE
:10736000DEB70E949B368111D6C28091CE08843050
:1073700008F067C00E9474339C0197FD62C0982F8B
:1073800000913509109136098A3019F09D3009F0C5
:1073900024C1109237090115110539F3F801EB5298
:1073A000F74F1082109236091092350925ED38E01A
:1073B0008901F90180812F5F3F4F8032C9F38E34FC
:1073C00009F073C078016AE270E0C8010E94CAF354
:1073D0006C01E114F10409F4AEC061E77AE0C80180
:1073E0000E9401E95C01892B09F062C04AE050E08B
:1073F00060E070E0C70101960E9496E66093D108B4
:107400007093D2088093D3089093D4084090B91514
:107410005090BA156090BB157090BC15FFEF4F1AD5
:107420005F0A6F0A7F0A641575058605970509F4DA
:107430004AC0AB2809F047C061E08EE39AE00E94A1
:10744000643980918C12882309F465C28091CE083A
:10745000811102C010923B098091B7039091B8034B
:10746000181619060CF0E7C0009138091091390977
:1074700020E6209FC001219F900D112487549C4F2E
:107480000E9480BD882309F446C20F5F1F4F1093EE
:107490003909009338098091B7039091B803019797
:1074A0009093B8038093B70336C2E12CF12C8BCFB5
:1074B0006EE470E0C80104960E94CAF3009709F4D4
:1074C00095CF7C0193CFC114D10401F180E0F12C60
:1074D000F801E80FF11D90819A3219F08F5FF926BB
:1074E000F7CF4AE050E060E070E0C60101960E94EC
:1074F00096E6CF2CD12CE12CF12C6C157D058E0558
:107500009F0541F061E08FE19AE099CF61E085EF5E
:1075100099E095CF8091D1089091D208A091D3089D
:10752000B091D4088093B9159093BA15A093BB1568
:10753000B093BC1506C0892B21F060E08BEC99E07C
:107540007ECF80912101811123C067E470E0C801E2
:107550000E94CAF30097E1F04AE050E060E070E07A
:1075600001960E9496E66430710590F4E4E5F9E036
:1075700084917F012FEFE21AF20A882321F00E9402
:107580009238F701F5CF60E08AE499E00E9407B3F2
:1075900068EB72E0C8010E94D5F3892B21F41092A8
:1075A00017011092E5116DEB72E0C8010E94D5F34E
:1075B000892B21F481E499E00E94DBC762EC72E040
:1075C000C8010E94D5F3892B11F40E942D8761E038
:1075D00085ED98E00E947E36C8CE0F3511050CF07F
:1075E000C4CE9C35A1F40E94743397FDBECE209189
:1075F00037092111BACE98012F5F3F4F30933609DA
:1076000020933509F801EB52F74F8083AECE9B33C0
:1076100019F481E080933709809137098111A5CE53
:10762000C80101969093360980933509F801EB5211
:10763000F74F20839ACEEE24E39440912715509182
:1076400028156091291570912A1580912315909124
:107650002415A0912515B0912615481759076A07DA
:107660007B0708F4E12C00E010E09924939480E675
:10767000882E9AE7A92E9AE0B92E26E7622E2AE0F4
:10768000722E8091CE08843008F045C1E11043C1CC
:1076900080913B0981113FC180915F1490916014EA
:1076A000A0916114B09162148093271590932815CE
:1076B000A0932915B0932A1541E050E0BE016F5FF9
:1076C0007F4F87E594E10E9458A8019719F48981BA
:1076D00090E002C08FEF9FEFF82E2090271530909A
:1076E00028154090291550902A1540912315509146
:1076F00024156091251570912615EE24E394241627
:1077000035064606570608F4E12C241635064606CB
:107710005706B0F4019609F4AFC0FAE0FF1609F479
:10772000CAC02DE0F21609F4C6C083E2F81619F0BB
:107730009AE3F912D6C080913A098111D2C0B6C03D
:10774000E5E9FAE084916F012FEFC21AD20A88238B
:1077500021F00E949238F601F5CF0E94876787E5F5
:1077600094E10E94BCA580919114882369F1815015
:1077700080939114EDE8E89FC001112441E061E09D
:107780008A569B4E0E945A62E091911424E0E29F37
:10779000F0011124EE56FB4E4081518162817381CC
:1077A00040932715509328156093291570932A1537
:1077B00087E594E10E9485D180918D12882309F498
:1077C0004BC090928C1248C010928C126AE58AE5E8
:1077D00098E10E9491BB10921C1610926A1840E02A
:1077E00050E0BA0186E794E10E9485D14FE452E06F
:1077F0006CE176E186E794E10E941CD2019679F46F
:1078000037ECC32E32E0D32EF60181916F0188232D
:1078100019F00E949238F8CF8AE00E94923886E7E9
:1078200094E10E94BCA51092B8031092B703B092E5
:10783000D50BA092D40B0E949B360E94EEBB0E94F7
:1078400019606D3371058105910530F07092D50B8B
:107850006092D40B0E949B3610922F1580918D124E
:10786000882319F00E941F5E21C00E94CF5E809184
:107870008D128111F7CF1AC0EFECF4E184916F0102
:107880002FEFC21AD20A882321F00E949238F60103
:10789000F5CFE6E8FAE084916F019FEFC91AD90AA3
:1078A000882321F00E949238F601F5CFE3E2FE1220
:1078B00002C090923B0910923A090115110509F492
:1078C000E0CE80912D07889E000D111D1124F80136
:1078D000E35BF84F108280E00E945B3300E010E031
:1078E000D0CE0F35110508F0CCCEFBE3FF1202C05D
:1078F00090923A0980913A098111C3CE80912D0767
:10790000F801889EE00DF11D1124E35BF84FF08231
:107910000F5F1F4FB6CE0F90DF91CF911F910F9148
:10792000FF90EF90DF90CF90BF90AF909F908F909F
:107930007F906F905F904F903F902F9008958F921F
:107940009F92AF92BF92CF92DF92EF92FF92CF932E
:107950006B017C01B42E20E030E0A9010E9483E994
:1079600087FF07C08DE20E949238F7FAF094F7F88B
:10797000F094C0E060E070E080E09FE3CB1541F060
:107980002DEC3CEC4CEC5DE30E94E9E9CF5FF6CFD7
:107990009B01AC01C701B6010E943DF06B017C0167
:1079A0000E94B0F14B015C014AE00E949938CC235F
:1079B00089F1C501B4010E9488E99B01AC01C701AE
:1079C000B6010E943CF06B017C018EE20E9492386D
:1079D00020E030E040E251E4C701B6010E94E9E94D
:1079E0004B015C010E94A9F16B01770FEE08FF08C3
:1079F000C701B6010E944839C701B6010E948AE951
:107A00009B01AC01C501B4010E943CF06B017C01FB
:107A1000C150F1F6CF91FF90EF90DF90CF90BF90E3
:107A2000AF909F908F9008951F920F920FB60F9274
:107A300011240BB60F922F938F939F93EF93FF9385
:107A4000E091B71581E08E0F8F779091C60020915D
:107A5000B815821731F0F0E0E95CFA4E908380931C
:107A6000B715FF91EF919F918F912F910F900BBEC2
:107A70000F900FBE0F901F9018952F923F924F922C
:107A80005F926F927F928F929F92AF92BF92CF92AE
:107A9000DF92EF92FF920F931F93CF93DF93CDB7B7
:107AA000DEB764970FB6F894DEBF0FBECDBF85E496
:107AB0000E94D337882329F00E94A0376B017C01F4
:107AC00005C0C12CD12CE12C30ECF32E8AE50E94AC
:107AD0000238882329F00E94A0372B013C0103C003
:107AE000412C512C320188E50E940238882319F07C
:107AF0000E94A03703C060E070E0CB0169877A87FD
:107B00008B879C8789E50E940238882319F00E94A0
:107B1000A03703C060E070E0CB016D877E878F8760
:107B2000988B85E50E94D337882329F00E94A037DF
:107B30004B015C0106C0812C912C28ECA22E22EC7A
:107B4000B22E8CE40E94D337882339F00E94A037EC
:107B5000698B7A8B8B8B9C8B04C0198A1A8A1B8A3F
:107B60001C8A82E40E940238882321F00E946C372C
:107B7000162F01C015E020907C1230907D1280916C
:107B8000C4158111A0C28091C10983FD3EC020E0CF
:107B900030E0A901C501B4010E9483E9811109C047
:107BA00020E030E0A901C701B6010E9483E98823E3
:107BB00061F18091C911811126C020912E07309169
:107BC0002F07809133019091340128173907DCF495
:107BD000EFECF4E184917F019FEFE91AF90A882321
:107BE00021F00E949238F701F5CFE4EDFAE084919C
:107BF0007F019FEFE91AF90A882309F464C20E9401
:107C00009238F701F4CF0E94F83381E08093C415D5
:107C100090918C12992321F010928C12809341093B
:107C20000E94D2CC81E08093DD1140E050E0BA01A7
:107C30008CE29CE90E94DA4F0E94876780E1EBE7C3
:107C4000F8E1A2E4B9E001900D928A95E1F720E015
:107C500030E0A901C701B6010E9483E98823F1F051
:107C60000E94BE35A70196016091EF157091F01545
:107C70008091F1159091F2150E943DF06093EF15FF
:107C80007093F0158093F1159093F21560E070E019
:107C900080E792E40E94D2350E94876720E030E0BE
:107CA000A901C301B2010E949DF2181624F580E0DB
:107CB00090E0A0EAB0E48D839E83AF83B887A301F0
:107CC0009201609183187091841880918518909129
:107CD00086180E943DF069837A838B839C839E0182
:107CE0002B5F3F4FAE014F5F5F4F6FE778E18BE750
:107CF00098E10E94CC3480E090E0A8ECB2E4898363
:107D00009A83AB83BC839E012F5F3F4F43E858E1CA
:107D1000BE01635F7F4FCE0109960E94CC3420E004
:107D200030E0A901C501B4010E9483E9882359F11B
:107D300081E08093DD1140E050E0BA018BE99BE9DE
:107D40000E94DA4F80E00E9444C80E94BE35A5011F
:107D500094016091EF157091F0158091F11590915B
:107D6000F2150E943DF06093EF157093F01580932B
:107D7000F1159093F21560E070E080E291E40E94CA
:107D8000D2350E94876701E00093DD1140E050E0AA
:107D9000BA0188EE99E90E94DA4F61E0812F0E94D2
:107DA000563480E00E9444C80E944BAEDC01CB01F7
:107DB00088539045AF4FBF4F8093B7109093B81042
:107DC000A093B910B093BA1010927C0983E090E0B0
:107DD0009093BE158093BD150093E5118091E51138
:107DE000882309F44EC060E0812F0E9456348091B0
:107DF0007C09882309F441C00093DD1140E050E084
:107E0000BA0189E79AE90E94DA4F8091E511811160
:107E100030C01092B7101092B8101092B910109292
:107E2000BA1010927C090E9444A40E94F833009377
:107E3000DD1140E050E0BA0188EE99E90E94DA4F86
:107E40000E944BAEDC01CB0188539045AF4FBF4F32
:107E50008093B7109093B810A093B910B093BA1054
:107E600010927C090093E51161E0812F0E94563445
:107E700004C081E00E9444C8C8CF81E00E9444C889
:107E8000ADCF81E090E09093BE158093BD158091B9
:107E9000C415882309F417C1F0907C091092B7101B
:107EA0001092B8101092B9101092BA1010927C096A
:107EB00080E00E9444A4F1100E94F83361E0812F19
:107EC0000E9456340E94BE3520E030E0A901698945
:107ED0007A898B899C890E9483E9882309F448C0A8
:107EE000FF2051F081E08093DD1140E050E0BA01C5
:107EF00088EE99E90E94DA4F83E090E09093BE15F6
:107F00008093BD1581E08093E5118091E511882370
:107F100011F0F110DEC081E090E09093BE158093E7
:107F2000BD158093DD1140E050E0BA0187E599E985
:107F30000E94DA4F29893A894B895C896091EF1553
:107F40007091F0158091F1159091F2150E943DF01D
:107F50006093EF157093F0158093F1159093F215DF
:107F600060E070E080EC90E40E94D2350E94876768
:107F700011E083E0C82ED12CEE24E394F12C109371
:107F8000DD1140E050E0BA0186EC98E90E94DA4F3A
:107F900020E030E048E452E46091EF157091F01574
:107FA0008091F1159091F2150E943DF06093EF15CC
:107FB0007093F0158093F1159093F21560E070E0E6
:107FC00080E490E40E94D2350E948767D092BE156B
:107FD000C092BD151092E5111093DD11109284111D
:107FE0001092831140E050E0BA018DEB9CE90E94B1
:107FF000DA4F8091831190918411009721F481E0F0
:108000000E9444C8F6CFF092BE15E092BD150197CC
:1080100009F4B5CF11E01093DD1140E050E0BA0152
:1080200087EA97E90E94DA4F80914E0990914F09B3
:10803000A0915009B09151098093871890938818A6
:10804000A0938918B0938A188093EF159093F01538
:10805000A093F115B093F2150E9425CC80E090E03A
:10806000A8ECB2E489839A83AB83BC839E012F5F23
:108070003F4F43E858E166E479E082E499E00E94EA
:10808000CC3480E090E0A0EAB0E489839A83AB83AB
:10809000BC839E012F5F3F4F4AE459E06FE778E1D0
:1080A0008BE798E10E94CC340E94FD4F80914109FA
:1080B000882339F080918D12811110938C121092C7
:1080C00041091092C4152A94232859F40E9463CCC4
:1080D00008C060E0812F0E94563481E00E9444C8AD
:1080E00014CF64960FB6F894DEBF0FBECDBFDF91FC
:1080F000CF911F910F91FF90EF90DF90CF90BF90A5
:10810000AF909F908F907F906F905F904F903F9037
:108110002F9008954F925F926F927F92AF92BF928D
:10812000CF92DF92EF92FF920F931F93CF93DF9343
:108130008C01EB01FC0147A050A461A472A4AFA084
:10814000B8A4C9A4DAA49501A601C301B2010E9492
:1081500083E987FF40C0A3019201C301B2010E94DD
:10816000E9E92B013C01F80183A994A9A5A9B6A9C5
:10817000BC01CD0190589B01AC010E943DF0F8017B
:1081800027A530A941A952A90E94E9E99B01AC01A8
:10819000C301B2010E943CF00E94EBF27B018C0112
:1081A0009B01AC01B501C6010E9483E987FF02C0B3
:1081B000750186019701A801B501C6010E9483E9F6
:1081C000882349F0C701D8018FA398A7A9A7BAA708
:1081D000888181608883DF91CF911F910F91FF90FB
:1081E000EF90DF90CF90BF90AF907F906F905F90B7
:1081F0004F900895CF92DF92EF92FF92CF93DF934B
:108200006A017B01FC018491EF012196882321F012
:108210000E949238FE01F7CF4AE0C701B601DF9114
:10822000CF91FF90EF90DF90CF900C949938CF9240
:10823000DF92EF92FF92CF93DF936A017B01FC0103
:108240008491EF012196882321F00E949238FE014B
:10825000F7CF42E0C701B601DF91CF91FF90EF90D9
:10826000DF90CF900C949F3C0F931F93CF93DF939D
:108270008B01FC018491EF012196882321F00E945B
:108280009238FE01F7CFB801110F880B990BDF91DF
:10829000CF911F910F910C9448390F931F93CF9357
:1082A000DF938B01FC018491EF012196882321F05B
:1082B0000E949238FE01F7CFE8018991882319F0D6
:1082C0000E949238FACFDF91CF911F910F910895BC
:1082D0008091C91181111AC06091330170913401EC
:1082E000072E000C880B990B0E948AE99B01AC01B8
:1082F0006091C5117091C6118091C7119091C811FC
:108300000E9483E9881F8827881F089580E00895C8
:1083100086E40E94D33780939E11882351F00E94F7
:10832000A03760931201709313018093140190930E
:10833000150183E50E94D337882351F00E94A037AE
:1083400060930E0170930F018093100190931101BF
:1083500082E40E94D337882351F00E94A0376093B3
:108360000A0170930B0180930C0190930D01089505
:108370004F925F926F927F928F929F92AF92BF9235
:10838000EF92FF920F931F93CF93DF93CCE3D1E152
:108390008BE8E82E88E1F82E0AE519E0412C512CF3
:1083A000320143946991799189919991F701819072
:1083B0009190A190B1907F010E9488E9A50194015C
:1083C0000E94E9E90E94B0F1F801619371938193F1
:1083D00091938F01461657066806790610F42B0113
:1083E0003C01F1E1CC34DF07E9F66FEF7FEFCB0121
:1083F000A30192010E94D9EF20936F093093700975
:108400004093710950937209DF91CF911F910F91A1
:10841000FF90EF90BF90AF909F908F907F906F9064
:108420005F904F9008952F923F924F925F926F927C
:108430007F928F929F92AF92BF92CF92DF92EF92F4
:10844000FF920F931F93CF93DF9300D000D0CDB74F
:10845000DEB77B016A011901ABE8B8E12D913D91CE
:108460004D915C91FC0160817181828193810E94B8
:10847000E9E90E94AAF22B013C010CE412E1D801C7
:108480006D937D938D939C93139720918F183091CA
:1084900090184091911850919218F7016081718164
:1084A000828193810E94E9E90E94AAF24B015C015A
:1084B000D80114966D937D938D939C93179720917B
:1084C0009318309194184091951850919618F60190
:1084D00060817181828193810E94E9E90E94AAF200
:1084E0006B017C01D80118966D937D938D939C93BD
:1084F0001B97209197183091981840919918509196
:108500009A18F10160817181828193810E94E9E969
:108510000E94AAF269837A838B839C83D8011C967C
:108520006D937D938D939C931F970E9487678FB760
:10853000F894EBE6F8E14082518262827382848291
:108540009582A682B782C086D186E286F38629818B
:108550003A814B815C8124873587468757878FBF57
:10856000109238121092391210923A1210923B1255
:1085700080E1ECE3F2E1DF011D928A95E9F70F90CB
:108580000F900F900F90DF91CF911F910F91FF905F
:10859000EF90DF90CF90BF90AF909F908F907F90A3
:1085A0006F905F904F903F902F9008950F931F937F
:1085B000CF93DF93CBE8D8E100E317E0299139911D
:1085C0004991599160E070E080E89FE30E9437F1A3
:1085D000F80161937193819391938F01F8E1CB3905
:1085E000DF0761F727E838E143E858E16FE778E112
:1085F0008BE798E10E941342DF91CF911F910F9179
:108600000C94B8412F923F924F925F926F927F925B
:108610008F929F92AF92BF92CF92DF92EF92FF9292
:108620000F931F93CF93DF93CDB7DEB7C657D10912
:108630000FB6F894DEBF0FBECDBF3B014A01590112
:10864000E9A6FBAE0CAF1EAF3C2C20918B183091ED
:108650008C1840918D1850918E18DC016D917D9190
:108660008D919C910E94E9E90E94AAF2AF966CAFAD
:108670007DAF8EAF9FAFAF9720918F18309190183C
:108680004091911850919218F3016081718182811B
:1086900093810E94E9E90E94AAF2E3966CAF7DAF54
:1086A0008EAF9FAFE397209193183091941840912B
:1086B000951850919618D4016D917D918D919C9152
:1086C0000E94E9E90E94AAF2E7966CAF7DAF8EAFF7
:1086D0009FAFE7972091971830919818409199187B
:1086E00050919A18F50160817181828193810E9475
:1086F000E9E90E94AAF269966CAF7DAF8EAF9FAF99
:10870000699780914C1290914D12A0914E12B091A8
:108710004F12AF968CAC9DACAEACBFACAF97881A85
:10872000990AAA0ABB0A8091501290915112A09105
:108730005212B0915312E396CCACDDACEEACFFAC70
:10874000E397C81AD90AEA0AFB0ACFA6D8AAE9AA67
:10875000FAAA8091541290915512A0915612B0919C
:108760005712E796CCACDDACEEACFFACE797C81A7D
:10877000D90AEA0AFB0ACBAADCAAEDAAFEAA8091D2
:10878000C10983FF0EC06996CCACDDACEEACFFAC8A
:108790006997C0925812D0925912E0925A12F092F0
:1087A0005B128091581290915912A0915A12B09177
:1087B0005B1269964CAC5DAC6EAC7FAC6997481AA5
:1087C000590A6A0A7B0A09F473C00E946841882327
:1087D00049F16996CCACDDACEEACFFAC6997C092C8
:1087E0005812D0925912E0925A12F0925B12E8E0BD
:1087F000F5E384918F010F5F1F4F882321F00E94C2
:108800009238F801F6CFECE1FBE084918F010F5F25
:108810001F4F882321F00E949238F801F6CF412C97
:10882000512C32017301620177FE07C0CC24DD2494
:108830007601C418D508E608F7086091971870917A
:1088400098188091991890919A180E94A9F19B010B
:10885000AC01A8ECB0E00E941AF06C157D058E0505
:108860009F054CF56996CCACDDACEEACFFAC6997DE
:10887000C0925812D0925912E0925A12F0925B12A2
:10888000E8E0F5E384918F010F5F1F4F882321F00B
:108890000E949238F801F6CFEDEFFAE084918F0153
:1088A0000F5F1F4F882321F00E949238F801F6CF06
:1088B000412C512C3201D501C4018827B7FD839585
:1088C0009927AA27BB27182FCFA4D8A8E9A8FAA8C8
:1088D000F7FC1260CBA8DCA8EDA8FEA8F7FC14609A
:1088E00077FC1860E32CF12CC701880F991F880FC3
:1088F000991F9C012A5A364F6901C301B2010E9497
:108900008AE9D6012D913D914D915C910E94E9E952
:108910002B013C01F701EE0FFF1FE85EFE4F608167
:108920007181072E000C880B990B0E948AE99B012C
:10893000AC01C301B2010E94E9E92AE037ED43E24C
:108940005CE30E94E9E92B013C0120E030E0A90151
:108950000E949DF218164CF420E030E040E05FE306
:10896000C301B2010E943DF008C0A301920160E082
:1089700070E080E09FE30E943CF00E94A9F16FABA1
:1089800078AF89AF9AAF80915C128F5F8F70A1969C
:108990008FAFA19780915D12A196CFACA197C8121D
:1089A00004C080E00E9444C8F5CFE0915C12EE2E36
:1089B000F12CFEA6EDA62DE4E29FF0011124EA526F
:1089C000F44F108212A3D501C401B7FE07C0882757
:1089D0009927DC0188199909AA09BB098283938325
:1089E000A483B5838DE4CDA4DEA48C9DF0018D9D80
:1089F000F00D1124EA52F44F8FA598A9A9A9BAA99C
:108A0000B7FF07C0B095A095909581959F4FAF4F48
:108A1000BF4F86839783A087B1878DE4EDA4FEA422
:108A20008E9DF0018F9DF00D1124EA52F44F8BA919
:108A30009CA9ADA9BEA9B7FF07C0B095A095909518
:108A400081959F4FAF4FBF4F82879387A487B5878C
:108A50008DE4CDA4DEA48C9DF0018D9DF00D11243C
:108A6000EA52F44FCFA8D8ACE9ACFAACC686D786A8
:108A7000E08AF18A02811381248135814681578100
:108A800060857185401751076207730714F4B901B7
:108A9000A8018DE4EDA4FEA48E9DF0018F9DF00D44
:108AA0001124EA52F44FC284D384E484F5848FA95C
:108AB00098ADA9ADBAADC416D506E606F70644F4DE
:108AC00084179507A607B70754F4DB01CA0107C04E
:108AD0008C159D05AE05BF0514F4D701C6014DE404
:108AE000CDA4DEA44C9DF0014D9DF00D1124EA5261
:108AF000F44F828B938BA48BB58B0697A105B105A0
:108B000010F40C947F4FDF01A95BBF4F80911016CA
:108B1000909111168D939C933182012B022B032B84
:108B200009F05E988DE4EDA4FEA48E9DF0018F9D6A
:108B3000F00D1124EA52F44F86819781A085B1850A
:108B4000892B8A2B8B2B09F05E988DE4CDA4DEA4B3
:108B50008C9DF0018D9DF00D1124EA52F44F828519
:108B60009385A485B585892B8A2B8B2B09F01598C5
:108B7000CFA8D8ACE9ACFAACCD28CE28CF2811F4D8
:108B80000C94654F80916E09882319F08150809371
:108B90006E09311004C05E9880E280936E092090C7
:108BA00028113090291100912A1110912B1129A51B
:108BB0003BAD4CAD5EADB101C8010E949DF21816EF
:108BC00014F00C94794FC501B4010E948AE92091F8
:108BD00030073091310740913207509133070E949E
:108BE000E9E969A77AA78BA79CA769837A838B8316
:108BF0009C836FA578A989A99AA90E948AE92091E6
:108C000034073091350740913607509137070E945D
:108C1000E9E94B015C016D837E838F8398876BA9A3
:108C20007CA98DA99EA90E948AE9209138073091DC
:108C3000390740913A0750913B070E94E9E96B01DF
:108C40007C0169877A878B879C8720913C073091CC
:108C50003D0740913E0750913F07C301B2010E947A
:108C6000E9E96D877E878F87988B2DE44DA55EA5FA
:108C7000249FF001259FF00D1124EA52F44F428009
:108C800053806480758056E0451651046104710478
:108C9000E4F44680578060847184A6E04A1651044B
:108CA0006104710494F44284538464847584B6E04E
:108CB0004B1651046104710444F4DC01CB01BF770D
:108CC00087A790ABA1ABB2AB34C029A53AA54BA501
:108CD0005CA5CA01B9010E94E9E92B013C01A5018B
:108CE0009401C501B4010E94E9E99B01AC01C301F3
:108CF000B2010E943DF04B015C01A7019601C70142
:108D0000B6010E94E9E99B01AC01C501B4010E94D2
:108D10003DF00E94EBF22DE4CDA4DEA42C9DF001E9
:108D20002D9DF00D1124EA52F44F67A770AB81AB73
:108D300092AB8DE4EDA4FEA48E9DF0018F9DF00D0D
:108D40001124EA52F44F27A530A941A952A960E0A5
:108D500070E080E89FE30E9437F122966CAF7DAF10
:108D60008EAF9FAF22979B01AC01B101C8010E9459
:108D7000E9E96B017C0180915C1290915D12891B85
:108D80008F7027968FAF2797A701960160E074E256
:108D900084E799E40E9437F10E94AAF24B015C013A
:108DA00027968FAD27978250863008F044C0809177
:108DB000520990915309A0915409B0915509881610
:108DC0009906AA06BB06B8F588199909AA09BB092C
:108DD000BC01CD01660F771F881F991F2796FFAC36
:108DE00027970F2D10E020E030E0A90198010E94A4
:108DF000D9EFCA01B9010E9488E90E94AAF2680D60
:108E0000791D8A1D9B1D0E9488E99B01AC0160E0D1
:108E100074E284E799E40E9437F16B017C019B01C5
:108E2000AC0160E074E284E799E40E9437F10E94AB
:108E3000AAF24B015C012FB7F8948091D91190915F
:108E4000DA11A091DB11B091DC11880E991EAA1ED7
:108E5000BB1E8092D9119092DA11A092DB11B092D0
:108E6000DC112FBF8DE42DA53EA5829F8001839F3D
:108E7000100D11240A52144FD8019F964D915D9107
:108E80006D917C91D297A5964CAF5DAF6EAF7FAFE1
:108E9000A5979A01AB01C701B6010E94E9E92696A0
:108EA0006CAF7DAF8EAF9FAF2697F80163A374A31D
:108EB00085A396A322893389448955892FA738AB86
:108EC00049AB5AABCA01B9010E9488E96BAB7CABD4
:108ED0008DAB9EAB9B01AC01C701B6010E94E9E9D5
:108EE0000E941BF10E94B0F12B966CAF7DAF8EAF4C
:108EF0009FAF2B97F80167AB70AF81AF92AF9E0128
:108F00002F5F3F4F3DAF2CAFAE014F5E5F4F61967D
:108F10005FAF4EAF61976CE271E12F967FAF6EAF9E
:108F20002F972D965FAF4EAF2D97212C312C70E8E7
:108F300079A78FE38BAFACADBDAD2D913D914D9138
:108F40005D91BDAFACAFC701B6010E94E9E92D96B6
:108F5000EEADFFAD2D9761937193819391932D9613
:108F6000FFAFEEAF2D974B015C01E894B7F82F9659
:108F7000AEADBFAD2F974D905D906D907D902F96CB
:108F8000BFAFAEAF2F97A3019201C501B4010E94FC
:108F90009DF2181694F4A5019401C301B2010E9438
:108FA00037F15B018C01910149A55BAD0E9483E91A
:108FB00087FF03C0150109A71BAF6196EEADFFAD9A
:108FC00061972CAD3DADE217F30709F0B4CF20E077
:108FD00030E040E85FE3B10189A59BAD0E9483E9E1
:108FE00087FF4BC07E0131E2E30EF11C61960EADAE
:108FF0001FAD6197910149A55BADD8016D917D9140
:109000008D919C910E94E9E9F8016193719381939C
:1090100091938F01EE16FF0669F78DE4CDA4DEA4CF
:109020008C9D80018D9D100D11240A52144F26969F
:109030002CAD3DAD4EAD5FAD2697B10189A59BAD81
:109040000E94E9E9D80193966D937D938D939C934B
:1090500096972B966CAD7DAD8EAD9FAD2B970E94F4
:1090600088E9910149A55BAD0E94E9E90E94B0F150
:10907000F80167AB70AF81AF92AF2BA93CA94DA9A6
:109080005EA922966CAD7DAD8EAD9FAD22970E94FC
:10909000E9E969A77AA78BA79CA78DE4CDA4DEA4F4
:1090A0008C9DF0018D9DF00D1124EA52F44F8280C9
:1090B0009380A480B58081149104A104B10409F5C2
:1090C00086819781A085B185892B8A2B8B2BC9F44A
:1090D00082859385A485B585892B8A2B8B2B89F472
:1090E00020915011309151114091521150915311D2
:1090F00069A57AA58BA59CA50E94E9E90E941BF1B0
:109100002BC2CFA8D8ACE9ACFAACCD28CE28CF285A
:1091100049F06091541170915511809156119091C0
:10912000571108C060914C1170914D1180914E11F2
:1091300090914F1129A53AA54BA55CA50E94E9E99C
:109140000E941BF10E94B0F16B017C0180916F09BC
:1091500090917009A0917109B09172092FA538A959
:1091600049A95AA982179307A407B50708F4DEC0D6
:1091700081149104A104B10421F160915A09709104
:109180005B0980915C0990915D096C157D058E05E8
:109190009F05B8F40E94C9EF2B013C01A70196017D
:1091A000C501B4010E94C9EF461657066806790644
:1091B00040F4C301B201A50194010E94D9EF6901F5
:1091C0007A018DE44DA55EA5849FF001859FF00D89
:1091D0001124EA52F44F86809780A084B1848114D0
:1091E0009104A104B10441F160915E0970915F099D
:1091F00080916009909161096C157D058E059F0530
:10920000D8F42FA538A949A95AA90E94C9EF2B0162
:109210003C01A7019601C501B4010E94C9EF4616A1
:1092200057066806790640F4C301B201A50194010E
:109230000E94D9EF69017A018DE46DA57EA5869F14
:10924000F001879FF00D1124EA52F44F8284938439
:10925000A484B58481149104A104B10441F1609106
:1092600062097091630980916409909165096C1598
:109270007D058E059F05D8F42FA538A949A95AA9BF
:109280000E94C9EF2B013C01A7019601C501B40161
:109290000E94C9EF461657066806790640F4C301D6
:1092A000B201A50194010E94D9EF69017A018DE410
:1092B000ADA5BEA58A9FF0018B9FF00D1124EA5247
:1092C000F44F86849784A088B18881149104A10406
:1092D000B10409F445C160916609709167098091F4
:1092E0006809909169096C157D058E059F0508F048
:1092F00037C12FA538A949A95AA90E94C9EF2B0146
:109300003C01A7019601C501B4010E94C9EF4616B0
:1093100057066806790608F023C1C301B201A5010A
:1093200094010E94D9EF69017A011AC18114910454
:10933000A104B104B9F160915A0970915B0980915F
:109340005C0990915D096C157D058E059F0550F5B2
:109350000E9488E92BA93CA94DA95EA90E94E9E9D0
:109360002B013C01C501B4010E948AE94B015C015B
:10937000C701B6010E9488E9A50194010E94E9E9AC
:109380009B01AC01C301B2010E9483E987FF0AC0BF
:10939000A5019401C301B2010E9437F10E94B0F10E
:1093A0006B017C018DE42DA53EA5829FF001839F7A
:1093B000F00D1124EA52F44F468057806084718486
:1093C0004114510461047104B9F160915E09709116
:1093D0005F0980916009909161096C157D058E058A
:1093E0009F0550F50E9488E92BA93CA94DA95EA9CB
:1093F0000E94E9E94B015C01C301B2010E948AE9C4
:109400002B013C01C701B6010E9488E9A30192012A
:109410000E94E9E99B01AC01C501B4010E9483E906
:1094200087FF0AC0A3019201C501B4010E9437F170
:109430000E94B0F16B017C018DE44DA55EA5849F77
:10944000F001859FF00D1124EA52F44F42845384B9
:10945000648475844114510461047104B9F160910C
:1094600062097091630980916409909165096C1596
:109470007D058E059F0550F50E9488E92BA93CA922
:109480004DA95EA90E94E9E94B015C01C301B2014B
:109490000E948AE92B013C01C701B6010E9488E9BC
:1094A000A30192010E94E9E99B01AC01C501B4014D
:1094B0000E9483E987FF0AC0A3019201C501B4019C
:1094C0000E9437F10E94B0F16B017C018DE46DA523
:1094D0007EA5869FF001879FF00D1124EA52F44F7C
:1094E00086849784A088B18881149104A104B10472
:1094F000B9F160916609709167098091680990914E
:1095000069096C157D058E059F0550F50E9488E957
:109510002BA93CA94DA95EA90E94E9E92B013C01B8
:10952000C501B4010E948AE94B015C01C701B60183
:109530000E9488E9A50194010E94E9E99B01AC0120
:10954000C301B2010E9483E987FF0AC0A50194010B
:10955000C301B2010E9437F10E94B0F16B017C019E
:109560008DE4ADA5BEA58A9F80018B9F100D1124AF
:109570000A52144FF801ED5BFF4FC082D182E282A4
:10958000F382C701B6010E9488E96B017C0129A51D
:109590003AA54BA55CA50E9437F1A9966CAF7DAFAB
:1095A0008EAF9FAFA997F80163AB74AB85AB96AB59
:1095B00020E030E040E85BE4C701B6010E94E9E941
:1095C00020E034E244EF59E40E9437F10E94A9F10F
:1095D000D8015E966D937D938D939C93919793960E
:1095E000CC909397CFAA9496DC909497DFA695960B
:1095F000EC909597EBAA9696FC90F9A629E631E1B6
:10960000AB963FAF2EAFAB972E0131E2430E511C0C
:1096100059E6252E51E1352E61966EAC7FAC6197EF
:10962000CBAEDCAEEEAE2396FFAE239710E0D301B7
:109630008D909D90AD90BD903D01E894B7F8F101FB
:10964000C190D190E190F1901F01A7019601C50151
:10965000B4010E949DF2181694F5112349F1A70157
:1096600096016FA97FA58BA999A50E94E9E96B01D5
:109670007C012BAD3CAD4EAD23965FAD2397C5016C
:10968000B4010E94E9E99B01AC01C701B6010E9447
:1096900083E987FF13C0A5019401C701B6010E94A9
:1096A00037F16BAF7CAF8EAF23969FAF239706C089
:1096B000CBAEDCAEEEAE2396FFAE239711E04614A0
:1096C000570409F0B4CF2796FFAD2797F23008F47E
:1096D00099C1C09038122796CFAE2797D0903912F3
:1096E0002896DFAE2897E0903A122C96EFAE2C9792
:1096F000F0903B122E96FFAE2E9727E137EB41ED0F
:1097000058E3B601C7010E949DF218160CF07AC109
:109710009601A7016FA97FA58BA999A50E9483E94E
:1097200087FF13C09601A7016FA97FA58BA999A5F3
:109730000E9437F1A0966CAF7DAF8EAF9FAFA09720
:109740002FA83FA40BA919A524C02FA93FA54BA959
:1097500059A527966FAD279728967FAD28972C9609
:109760008FAD2C972E969FAD2E970E9437F1A09625
:109770006CAF7DAF8EAF9FAFA09727962FAC27978A
:1097800028963FAC28972C960FAD2C972E961FADA0
:109790002E972CE332E16C963FAF2EAF6C97C12C25
:1097A000D12C40E8E42E4FE3F42E6596CCAEDDAE2E
:1097B000EEAEFFAE65976A961FAE6A976C96AEAD39
:1097C000BFAD6C97CD90DD90ED90FD906C96BFAFE6
:1097D000AEAF6C976196EEADFFAD619781909190C1
:1097E000A190B1906196FFAFEEAF619727962FAD34
:1097F000279728963FAD28972C964FAD2C972E96FD
:109800005FAD2E976FA97FA58BA999A50E9483E9CB
:1098100087FF0CC0A0962CAD3DAD4EAD5FADA097BF
:10982000C701B6010E94E9E96B017C016A96FFADB0
:109830006A97FF23C1F065962CAD3DAD4EAD5FAD8F
:109840006597C701B6010E94E9E96B017C01659645
:109850002CAD3DAD4EAD5FAD6597C501B4010E9425
:10986000E9E94B015C01A5019401C701B6010E9421
:109870009DF220E030E0A90118162CF5C501B401D5
:109880000E949DF218164CF020E030E0A901C701BB
:10989000B6010E9483E987FF05C0A5019401C701B5
:1098A000B60124C02401350177FA709477F87094DA
:1098B000A3019201C701B6010E949DF218165CF542
:1098C0002601370128C0C501B4010E9483E987FD44
:1098D00009C020E030E0A901C701B6010E949DF255
:1098E00018164CF4A7019601C501B4010E943CF082
:1098F0002B013C0110C02601370177FA709477F8EC
:109900007094A3019201C501B4010E9483E987FD0F
:1099100002C024013501AB96AEADBFADAB97CD9083
:10992000DD90ED90FD90AB96BFAFAEAFAB97A701CA
:109930009601C301B2010E949DF21816ECF4A30136
:109940009201C701B6010E9437F19B01AC016596F7
:109950006CAD7DAD8EAD9FAD65970E94E9E96596D2
:109960006CAF7DAF8EAF9FAF65976A96BFAD6A97BC
:10997000BF5F6A96BFAF6A97ECE4F2E16C96CEAC3B
:10998000DFAC6C97EC15FD0509F018CF6A96DFACDB
:109990006A97DD2061F065962CAD3DAD4EAD5FADB3
:1099A0006597B101C8010E94E9E91B018C0124EA15
:1099B00030E74DE75FE3B101C8010E94E9E96B01BF
:1099C0007C0120916A0930916B0940916C0950919A
:1099D0006D090E9483E987FF28C0A70196016BAD3E
:1099E0007CAD8EAD23969FAD23970E949DF21816F5
:1099F000E4F48DE4EDA4FEA48E9DF0018F9DF00DA6
:109A0000112408C08DE4CDA4DEA48C9DF0018D9DB1
:109A1000F00D1124EA52F44F8081846080832BACD6
:109A20003CAC0EAD23961FAD23978DE4EDA4FEA4B0
:109A30008E9DF0018F9DF00D1124EA52F44FC1016B
:109A4000D80183A794A7A5A7B6A7A9966CAD7DADAD
:109A50008EAD9FADA99790589B01AC010E943DF03F
:109A6000A5962CAD3DAD4EAD5FADA5970E94E9E941
:109A70009B01AC016BE077ED83E29BE30E943CF03D
:109A80000E94EBF26B017C019B01AC01B101C801AA
:109A90000E9483E987FD02C0160187018DE42DA590
:109AA0003EA5829FF001839FF00D1124EA52F44FEE
:109AB000C101D80187A390A7A1A7B2A7B080960142
:109AC000A7016FA97FA58BA999A50E9483E9181604
:109AD00014F481E001C083E09DE4CDA4DEA49C9D4C
:109AE00090019D9D300D1124A9014A52544F7A01D5
:109AF000B82ADA01BC9280E1FE017196ACE3B2E1D2
:109B000001900D928A95E1F78FA99FA5ABA9B9A500
:109B10008093381290933912A0933A12B0933B126B
:109B20008BAD9CADAEAD2396BFAD239780936A09F4
:109B300090936B09A0936C09B0936D092FA93FA571
:109B40004BA959A5BC01CD010E9437F16DA37EA39D
:109B50008FA398A72FA93FA54BA959A5B101C8016B
:109B60000E9437F169A37AA38BA39CA3AE014B5D3E
:109B70005F4FBE016F5D7F4FC7010E94D576A196F2
:109B8000CFACA197C0925C12AF96CCACDDACEEAC82
:109B9000FFACAF97C0924C12D0924D12E0924E1291
:109BA000F0924F12E396CCACDDACEEACFFACE39799
:109BB000C0925012D0925112E0925212F09253126F
:109BC000E796CCACDDACEEACFFACE797C09254129C
:109BD000D0925512E0925612F09257126996CCAC80
:109BE000DDACEEACFFAC6997C0925812D09259121E
:109BF000E0925A12F0925B1280915C1290915D1289
:109C0000891B8F70843008F49DC040905D12809154
:109C10005C1283508F70F82E812C912C00E010E0A4
:109C20003DE4532E4F1409F48DC00115110521F0A8
:109C3000D8018C9182FD86C08FEF8F0D8F70F82E2A
:109C4000589EC0011124FC01EA52F44FFEA7EDA773
:109C50000115110521F448010DA51EA5E3CF8114BE
:109C60009104C9F3D8019B967C909B979C96CC90CD
:109C70009C979D96DC909D979E96EC909E979796CC
:109C80002D913D914D915C919A97672D7C2D8D2D55
:109C90009E2D0E9483E98823F1F2F801608061FC27
:109CA00042C0D40197968D909D90AD90BC909A97AC
:109CB000A5019401672D7C2D8D2D9E2D0E9483E999
:109CC00018168CF5A5019401C501B4010E94E9E9BB
:109CD0004B015C01F80183A994A9A5A9B6A9BC010F
:109CE000CD0190589B01AC010E943DF0D8019F9698
:109CF0002D913D914D915C91D2970E94E9E99B0194
:109D0000AC01C501B4010E943CF00E94EBF21B01C2
:109D10004C019B01AC01672D7C2D8D2D9E2D0E9449
:109D200083E987FF04C0272C3C2C8D2C9E2CC1017D
:109D3000D401F80187A390A7A1A7B2A7862D8160BF
:109D4000808389CF10915D12F12C00E080E090E0DB
:109D50002DE4E22E20915C122117C1F0E19E9001CA
:109D60001124A9014A52544F6A01009741F0DC01C5
:109D70002C9121FD04C06F2D702F0E948A401F5F1F
:109D80001F708F2D902FFC2C0D2DE4CF009741F0EC
:109D9000FC01208121FD04C06F2D702F0E948A409C
:109DA000F0905D1200E010E08DE4E82E8F2D0F2C76
:109DB000000C990B20915C1230E08217930709F494
:109DC0004EC0E89E9001E99E300D1124A9014A522F
:109DD000544F6A0101151105E1F1D8012C9120FDC4
:109DE00004C0FA01208120FF34C0D80193968D90E1
:109DF0009D90AD90BC909697E89EF001E99EF00D85
:109E00001124EA52F44FA501940167A170A581A520
:109E100092A50E9437F169A37AA38BA39CA3A50105
:109E20009401F80167A170A581A592A50E9437F160
:109E30006DA37EA38FA398A7AE014F5D5F4FBE01B8
:109E40006B5D7F4FC8010E94D576D8018C918E7FC3
:109E50008C9381E08F0D8F70F82E8601A7CF0115AE
:109E6000110569F1F801C3A0D4A0E5A0F6A0A701EF
:109E700096016DEC7CEC8CE49DE30E9437F169A3C4
:109E80007AA38BA39CA3A7019601D80197966D9105
:109E90007D918D919C919A970E9437F16DA37EA33D
:109EA0008FA398A7AE014F5D5F4FBE016B5D7F4FE3
:109EB000C8010E94D576F80180818E7F80838091D1
:109EC0006F00826080936F001AC020902411309040
:109ED000251100912611109127119101A80169A562
:109EE0007BAD8CAD9EAD0E9483E987FF02C00C94D0
:109EF000E34529A43BAC0CAD1EAD0C94E345CA5818
:109F0000DF4F0FB6F894DEBF0FBECDBFDF91CF910C
:109F10001F910F91FF90EF90DF90CF90BF90AF9087
:109F20009F908F907F906F905F904F903F902F9079
:109F30000895CF93DF9300D000D0CDB7DEB788234C
:109F400019F00E9410B20FC088EB91E09C838B83C4
:109F500084E190E09A838983BE016D5F7F4FCE01DB
:109F600001960E94D6CB0F900F900F900F90DF912B
:109F7000CF9108958091A1098630D8F496E0899F09
:109F8000F0011124E358F64F2091870130918801A8
:109F9000318320834091FB155091FC156091FD1594
:109FA0007091FE1542835383648375838F5F809322
:109FB000A109089520918701309188012817390758
:109FC000D9F090938801809387014093FB155093BB
:109FD000FC156093FD157093FE15855A904521F48C
:109FE0001092DD111092A10982E080938F0181E02F
:109FF000809385111092E311089540E050E0BA017A
:10A0000085EA90E50C94DA4FE091A109EE2389F0FE
:10A01000E150E093A10986E0E89FF0011124E358A4
:10A02000F64F4281538164817581808191810C94C6
:10A03000DA4F0C94FD4F9CE0899F802D112491E014
:10A04000980F90931A162CE0280F20931B1640911E
:10A05000321250E030E02E5F3F4F24173507CCF02E
:10A06000292F30E04091341250E0241735078CF44A
:10A07000662341F08E5F0E9404CD80911B168E5F97
:10A080000E9404CD80911B161092351280933612D7
:10A09000089508950F931F93CF93DF931F92CDB729
:10A0A000DEB780913712811105C081E080933712AD
:10A0B0000E94A8BC609100127091011219829E0149
:10A0C0002F5F3F4F4FE08EEF91E10E94D4AE809121
:10A0D0001601882331F1109216018091FE1190E053
:10A0E0008058910997FD019695958795182F0E94A4
:10A0F0000FBD00E420E840E0612F8EEF91E10E9467
:10A10000F3AE882339F027E33BE040E460E0812FA1
:10A110000E9442BD84E00E9419D60E9407BC8111B2
:10A12000E8CF0F90DF91CF911F910F910895CF93BA
:10A13000DF93EC01FE018491882321F00E944BD62D
:10A140002196F8CFDF91CF9108952F923F924F92B1
:10A150005F927F928F929F92AF92BF92CF92DF9247
:10A16000EF92FF920F931F93CF93DF93CDB7DEB79C
:10A170002A970FB6F894DEBF0FBECDBF1092E21142
:10A180008091E411882351F00E944A5040E050E051
:10A19000BA0189EF96E50E94DA4FF8C44091FB15A9
:10A1A0005091FC156091FD157091FE1520911A01DA
:10A1B00030911B01C901840F951F2436310524F409
:10A1C000853691053CF416C02436310531F08436CD
:10A1D000910584F484E690E00DC047305105610597
:10A1E000710514F0069706C04A3F5F4F6F4F7F4FCF
:10A1F0006CF4069690931B0180931A011092FB1544
:10A200001092FC151092FD151092FE1580911A0106
:10A2100090911B018A3091053CF0883E23E0920723
:10A220002CF087EE93E002C08AE090E090931B014F
:10A2300080931A010E946ABA182F0E9484B28091FA
:10A240003212853108F5112359F080911016909142
:10A250001116892B29F0B0E9EB2EB0E1FB2E04C0DA
:10A26000A0E6EA2EAFE0FA2E03E120E841E060E04C
:10A270008EEF91E10E94F3AE882331F0970143E124
:10A2800061E080E00E9442BD809132128D3108F081
:10A290007DC1883008F041C080917C091123D9F13B
:10A2A00060912E0770912F07072E000C880B990BD9
:10A2B0000E948AE920E030E040E05FE30E943DF048
:10A2C0000E94A9F19B01643671051CF52A30310505
:10A2D000F4F04CE022E130E0241B310937FF02C0EA
:10A2E0002F5F3F4F359527953195219531092A5D8F
:10A2F0002093351227E020933612CB010E94B6B18D
:10A300000E9460D68DE59FE00E94975006C046E00F
:10A31000E1CF42E1DFCF882319F2809132128D31F3
:10A32000D0F5809134128531B0F120E030E040E08A
:10A330005FE36091C5117091C6118091C711909132
:10A34000C8110E943DF00E94A9F19B01643671057D
:10A350000CF001C32A3031050CF4FBC24CE022E1C1
:10A3600030E0241B310937FF02C02F5F3F4F359586
:10A3700027953195219531092A5D209335122CE1DD
:10A3800020933612CB010E94B6B10E9460D68DE5B3
:10A390009FE00E94975080913212853108F580919C
:10A3A00034128131E8F060912E0770912F07072E4B
:10A3B000000C880B990B0E948AE92091C5113091FD
:10A3C000C6114091C7115091C8110E949DF21816F4
:10A3D0000CF4C3C222E042E061E18EE20E9463CD50
:10A3E00080913212883008F03FC080917B091111B2
:10A3F00002C0811139C060910E1670910F16072EA0
:10A40000000C880B990B0E948AE920E030E040E0C4
:10A410005FE30E943DF00E94A9F1643671052CF4BF
:10A420006A30710524F446E003C042E101C04CE00B
:10A4300022E130E0241B310937FF02C02F5F3F4F7C
:10A4400035952795319521953109285B2093351253
:10A4500027E020933612CB010E94B6B10E9460D64D
:10A460008DE59FE00E949750809132128D31D0F59A
:10A47000809134128531B0F120E030E040E05FE3BC
:10A4800060917709709178098091790990917A09A2
:10A490000E943DF00E94A9F19B01643671050CF009
:10A4A0006AC22A3031050CF064C246E022E130E095
:10A4B000241B310937FF02C02F5F3F4F3595279589
:10A4C000319521953109285B209335122CE1209399
:10A4D0003612CB010E94B6B10E9460D68DE59FE096
:10A4E0000E94975080913212853130F5809134125C
:10A4F000813110F160910E1670910F16072E000C2D
:10A50000880B990B0E948AE920917709309178098C
:10A510004091790950917A090E949DF218160CF029
:10A520002CC210921E1222E042E062E18FE40E94EF
:10A5300063CD81E080931E12809132128C3130F510
:10A5400080913412843110F180911016909111167F
:10A55000019644E6489F9001499F300D112437FF32
:10A5600002C021503F4F832F932F990F990B0097D3
:10A5700069F028E6209335122BE1209336120E94D1
:10A58000B6B10E9460D685E20E9441BC8091321231
:10A59000843328F4809134128A3208F0F5C1809116
:10A5A0003212853328F480913412813308F010C2BE
:10A5B00080918C12882309F449C08091321284332F
:10A5C00008F044C080913412823308F43FC02091D7
:10A5D0005A14222319F18091231590912415A091EA
:10A5E0002515B09126150097A105B10509F4F7C10D
:10A5F000BC01CD016D597F4F8F4F9F4F24E630E056
:10A6000040E050E00E94D9EF609127157091281525
:10A610008091291590912A150E94D9EF85E3289FF2
:10A62000B0011124072E000C880B990B0E948AE9B7
:10A630002AE037ED43E25CE30E94E9E90E94B0F1D1
:10A64000462F22E062E387E30E9463CD80913212BD
:10A65000813308F079C080913412893208F474C0D3
:10A660000E9419604B015C0120E13EE040E050E0B7
:10A670000E94D9EF722E032FE22EF32E8CE3282EA8
:10A68000312C412C512CC501B401A20191010E9431
:10A69000D9EFCA01B901A20191010E94D9EFCE01FF
:10A6A00001966C0191E8891691E5990691E0A90659
:10A6B000B10408F496C17F936F93C70168E170E01D
:10A6C0000E944AF39F938F93C501B40120E831E5BE
:10A6D00041E050E00E94D9EF3F932F9389E49FE03F
:10A6E0009F938F93DF92CF920E941BE90FB6F8944D
:10A6F000DEBF0FBECDBF8CE38093351280E3809325
:10A700003612C6010E9460D68091290790912A07CF
:10A71000A0912B07B0912C07892B8A2B8B2B09F446
:10A72000A2C120915A14211179C188E68093351273
:10A7300083E380933612822F90E00E94B6B10E948C
:10A7400051CD85E20E9441BCE091F811F091F911E0
:10A7500084818111CCC060917B1870917C188091AC
:10A760007D1890917E180E94A9F1CB010E9435B10D
:10A77000BC018EEA99E00E94DEF360917F1870912F
:10A78000801880918118909182180E94A9F1CB01C4
:10A790000E9435B1BC0189EA99E00E94DEF32CEAFF
:10A7A00035EC47E257E360918318709184188091EB
:10A7B0008518909186180E943DF020E030E048EC2A
:10A7C00052E40E94E9E90E94A9F16B017C0197FD26
:10A7D00019C090E1C91697E2D906E104F104E4F04A
:10A7E000C701B60120E137E240E050E00E94FBEFF4
:10A7F000CA01B9012AE030E040E050E00E94FBEFDE
:10A80000605D0BC0F094E094D094C094C11CD11C46
:10A81000E11CF11C6DE201C060E26093131628EEAA
:10A82000C21623E0D206E104F10494F0C701B60198
:10A8300028EE33E040E050E00E94FBEFCA01B9018E
:10A840002AE030E040E050E00E94FBEF605D01C094
:10A8500060E260931416C701B60124E630E040E0E0
:10A8600050E00E94FBEF9AE0892E912CA12CB12C94
:10A87000CA01B901A50194010E94FBEF605D6093DC
:10A880001516C701B601A50194010E94FBEF062F22
:10A89000662381F08EE280931616CA01B901A501E4
:10A8A00094010E94FBEF605D60931716005D0093BA
:10A8B000181617C0CA01B901A50194010E94FBEF47
:10A8C000662339F08EE280931616605D609317164A
:10A8D00005C080E2809317168093161680E280935D
:10A8E000181663E176E182EA99E00E94DEF3809136
:10A8F0003212883298F4809134128D3178F02BE046
:10A9000040E86DE180E00E941BCD809132128732D9
:10A9100028F4809134128F3108F0AEC08091321249
:10A92000823328F4809134128B3208F010C1809168
:10A930003212803408F02AC180913412883308F42E
:10A9400025C1109235128FE3809336120E9493BC7A
:10A950001DC146E004CD42E102CD10921E1222E05C
:10A9600042E061E18EE20E9463CD81E080931E129D
:10A9700037CD4CE09BCD42E199CD22E042E062E14F
:10A980008FE40E9463CDD8CD27E048E06AE28AE2F6
:10A990000E9463CD25E042E06CE282E30E9463CD39
:10A9A00024E04AE061E38AE20E941BCD609100123C
:10A9B0007091011282E380931A128BE280931B1232
:10A9C0002AE132E142E38EEF91E10E94D4AEE7CD7D
:10A9D00024E045E361E386E30E941BCDE9CD20E05E
:10A9E0001DCE94E6E916F10460F47F936F93C701DE
:10A9F00068E170E00E944AF39F938F938FE39FE09A
:10AA000006C07F936F930F937F9287E39FE09F939E
:10AA10008F93DF92CF920E941BE968CE809123151D
:10AA200090912415A0912515B09126150097A105A8
:10AA3000B105B9F0BC01CD016D597F4F8F4F9F4FCC
:10AA400024E630E040E050E00E94D9EF6091271505
:10AA5000709128158091291590912A150E94D9EF9F
:10AA600064CE20E062CE88E68093351283E3809343
:10AA7000361280E090E061CE83E08093351286E26A
:10AA800080933612112329F08BE59FE00E949750A6
:10AA90000DC080917409811102C08FE305C08091BF
:10AAA000B4038111F1CF80E20E9441BC8BE080931E
:10AAB000351206E2009336128EEA99E00E9460D6C3
:10AAC0008BE28093351200933612112329F089E529
:10AAD0009FE00E9497500DC080917509811102C0BE
:10AAE0008FE305C08091B5038111F1CF80E20E9410
:10AAF00041BC83E38093351206E20093361289EA63
:10AB000099E00E9460D683E5809335120093361257
:10AB1000112329F087E59FE00E9497500DC0809196
:10AB20007609811102C08FE305C08091B6038111BF
:10AB3000F1CF80E20E9441BC8BE58093351286E222
:10AB40008093361282EA99E00E9460D6E7CE84E0D4
:10AB50000E9419D683E08093351212E310933612C7
:10AB600086E00E944BD60E9484B28CE0809335121E
:10AB70001093361280911A0190911B010E94B6B178
:10AB80000E9460D685E20E9441BCD1CE2A960FB6C3
:10AB9000F894DEBF0FBECDBFDF91CF911F910F9113
:10ABA000FF90EF90DF90CF90BF90AF909F908F90ED
:10ABB0007F905F904F903F902F900895CF92DF92BB
:10ABC000EF92FF920F931F93CF93DF939C017B0132
:10ABD00080E090E0F901E80FF91FE491EE2311F015
:10ABE0000196F8CFF701AF014E195F09619161112C
:10ABF000FACF04E110E0041B11099927081719077F
:10AC00001CF0DD24D39402C082E0D82E8091FF1185
:10AC100090E06D2D70E06F5F7F4F0E945EF3C62E57
:10AC2000C6E0C60F80913212C81748F04091341226
:10AC300050E08C2F90E00B97481759078CF5D0E027
:10AC4000E114F104B1F18AE30E9441BC82E0D81220
:10AC50000FC0CC0D80913212C81758F120913412D8
:10AC600030E08C2F90E00B97281739071CF421C097
:10AC7000DD23F9F0802F880F080F000F00933512A5
:10AC8000C093361280E20E9441BCC701DF91CF9190
:10AC90001F910F91FF90EF90DF90CF900C9460D6B2
:10ACA00010923512C0933612C9010E949750D1E01C
:10ACB000C7CFDF91CF911F910F91FF90EF90DF9061
:10ACC000CF90089580E00C9444A40C94DBA340E062
:10ACD00050E0BA018AE796E50E94DA4F1092C40963
:10ACE0001092C5091092C6091092C70981E080939D
:10ACF000DD110895CF93DF9300D000D0CDB7DEB73C
:10AD00008091E411882329F01092DD110E940450F3
:10AD100069C04091FB155091FC156091FD15709133
:10AD2000FE154115510561057105B9F124E6249F11
:10AD3000C001259F900D11241092FB151092FC1557
:10AD40001092FD151092FE1521E020938F012091A5
:10AD5000B603222351F02091BF093091C009280F7A
:10AD6000391F3093C0092093BF09092E000CAA0B8C
:10AD7000BB0B4091C4095091C5096091C6097091FF
:10AD8000C709840F951FA61FB71F8093C40990930E
:10AD9000C509A093C609B093C70980918F01882384
:10ADA00009F16091C4097091C5098091C60990911B
:10ADB000C7090E948AE920913807309139074091EC
:10ADC0003A0750913B070E94E9E969837A838B83B4
:10ADD0009C83CE0101960E9487CDBC0181E093E166
:10ADE0000E94DE550F900F900F900F90DF91CF9142
:10ADF0000895CF92DF92EF92FF921F93CF93DF934C
:10AE00001092E2118091FB159091FC15A091FD1517
:10AE1000B091FE1581309048A105B10540F0109227
:10AE2000FB151092FC151092FD151092FE15C091A5
:10AE3000FB158091C3091816DCF4282F082E000C8E
:10AE4000330B215031094C2F0C2E000C550B42179F
:10AE5000530774F0CFEFC80F8C2F90E0A0E0B0E064
:10AE60008093FB159093FC15A093FD15B093FE15F0
:10AE70001092851180918611C81714F4C093861121
:10AE800080918611082E000C990B04962C2F0C2E05
:10AE9000000C330B8217930724F48CEF8C0F8093F4
:10AEA000861110918611D0E08AE5E82E82E1F82E15
:10AEB00098E7C92E92E1D92E11111BC08091E4119F
:10AEC000811105C080918F01882399F009C0C111BB
:10AED000F9CF0E94045080918511882399F3E3C132
:10AEE00081E0C11180E024E045EF52E16D2F0E9426
:10AEF00045B280915C1290915D12891B8F7011F5A3
:10AF000080918C1281111EC01130F9F48091E411EE
:10AF1000811105C080918F018823B9F10BC0C13028
:10AF2000C9F78AE293E70E94AFBA8091851188231E
:10AF300089F3B9C181E0C13009F080E023E048EE37
:10AF400052E120C0113009F491C11230F1F4809126
:10AF5000E411811105C080918F018823B1F00BC0ED
:10AF6000C230C9F78FE592E80E94AFBA809185118F
:10AF7000882389F398C181E0C23009F080E023E0A2
:10AF800040EE52E16D2F0E9445B280918D128823D0
:10AF900009F404C180915A14882309F4BEC0209199
:10AFA000B7033091B80380918C12121613060CF07F
:10AFB0005AC08823E9F01330C1F58091E411811162
:10AFC00006C080918F01882309F447C109C0C330AE
:10AFD000C1F70E9402DF80918511882391F363C13C
:10AFE00081E0C33009F080E020E244ED52E132C15B
:10AFF0001330D9F48091E411811106C080918F0142
:10B00000882309F42AC109C0C330C1F70E9491DF27
:10B0100080918511882391F346C181E0C33009F006
:10B0200080E020E247EC52E115C1143009F0F5C090
:10B030008091E411811106C080918F01882309F469
:10B040000CC109C0C430C1F70E943DDF8091851159
:10B05000882391F328C181E0C43009F080E020E228
:10B060004CEB52E1F7C08823E9F01330C1F5809131
:10B07000E411811106C080918F01882309F4EDC08D
:10B0800009C0C330C1F70E9402DF80918511882377
:10B0900091F309C181E0C33009F080E020E240EB88
:10B0A00052E1D8C01330D9F48091E411811106C067
:10B0B00080918F01882309F4D0C009C0C330C1F743
:10B0C0000E9491DF80918511882391F3ECC081E08B
:10B0D000C33009F080E020E243EA52E1BBC0143003
:10B0E00009F09BC08091E411811106C080918F010D
:10B0F000882309F4B2C009C0C430C1F70E943DDF03
:10B1000080918511882391F3CEC081E0C43009F08D
:10B1100080E020E24AE852E19DC01330E9F48091DA
:10B12000E411811106C080918F01882309F495C034
:10B130000BC0C330C1F78DE995E90E94AFBA809189
:10B140008511882381F3AFC081E0C33009F080E02E
:10B1500023E04CE752E17EC0143009F05EC08091DC
:10B16000E411811106C080918F01882309F475C014
:10B170000DC0C430C1F7D092D50BC092D40B0E9441
:10B180009B3680918511882371F38DC081E0C43096
:10B1900009F080E020E249E652E15CC01330E9F4B6
:10B1A0008091E411811106C080918F01882309F4F8
:10B1B00054C00BC0C330C1F78DE995E90E94AFBA06
:10B1C00080918511882381F36EC081E0C33009F03E
:10B1D00080E023E04EE552E13DC01430F1F480916F
:10B1E000E411811105C080918F018823B1F10DC058
:10B1F000C430C9F7F092D50BE092D40B0E949B3675
:10B2000080918511882379F34EC081E0C43009F024
:10B2100080E020E24CE452E11DC01530F1F4809151
:10B22000E411811105C080918F018823B1F00BC01A
:10B23000C530C9F787E198E90E94AFBA80918511BE
:10B24000882389F330C081E0C53009F080E023E035
:10B2500045E952E16D2F0E9445B2DF5F1F5FD53097
:10B2600009F02ACE86E08093C3091DC08091E411C5
:10B27000811106C080918F01882309F486CE0BC00E
:10B28000C130C1F784E19AE50E94AFBA809185117F
:10B29000882381F308C081E0C13009F080E023E019
:10B2A00040EF52E16FCEDF91CF911F91FF90EF9071
:10B2B000DF90CF9008951F93CF93DF931092E21108
:10B2C0008091FB159091FC15A091FD15B091FE1594
:10B2D00081309048A105B10540F01092FB15109205
:10B2E000FC151092FD151092FE15C091FB15809172
:10B2F000C2091816DCF4282F082E000C330B21503D
:10B3000031094C2F0C2E000C550B4217530774F0CB
:10B31000CFEFC80F8C2F90E0A0E0B0E08093FB153A
:10B320009093FC15A093FD15B093FE151092851116
:10B3300080918611C81714F4C093861180918611EC
:10B34000082E000C990B04962C2F0C2E000C330B9E
:10B350008217930724F48CEF8C0F80938611109141
:10B360008611D0E0111116C08091E411882331F0CC
:10B37000C11104C080918511811152C080918F014B
:10B38000882309F445C081E0C11180E020E248E350
:10B3900052E13BC01130E1F48091E411811105C00C
:10B3A00080918F018823A1F10BC0C130C9F70E94A1
:10B3B00091DF0E94FD4F80918511882389F330C071
:10B3C00081E0C13009F080E020E240E252E11DC09E
:10B3D0001230F1F48091E411811105C080918F0148
:10B3E0008823B1F00BC0C230C9F70E943DDF0E9434
:10B3F000FD4F80918511882389F312C081E0C2300E
:10B4000009F080E020E24DE252E16D2F0E9445B24A
:10B41000DF5F1F5FD53009F0A5CF83E08093C209BD
:10B42000DF91CF911F9108952F923F924F926F928B
:10B430007F928F929F92AF92BF92CF92DF92EF92C4
:10B44000FF920F931F93CF93DF931092E21180919D
:10B45000FB159091FC15A091FD15B091FE15813062
:10B460009048A105B10540F01092FB151092FC1513
:10B470001092FD151092FE15C091FB158091C80920
:10B480001816DCF4282F082E000C330B215031093C
:10B490004C2F0C2E000C550B4217530774F0CFEFB6
:10B4A000C80F8C2F90E0A0E0B0E08093FB15909344
:10B4B000FC15A093FD15B093FE1510928511809197
:10B4C0008611C81714F4C093861180918611082E36
:10B4D000000C990B04962C2F0C2E000C330B8217AA
:10B4E000930724F48CEF8C0F80938611D0918611F2
:10B4F000612C4424439487EE782E9FE2292E93E119
:10B50000392E00E613E128E6E22E23E1F22E3FE693
:10B51000C32E33E1D32E4DE7A42E43E1B42E53E8DE
:10B52000852E53E1952ED1111AC08091E41181111D
:10B5300006C080918F01882309F4B4C009C0C111ED
:10B54000F8CF0E94045080918511882391F3AEC1F9
:10B5500081E0C11180E024E04FE853E1A0C0D13088
:10B56000D1F58091E411811106C080918F0188236B
:10B5700009F498C011C0C130C1F727EE33E04AE0AA
:10B5800050E06AE171E089E893E10E94F1E0809186
:10B590008511882351F38AC183E08F937F921F9294
:10B5A0008AE08F938AE191E09F938F93BF92AF924D
:10B5B0009F928F926F9281E0C13009F080E08F936B
:10B5C0000E94EBDE8DB79EB70C960FB6F8949EBF27
:10B5D0000FBE8DBF67C0D23009F047C08091E41123
:10B5E000811106C080918F01882309F45BC01BC0C4
:10B5F000C230C1F74092E2111092DE111092DF11B9
:10B600001092E0111092E11122E636E544E051E09B
:10B610006EE277E086E793E10E94F3E28091851184
:10B62000882301F343C182E696E59F938F934F925F
:10B6300084E08F931F921F928EE297E09F938F93E7
:10B64000FF92EF92DF92CF926F9281E0C23009F0C9
:10B6500080E08F930E94EBDE8DB79EB70E960FB6FB
:10B66000F8949EBF0FBE8DBF1DC0D33009F447C0F4
:10B67000D43009F48CC0D53009F4D0C0D63091F460
:10B680008091E411811106C180918F01882351F0CE
:10B6900081E0C63009F080E023E044E253E1662D0A
:10B6A0000E9445B20E9493B2811120C0D730E1F4CC
:10B6B0008091E411811105C080918F018823A1F050
:10B6C00009C0C730C9F70E9457E0809185118823CF
:10B6D00099F3ECC081E0C73009F080E020E244E15A
:10B6E00053E1662D0E9445B288E001C087E0639473
:10B6F000DF5F95E0691217CF8093C809D7C08091AA
:10B70000E411811105C080918F01882359F21BC07B
:10B71000C330C9F74092E2111092DE111092DF118E
:10B720001092E0111092E11125E636E547E850E06D
:10B730006EE076E184E693E10E94F3E28091851168
:10B74000882309F3B3C085E696E59F938F931F92F4
:10B7500087E88F931F921F928EE096E19F938F93BD
:10B760008CE593E19F938F931F930F936F9281E0EA
:10B77000C33009F080E08F930E94EBDE8DB79EB757
:10B780000E960FB6F8949EBF0FBE8DBF8BCF8091E3
:10B79000E411811106C080918F01882309F482CFC2
:10B7A0001BC0C430C1F74092E2111092DE1110921A
:10B7B000DF111092E0111092E1112FEF30E040E024
:10B7C00050E060E176E182E593E10E94F1E0809152
:10B7D0008511882301F36AC01F928FEF8F931F9208
:10B7E0001F9280E196E19F938F938EE393E19F9365
:10B7F0008F9388E493E19F938F936F9281E0C4309D
:10B8000009F080E08F930E94EBDE8DB79EB70C9617
:10B810000FB6F8949EBF0FBE8DBF44CF8091E41148
:10B82000811106C080918F01882309F43BCF11C09C
:10B83000C530C1F727EE33E04AE050E068E171E03F
:10B8400089E393E10E94F1E080918511882351F30F
:10B850002DC083E08F937F921F928AE08F9388E1BF
:10B8600091E09F938F933F922F9284E393E19F9374
:10B870008F936F9281E0C53009F080E08F930E9432
:10B88000EBDE8DB79EB70C960FB6F8949EBF0FBE39
:10B890008DBF08CFC63009F0F7CE87E696E50E9447
:10B8A000AFBA80918511882309F4EECEDF91CF9154
:10B8B0001F910F91FF90EF90DF90CF90BF90AF90CE
:10B8C0009F908F907F906F904F903F902F90089512
:10B8D0008F929F92AF92BF92CF92DF92EF92FF92A0
:10B8E0001F93CF93DF93C82F80E394E19093D30B02
:10B8F0008093D20B10924C1482E090E0A0E0B0E074
:10B900008093351490933614A0933714B093381461
:10B910001092D10B1092CD0B1092CE0B1092CF0B38
:10B920001092D00B8FEF9FEFDC018093C90B9093A7
:10B93000CA0BA093CB0BB093CC0BCC2379F1C530C1
:10B9400008F0F8C040E060E070E0CB010E943CCF1E
:10B95000882309F4EFC020E1C29FC001112487545D
:10B96000964FFC01E254FE4F20812F7709F0E2C090
:10B970003C96408151816281738144365105610555
:10B98000710508F4D7C03497C080D180E280F3807D
:10B99000C114D104E104F10421F4CCC0C12CD12C98
:10B9A000760140E0C701B6010E943CCF182F8823E2
:10B9B00009F4C0C08091D4099091D50981159240B5
:10B9C00009F0B8C0A091D909AA2309F4B3C06091C5
:10B9D000D7097091D8096115710509F4ABC02091A0
:10B9E000D609222309F4A6C0A09347142093391442
:10B9F00080E030E041E050E0C82FFA01082E02C09C
:10BA0000EE0FFF1F0A94E2F72E173F0739F08F5F02
:10BA1000C83091F789E0809342148CC0809342141F
:10BA20002091DF093091E0092115310519F040E03E
:10BA300050E008C02091ED093091EE094091EF09E6
:10BA40005091F00920933A1430933B1440933C14E6
:10BA500050933D1446015701860E971EA11CB11C40
:10BA60008092481490924914A0924A14B0924B14B8
:10BA7000E091DA09F091DB09F0934E14E0934D1454
:10BA8000B0E00E941AF0860E971EA81EB91E809282
:10BA90004F1490925014A0925114B092521485E019
:10BAA000EE0FFF1F8A95E1F7E150FE4FEF2FFF27C2
:10BAB000E6958E0E9F1EA11CB11C8092431490929D
:10BAC0004414A0924514B09246142091DC093091A0
:10BAD000DD092115310521F0A90160E070E008C001
:10BAE0004091E9095091EA096091EB097091EC09E4
:10BAF000D701C60188199909AA09BB09840F951FA6
:10BB0000A61FB71F04C0B695A79597958795CA95A8
:10BB1000D2F780933E1490933F14A0934014B093B7
:10BB20004114853F2FE09207A105B10528F48CE070
:10BB300080934C1410E01AC0853F9F4FA105B105BA
:10BB400010F480E111C08091F5099091F609A0915F
:10BB5000F709B091F80980934F1490935014A09373
:10BB60005114B093521480E280934C14812FDF91D2
:10BB7000CF911F91FF90EF90DF90CF90BF90AF904B
:10BB80009F908F900895CF92DF92EF92FF920F9344
:10BB90001F93CF93DF93CDB7DEB7EDB6FEB6DC01D2
:10BBA0000D900020E9F79D01281B390B2C5F3F4FBA
:10BBB0004DB75EB7421B530B0FB6F8945EBF0FBE76
:10BBC0004DBF0DB71EB70F5F1F4F9F938F9381EF30
:10BBD00094E19F938F931F930F930E941BE9680139
:10BBE00054E0C50ED11C0F900F900F900F900F9046
:10BBF0000F90F6018081882349F0082E000C990BE4
:10BC00000E9487F3F60181936F01F3CFC8010E9470
:10BC100080BD8DEE94E19093D50B8093D40B0E9460
:10BC20009B360FB6F894FEBE0FBEEDBEDF91CF91EE
:10BC30001F910F91FF90EF90DF90CF900895AF92FA
:10BC4000BF92CF92DF92EF92FF920F931F93CF9309
:10BC5000DF93CDB7DEB7AA970FB6F894DEBF0FBE5D
:10BC6000CDBF8091B8128F938091B7128F9384EEDD
:10BC700094E19F938F937E0181E2E80EF11CFF9285
:10BC8000EF920E941BE90F900F900F900F900F9072
:10BC90000F9010E0F70101900020E9F73197EE19BD
:10BCA000FF091E1784F46701C10ED11C17FDDA9439
:10BCB000F6018081082E000C990B0E9487F3F60193
:10BCC00080831F5FE7CF8DEB92E10E941AA700E00F
:10BCD000CE0101966C018091C012823080F080917B
:10BCE000C5129091C612A091C712B091C8128F715F
:10BCF0009927AA27BB27892B8A2B8B2BF9F00111B7
:10BD000003C08FEF9FEF05C08091B7129091B812DA
:10BD100001969093B8128093B712AA960FB6F89432
:10BD2000DEBF0FBECDBFDF91CF911F910F91FF906E
:10BD3000EF90DF90CF90BF90AF90089540E050E03B
:10BD4000B6018DEB92E10E94F0D01816C4F6F60110
:10BD500001900020E9F731971E2F1C19115068F04F
:10BD60005601A10EB11C17FDBA94F501808190E037
:10BD70000E9487F3F5018083F1CF8A858E3709F41D
:10BD8000AACF45E050E0B701C6010E94E5F3892B38
:10BD900009F0A1CFC7010E94C35D01E09CCFCF9203
:10BDA000DF92EF92FF921F93CF93DF9310928D1249
:10BDB0008091C012882321F08DEB92E10E94BCA5F6
:10BDC00010923414109231148FE1809330140E9439
:10BDD0004BAEEB01A89561E0809130140E9463ADF9
:10BDE00080E394E10E941FA72698259A279A249A17
:10BDF0002C9A85E08093321482E58CBD1DBC1AE03C
:10BE00008FEF0E9424A71150D9F720E030E0A9015C
:10BE100060E080E394E10E9429A7182F80933314F7
:10BE2000813049F00E944BAE6C1B7D0B613D774029
:10BE300060F381E054C02AEA31E040E050E068E07D
:10BE400080E394E10E9429A782FF03C01093341479
:10BE50000EC014E00E944DC6809333141150D1F7E8
:10BE60008A3A11F082E03BC082E0809334148091E2
:10BE70003414823021F0C12CD12C760105C0C12CA4
:10BE8000D12CE12C80E4F82E20E030E0A90167E31A
:10BE900080E394E10E9429A7A701960169E280E36B
:10BEA00094E10E9429A780933314882349F00E94CB
:10BEB0004BAE6C1B7D0B613D774030F38AE00FC0C9
:10BEC00080913414823011F520E030E0A9016AE35A
:10BED00080E394E10E9429A7882351F088E08093B1
:10BEE000311480E394E10E941FA7E8E0F5E31AC053
:10BEF0000E944DC6807C803C19F483E0809334140A
:10BF00000E944DC60E944DC60E944DC680E394E13A
:10BF10000E941FA71092321481E00E94685C811178
:10BF200032C015C08491EF012196882321F00E9430
:10BF30009238FE01F7CFE6EDF4E18491EF0121960E
:10BF4000882309F457C00E949238FE01F6CF80E0A2
:10BF50000E94685C811117C0EFECF4E18491EF015D
:10BF60002196882321F00E949238FE01F7CFEBEB57
:10BF7000F4E18491EF012196882309F43BC00E94EB
:10BF80009238FE01F6CF65E374E18DEB92E10E94F9
:10BF900069A5811116C0EFECF4E18491EF012196BF
:10BFA000882321F00E949238FE01F7CFEAEAF4E1FB
:10BFB0008491EF0121968823E9F00E949238FE01D6
:10BFC000F7CF81E080938D12E8E0F5E38491EF01F3
:10BFD0002196882321F00E949238FE01F7CFEEE9E6
:10BFE000F4E18491EF012196882321F00E94923898
:10BFF000FE01F7CF8BE1EDEBF2E1AEEDB2E10190A6
:10C000000D928A95E1F78091BB129091BC129093AA
:10C01000DD128093DC1289EB92E19093D912809328
:10C02000D812DF91CF911F91FF90EF90DF90CF90CA
:10C0300008950F931F9380917C1290917D12019728
:10C0400019F40E944BAE08C060918612709187125D
:10C05000809188129091891200918212109183121E
:10C060002091841230918512601B710B820B930B0F
:10C0700028EE33E040E050E00E94D9EF80917E123C
:10C0800090917F12A0918012B0918112BC01CD01DC
:10C09000620F731F841F951F1F910F9108952F9298
:10C0A0003F924F925F926F927F928F929F92AF9248
:10C0B000BF92CF92DF92EF92FF920F931F93CF9395
:10C0C000DF93CDB7DEB7C057D1090FB6F894DEBF06
:10C0D0000FBECDBF7C013B014A012DB73EB7AF96E5
:10C0E0003FAF2EAFAF97AD961FAEAD972B0134E0AB
:10C0F000430E511C8E01015A1F4F80E490E08C0FBB
:10C100009D1F0496E1969FAF8EAFE197F301878163
:10C11000823008F45AC184859585A685B7858F71CC
:10C120009927AA27BB27892B8A2B8B2B09F04DC176
:10C130008CE992E1892B11F010929C124CE952E1AA
:10C14000BE016F5F7F4FC2010E94F0D018160CF045
:10C150003CC18C85982F9871903109F0AFC0209127
:10C16000301530913115215031092230310508F454
:10C17000A5C02DB63EB6BE016F5F7F4FC8010E94BD
:10C18000DCCEF7018081882341F0F7010190002087
:10C19000E9F73197EE19FF0902C0E1E0F0E0D801BC
:10C1A0000D900020E9F7E01BF10BEA0FFB1F319621
:10C1B0002DB73EB72E1B3F0B0FB6F8943EBF0FBEF8
:10C1C0002DBFEDB7FEB731965F01882311F0B7019F
:10C1D00002C06CE073E0C5010E94DEF3B801C50146
:10C1E0000E94BFF36CE073E0C5010E94BFF3CE0173
:10C1F000805C9F4F0E94F2CE21E0A801B201E1963F
:10C200008EAD9FADE1970E946BAB81112CC08091E8
:10C21000301590913115892B31F5E8E0F5E38491E3
:10C220006F012FEFC21AD20A882321F00E949238A0
:10C23000F601F5CFEAE8F4E184916F013FEFC31A0C
:10C24000D30A882321F00E949238F601F5CF6801C5
:10C25000F60181916F01882319F00E949238F8CF7E
:10C260008AE00E9492388BE1FE01EC5BFF4FDE0119
:10C27000959601900D928A95E1F724968EAD9FAD2B
:10C2800024979CA38BA32CE931E03AA329A340E097
:10C2900050E0BE016F5D7F4FC5010E944F60CE012F
:10C2A00081960E94C9C7CE01805C9F4F0E94C9C77A
:10C2B0000FB6F8943EBE0FBE2DBE28CF2981222393
:10C2C00009F483C0253E09F421CF2E3209F41ECF94
:10C2D00020919C122E3209F419CF8A7009F016CFE2
:10C2E00081E0903109F080E080938E12903141F02E
:10C2F0008985873409F00ACF8A858E3709F406CFFD
:10C3000080913015909131158130910521F068F0C0
:10C310000297A9F1FBCE80913215909133150196C9
:10C320009093331580933215F1CEBE016F5F7F4F2E
:10C330008FE892E10E94DCCE6701F60181916F01E6
:10C34000882319F00E949238F8CF8FE8C82E82E136
:10C35000D82EF60181916F01882319F00E9492383E
:10C36000F8CF80E20E9492386D8D7E8D8F8D98A1DE
:10C370004AE00E9499388AE00E949238C7CEBE01F6
:10C380006F5F7F4F8FE892E10E94DCCE81149104B1
:10C3900041F06FE872E1C4010E94ACF3892B69F4AB
:10C3A00014C0AD96FFADAD978F2F90E02091321560
:10C3B000309133158217930741F0AD962FADAD97AD
:10C3C0002F5FAD962FAFAD97A1CEAF962EAD3FADFF
:10C3D000AF970FB6F8943EBF0FBE2DBFC059DF4FC9
:10C3E0000FB6F894DEBF0FBECDBFDF91CF911F9186
:10C3F0000F91FF90EF90DF90CF90BF90AF909F9004
:10C400008F907F906F905F904F903F902F90089506
:10C41000EF92FF920F931F93CF93DF93CDB7DEB7C9
:10C420006F970FB6F894DEBF0FBECDBF7B0108ED4E
:10C4300012E12AED32E1F8013183208322E030E07D
:10C440003093311520933015909333158093321526
:10C450008EED92E10E941AA7F801808191812BE173
:10C46000FC013496DE01159601900D922A95E1F7B4
:10C47000FC01828193819C838B838CE991E09A8378
:10C480008983A701BE016F5F7F4F8BE792E00E9417
:10C490004F60CE0101960E94C9C76F960FB6F894FF
:10C4A000DEBF0FBECDBFDF91CF911F910F91FF90E7
:10C4B000EF9008956F927F929F92AF92BF92CF922A
:10C4C000DF92EF92FF920F931F93CF93DF93CDB73D
:10C4D000DEB7AC970FB6F894DEBF0FBECDBF20918C
:10C4E0008D12222309F4C3C1962E7C0180915A1427
:10C4F000882309F474C0442309F48EC180919114F7
:10C50000882329F1EFECF4E184918F010F5F1F4F35
:10C51000882321F00E949238F801F6CFE7E4F4E195
:10C5200084918F010F5F1F4F882321F00E94923862
:10C53000F801F6CF61E070E080E090E00E944839B9
:10C540008AE00E9492388EE394E10E94DBC786E97C
:10C5500094E10E94C8BAE8E0F5E384918F010F5F8F
:10C560001F4F882321F00E949238F801F6CFB701BF
:10C5700085E294E10E944D41609191148DE8689F9D
:10C58000B00111246A567B4E8AE194E10E944D412C
:10C5900040912715509128156091291570912A1501
:10C5A00084E194E10E94FA408AE00E9492388091EE
:10C5B000911494E0899FF0011124EE56FB4E4091B6
:10C5C0002715509128156091291570912A154083DF
:10C5D0005183628373838F5F809391140DC0109297
:10C5E000911482E0D82E1AC1B70187E094E10E942D
:10C5F0004D418AE00E94923810928C1280915A1418
:10C60000882321F087E594E10E94BCA5CE01019624
:10C610006C010E94F2CE89EB92E19093D912809343
:10C62000D812F70180818F3209F060C087010F5F57
:10C630001F4F09F461C06FE270E0C8010E94CAF3A5
:10C640005C01009709F459C00817190708F055C094
:10C650003C01601A710AA301B801CE0180960E94C4
:10C66000F3F3E0E2F0E0EC0FFD1FE60DF71D1082A2
:10C67000CE0180963C018C01F80181918F018823C5
:10C6800019F00E949238F8CF8AE00E9492386091A7
:10C69000D8127091D9126115710511F06C5F7F4F3E
:10C6A00021E0AE01405E5F4FCE0105960E946BAB6C
:10C6B000811116C0E3EFF3E184918F010F5F1F4FEB
:10C6C000882321F00E949238F801F6CFF30181917E
:10C6D0003F01882319F00E949238F8CF8EE286C07D
:10C6E000D092D912C092D8128501A1CF8AED92E1E1
:10C6F0009093D9128093D81287019091D81280918B
:10C70000D912692F782F992009F45AC06115710543
:10C7100011F06C5F7F4F21E0A80187E594E10E9452
:10C720006BAB882309F448C0809168149091691418
:10C73000A0916A14B0916B148093231590932415E3
:10C74000A0932515B0932615B80185EE93E10E94BC
:10C750004D414091231550912415609125157091FC
:10C7600026158DED93E10E94FA408AE00E949238EE
:10C7700010922715109228151092291510922A153B
:10C78000EEECF3E184917F019FEFE91AF90A882327
:10C7900021F00E949238F701F5CFB80180E090E0D7
:10C7A0000E94086280919C12882319F08CE992E122
:10C7B00001C0C80160E02AC0B8018AEB93E110C053
:10C7C0006115710511F06C5F7F4F26E5A80187E5C3
:10C7D00094E10E946BAB81110CC0B80186EA93E131
:10C7E0000E944D418EE20E9492388AE00E94923867
:10C7F0000FC081E080938A12B70184E993E10E941F
:10C800004D418AE00E94923860E0C8010E9425B341
:10C81000C6010E94C9C72BC0DD24D394E8E0F5E32C
:10C8200084918F010F5F1F4F882321F00E9492385F
:10C83000F801F6CFEFE0F4E184918F010F5F1F4F15
:10C84000882321F00E949238F801F6CFE1E0DE164D
:10C8500019F00EE013E002C004E113E0F801819149
:10C860008F01882309F4C0CE0E949238F7CFAC968E
:10C870000FB6F894DEBF0FBECDBFDF91CF911F91F1
:10C880000F91FF90EF90DF90CF90BF90AF909F906F
:10C890007F906F900895FF920F931F93CF93DF9334
:10C8A00090912101992309F440C0072FF62E182FEB
:10C8B000EFECF4E18491EF012196882321F00E94AE
:10C8C0009238FE01F7CFEF2DF02F8491EF012196E2
:10C8D000882321F00E949238FE01F7CFE9E0FDE1C4
:10C8E0008491EF012196882321F00E949238FE0165
:10C8F000F7CF17FD0FC0612F110F770B880B990B26
:10C900000E9448398AE0DF91CF911F910F91FF90EB
:10C910000C949238E4E0FDE18491EF0121968823A4
:10C9200021F00E949238FE01F7CFDF91CF911F9145
:10C930000F91FF9008954F925F926F927F928F9226
:10C940009F92AF92BF92CF92DF92EF92FF920F939E
:10C950001F93CF93DF93CDB7DEB728970FB6F89428
:10C96000DEBF0FBECDBF80919F11811117C02896E9
:10C970000FB6F894DEBF0FBECDBFDF91CF911F91F0
:10C980000F91FF90EF90DF90CF90BF90AF909F906E
:10C990008F907F906F905F904F9008950E942AA58E
:10C9A0000E944BAE2B013C0180917C09811117C084
:10C9B0008091B7109091B810A091B910B091BA10B1
:10C9C0000097A105B10559F0A3019201281B390B6D
:10C9D0004A0B5B0B57FD03C081E080937C0960919B
:10C9E0002E0770912F07072E000C880B990B0E94C1
:10C9F0008AE92091C5113091C6114091C71150911B
:10CA0000C81114E0812E912C08E2A02EB12CC12C6B
:10CA1000D12C7B018C016AEF70E188EF90E10E94DC
:10CA2000BAA28090C5119090C611A090C711B09085
:10CA3000C8116091B1037091B203072E000C880BEE
:10CA4000990B0E948AE99B01AC01C501B4010E94C7
:10CA50009DF218160CF008C1609104017091050157
:10CA6000072E000C880B990B0E948AE99B01AC01F0
:10CA7000C501B4010E9483E987FFF6C040912E07EB
:10CA800050912F075A83498320ED3CEC4CE45DE341
:10CA90006091B3107091B4108091B5109091B61060
:10CAA0000E94E9E96B017C012091EA103091EB10C2
:10CAB0004091EC105091ED10C501B4010E943CF082
:10CAC0009B01AC01C701B6010E94E9E96B017C0141
:10CAD00023E333E343E75FE36091E6107091E710EF
:10CAE0008091E8109091E9100E94E9E99B01AC0166
:10CAF000C701B6010E943DF06B017C016093E61016
:10CB00007093E7108093E8109093E9108092EA10F8
:10CB10009092EB10A092EC10B092ED1080917C09F5
:10CB2000811189C1A981BA81BD01BB0F880B990B05
:10CB30000E948AE9A50194010E943CF04B015C012E
:10CB400020E030E040E251E40E949DF218160CF41F
:10CB500078C120E030E040E251ECC501B4010E9410
:10CB600083E987FD68C129813A81232B09F463C1D8
:10CB70008091E51081116AC18091E1109091E210DD
:10CB8000A091E310B091E41089839A83AB83BC83B6
:10CB90002091AF103091B0104091B1105091B2106F
:10CBA000C501B4010E94E9E96D837E838F83988774
:10CBB000A501940169817A818B819C810E943DF05D
:10CBC00069837A838B839C836093E1107093E21076
:10CBD0008093E3109093E4102091AB103091AC104F
:10CBE0004091AD105091AE100E94E9E92D813E8137
:10CBF0004F8158850E943DF0A70196010E943CF0AC
:10CC00006B017C0120E030E04FE753E40E949DF28D
:10CC100020E030E0A90118160CF41FC1C701B601CD
:10CC20000E9483E987FD07C0C701B6010E94A9F1F0
:10CC3000759567951AC020E030E0A901C501B401DF
:10CC40000E9483E987FF10C0A501940169817A8160
:10CC50008B819C810E943CF06093E1107093E21004
:10CC60008093E3109093E41060E06093A1118091B1
:10CC7000921190919311A0919411B09195110097F8
:10CC8000A105B10509F1A3019201281B390B4A0B3B
:10CC90005B0B57FD19C0609196117091971180E060
:10CCA00090E00E9488E99B01AC016091C5117091F0
:10CCB000C6118091C7119091C8110E9483E987FD28
:10CCC000B2C080E00E9444A4809198119091991183
:10CCD000A0919A11B0919B110097A105B10529F17E
:10CCE000A3019201281B390B4A0B5B0B57FD1DC09A
:10CCF00060919C1170919D1180E090E00E9488E904
:10CD00009B01AC0160917709709178098091790954
:10CD100090917A090E9483E987FF82C047E25DE132
:10CD200066E37DE18FEF0E944B648091F410909157
:10CD3000F510A091F610B091F710A3019201281BF5
:10CD4000390B4A0B5B0B57FD12CE38E8430E33E12B
:10CD5000531E611C711C4092F4105092F5106092A9
:10CD6000F6107092F71060910E1670910F16072E44
:10CD7000000C880B990B0E948AE920917709309169
:10CD800078094091790950917A09E2E08E2E912C30
:10CD9000F4E1AF2EB12CCC24CA94DC2C7B018C01A5
:10CDA0006EEE70E182EF90E10E94BAA280917B0961
:10CDB000811132C0C0907709D0907809E09079094C
:10CDC000F0907A0920E030E040EA50E4C701B60173
:10CDD0000E949DF287FD20C020E030E046E153E450
:10CDE000C701B6010E9483E91816B4F060910E16CF
:10CDF00070910F16072E000C880B990B0E948AE980
:10CE00009B01AC01C701B6010E9483E987FD17C0F1
:10CE100080E08093A011ABCD1092A0115C98A7CDBB
:10CE20000E94DBA382CF45E45DE164E57DE180E023
:10CE30000E944B6449CF81E08093E51015CF8FE7C6
:10CE4000E8CF81E08093E5106FE70FCF1092E510F7
:10CE500019821A821B821C829BCEC501B4010E94DA
:10CE60009DF218168CF7A501940169817A818B8156
:10CE70009C810E943CF06093E1107093E2108093DB
:10CE8000E3109093E4106FE7F0CE880F991F880F9E
:10CE9000991FFC01E559F74E4081518162817381F0
:10CEA000FC01E05CF84F4083518362837383E0911F
:10CEB000A910F091AA1082899389A489B5898093D9
:10CEC000DD109093DE10A093DF10B093E010089572
:10CED000CF93DF932FB7F894AC01440F551F440F45
:10CEE000551FFA01E559F74E608171818281938166
:10CEF0002FBFEA01C05DD84F0E948AE9288139819D
:10CF00004A815B810E94E9E9DF91CF910895909178
:10CF10005C1280915D12981721F080E00E9444C855
:10CF2000F6CF08958091A61080FF03C0459A8FEF39
:10CF300002C0459881E080931C018091A61081FF7A
:10CF400003C0479A8FEF02C0479881E080931D018C
:10CF50008091A61082FF03C02A988FEF02C02A9A00
:10CF600081E080931E018091A61083FF03C0289A60
:10CF70008FEF02C0289881E080931F01089590915F
:10CF80005C1280915D12981731F080915D128F5F75
:10CF90008F7080935D1208951F920F920FB60F92BB
:10CFA00011240BB60F92BF92CF92DF92EF92FF92B5
:10CFB0000F931F932F933F934F935F936F937F93A1
:10CFC0008F939F93AF93BF93EF93FF93CF93DF9391
:10CFD000CDB7DEB72697DEBFCDBF80916E008B7FC9
:10CFE00080936E0080916F008D7F80936F007894A6
:10CFF000C090D910D090DA10E090DB10F090DC10E7
:10D00000C114D104E104F104F1F18091B303882348
:10D01000D1F10E94A47809EBC0160BE0D006E10420
:10D02000F10488F018EBC11A1BE0D10AE108F108FD
:10D03000C092D910D092DA10E092DB10F092DC109E
:10D0400088EB9BE009C0C6011092D9101092DA104B
:10D050001092DB101092DC1090938900809388006E
:10D060002091880030918900809184009091850002
:10D0700040962817390708F058C68091840090918F
:10D080008500409611C22091A7103091A8103A83D4
:10D09000298321153105E9F0215031093A8329838B
:10D0A0003093A8102093A7101092AA101092A910E4
:10D0B0000E94BF6709811A81012B41F488EF9CE12E
:10D0C0009093D50B8093D40B0E949B3688EC90E014
:10D0D000EBC10091A9101091AA100115110509F0DA
:10D0E000E8C190915C1280915D12981761F10091F6
:10D0F0005D122DE4029F80011124F801EA52F44FE1
:10D10000C090D911D090DA11E090DB11F090DC11D1
:10D11000CF01875B9F4FDC014D915D916D917C91BB
:10D12000D701C601841B950BA60BB70B8093D911B1
:10D130009093DA11A093DB11B093DC1180818860A9
:10D1400080838F010BC08FB7F8941092D911109281
:10D15000DA111092DB111092DC118FBF1093AA101C
:10D160000093A9100115110509F49CC1F80152A101
:10D170008091A610418158130AC0242F30E080917D
:10D180002001082E000C990B2817390731F0509315
:10D19000A610409320010E9492671092D510109221
:10D1A000D6101092D7101092D810D801D7960D90A3
:10D1B000BC91A02DBA83A983A134ECE9BE0720F469
:10D1C000A132BE4478F004C020E43CE93A832983CC
:10D1D00049815A8156954795569547955A83498373
:10D1E00084E00BC089819A818131A7E29A0740F0DF
:10D1F000969587959A83898382E08093D4100BC09B
:10D2000081E08093D410E981FA81B09720F420E284
:10D2100030E03A83298349815A81405251095A8327
:10D220004983411568E05607F0F0E52FFF27EE0F20
:10D23000FF1FEE0FFF1FCF018850974EFC01329663
:10D2400045915491B981AA27B59F9001B49F210DB2
:10D250003A1F06942A1F3A1F1124FC0185919491CC
:10D26000821B930B22C089819A81969587958C7F2A
:10D2700088509B4EFC0125913491FC0132964591DA
:10D28000549169817A8167707727649FC001659F97
:10D29000900D749F900D112453E0969587955A95A3
:10D2A000E1F7F901E81BF90BCF018436910590F401
:10D2B0003AE1E32E33E0F32ED7018D917D018823EF
:10D2C00019F00E949238F8CF89819A810E94BCBAE5
:10D2D00084E690E09093D3108093D2108091D41084
:10D2E0008093D110F80103ACF4ADE02DFA83E9830B
:10D2F000F093D010E093CF10E1342CE9F20720F442
:10D30000E132FE4478F004C040E45CE95A8349838A
:10D3100089819A8196958795969587959A83898331
:10D3200084E00BC0A981BA81A131E7E2BE0740F0D9
:10D33000B695A795BA83A98382E08093D4100CC0D8
:10D3400081E08093D41029813A812032310520F484
:10D3500040E250E05A83498389819A8180979A8379
:10D3600089838115A8E09A07F0F0E92FFF27EE0FD7
:10D37000FF1FEE0FFF1FCF018850974EFC01329622
:10D3800045915491B981AA27B59F9001B49F210D71
:10D390003A1F06942A1F3A1F1124FC01859194918B
:10D3A000821B930B22C089819A81969587958C7FE9
:10D3B00088509B4EFC0125913491FC013296459199
:10D3C000549169817A8167707727649FC001659F56
:10D3D000900D749F900D112473E0969587957A9522
:10D3E000E1F7F901E81BF90BCF018436910590F4C0
:10D3F0005AE1E52E53E0F52ED7018D917D0188236A
:10D4000019F00E949238F8CF89819A810E94BCBAA3
:10D4100084E690E0AC0160E070E04093CB10509364
:10D42000CC106093CD107093CE10909389008093B0
:10D430008800F80182899389A489B589B695A79552
:10D4400097958795B095A095909581959F4FAF4FF3
:10D45000BF4F8093C7109093C810A093C910B0938A
:10D46000CA108093C3109093C410A093C510B093BA
:10D47000C6108093BF109093C010A093C110B093BA
:10D48000C2108093BB109093BC10A093BD10B093BA
:10D49000BE101092DD101092DE101092DF1010926C
:10D4A000E01007C080ED97E090938900809388009A
:10D4B0003CC48091B30381110E94A4782091D410C0
:10D4C000222309F4A1C1E091A910F091AA10428190
:10D4D0005381648175818091BB109091BC10A091A3
:10D4E000BD10B091BE10840F951FA61FB71F80936B
:10D4F000BB109093BC10A093BD10B093BE10181633
:10D5000019061A061B060CF45F9AE091A910F09117
:10D51000AA1046815781608571858091BF109091D6
:10D52000C010A091C110B091C210840F951FA61F0A
:10D53000B71F8093BF109093C010A093C110B093F9
:10D54000C210181619061A061B060CF4469AE0912A
:10D55000A910F091AA104285538564857585809144
:10D56000C3109091C410A091C510B091C610840F43
:10D57000951FA61FB71F8093C3109093C410A0934C
:10D58000C510B093C610181619061A061B060CF41F
:10D590002B9AE091A910F091AA10468557856089D1
:10D5A00071898091C7109091C810A091C910B09155
:10D5B000CA10840F951FA61FB71F8093C7109093A2
:10D5C000C810A093C910B093CA10181619061A06ED
:10D5D0001B060CF4299A8091BB109091BC10A0916D
:10D5E000BD10B091BE10181619061A061B0684F558
:10D5F000E091A910F091AA10428953896489758934
:10D60000841B950BA60BB70B8093BB109093BC109B
:10D61000A093BD10B093BE1080911C0140916B1877
:10D6200050916C1860916D1870916E18082E000C56
:10D63000990BAA0BBB0B840F951FA61FB71F8093D6
:10D640006B1890936C18A0936D18B0936E185F9838
:10D650008091BF109091C010A091C110B091C210E4
:10D66000181619061A061B0684F5E091A910F09108
:10D67000AA104289538964897589841B950BA60B6E
:10D68000B70B8093BF109093C010A093C110B093BC
:10D69000C21080911D0140916F18509170186091D7
:10D6A000711870917218082E000C990BAA0BBB0B05
:10D6B000840F951FA61FB71F80936F189093701843
:10D6C000A0937118B093721846988091C3109091EE
:10D6D000C410A091C510B091C610181619061A06EC
:10D6E0001B0684F5E091A910F091AA104289538994
:10D6F00064897589841B950BA60BB70B8093C310A7
:10D700009093C410A093C510B093C61080911E01D1
:10D710004091731850917418609175187091761833
:10D72000082E000C990BAA0BBB0B840F951FA61F8C
:10D73000B71F8093731890937418A0937518B093C3
:10D7400076182B988091C7109091C810A091C9109D
:10D75000B091CA10181619061A061B0684F5E09136
:10D76000A910F091AA104289538964897589841B94
:10D77000950BA60BB70B8093C7109093C810A0937E
:10D78000C910B093CA1080911F0140917718509131
:10D7900078186091791870917A18082E000C990BFE
:10D7A000AA0BBB0B840F951FA61FB71F809377187A
:10D7B00090937818A0937918B0937A18299880914B
:10D7C000DD109091DE10A091DF10B091E010019675
:10D7D000A11DB11D8093DD109093DE10A093DF108A
:10D7E000B093E0102150E091A910F091AA10428965
:10D7F00053896489758984179507A607B70708F4C4
:10D800005FCEBB24B39401C0B12CE091A910F0917C
:10D81000AA108091DD109091DE10A091DF10B091E0
:10D82000E01046895789608D718D481759076A073E
:10D830007B0708F416C14091CB105091CC10609139
:10D84000CD107091CE10068D178D20A131A1AA2781
:10D85000419FB12D529FC001629F900D619F800D2D
:10D86000911D429FB00D811D9A1F519FB00D811DCA
:10D870009A1F609FB00D811D9A1F509FB10D8A1F86
:10D880009A1FB6958A1F9A1F349F800D911D359F50
:10D89000900D112423AD34AD820F931F9093D010BF
:10D8A0008093CF1047A950AD61AD72ADA0E0B0E05C
:10D8B000481759076A077B0720F45093D01040930C
:10D8C000CF100091CF101091D0101A83098301342A
:10D8D0002CE9120720F401321E4478F004C040E421
:10D8E0005CE95A83498389819A81969587959695B3
:10D8F00087959A83898384E00BC0A981BA81A1317D
:10D90000E7E2BE0740F0B695A795BA83A98382E007
:10D910008093D4100CC081E08093D41009811A81C7
:10D920000032110520F420E230E03A832983098196
:10D930001A81005211091A830983011528E0120780
:10D94000E8F0E12FFF27EE0FFF1FEE0FFF1FCF01C3
:10D950008850974EFC01329625913491AA27039F57
:10D96000A001029F410D5A1F06944A1F5A1F1124FD
:10D97000FC0125913491241B350B20C089819A81AB
:10D98000969587958C7F88509B4EFC01259134910C
:10D99000FC0132964591549169817A8167707727AD
:10D9A000649FC001659F900D749F900D1124B3E09A
:10D9B00096958795BA95E1F7281B390B24363105E2
:10D9C00090F4FAE1EF2EF3E0FF2ED7018D917D0167
:10D9D000882319F00E949238F8CF89819A810E9499
:10D9E000BCBA24E630E08091B303882301F1C90179
:10D9F000293BBBE03B07E0F068EB7BE00E944AF389
:10DA0000883EE3E09E0718F48854944F02C088EBE8
:10DA10009BE0A901481B590B60E070E04093D910CE
:10DA20005093DA106093DB107093DC1001C0C901D1
:10DA300090938900809388008091CB109091CC10B6
:10DA4000A091CD10B091CE10820F931FA11DB11DDA
:10DA50008093CB109093CC10A093CD10B093CE10A8
:10DA600047C18091DD109091DE10A091DF10B09140
:10DA7000E010428D538D648D758D481759076A07E4
:10DA80007B0708F005C10091D5101091D6102091A8
:10DA9000D7103091D81009831A832B833C83468D8D
:10DAA000578D60A171A1AA27059FB12D169F700106
:10DAB000269FF00C259FE00CF11C069FB00DE11C89
:10DAC000FA1E159FB00DE11CFA1E249FB00DE11C3B
:10DAD000FA1E149FB10DEA1EFA1EB695EA1EFA1E32
:10DAE000709FE00CF11C719FF00C11248091CF10FD
:10DAF0009091D010FF96E816F90680F48E199F09D0
:10DB000040815181628173816C01E12CF12CC4163A
:10DB1000D506E606F70620F4CA0102C0808191818D
:10DB200081341CE9910728F481322EE4920748F0F1
:10DB300002C080E49CE9969587959695879524E0A8
:10DB400007C0813137E2930730F09695879522E040
:10DB50002093D41008C021E02093D4108032910586
:10DB600010F480E290E08C01005211091E830D83B5
:10DB7000011528E01207E8F0E12FFF27EE0FFF1F45
:10DB8000EE0FFF1FCF018850974EFC013296259172
:10DB90003491AA27039FA001029F410D5A1F0694AA
:10DBA0004A1F5A1F1124FC0125913491241B350B67
:10DBB00020C08D819E81969587958C7F88509B4E45
:10DBC000FC0125913491FC013296459154916D816F
:10DBD0007E8167707727649FC001659F900D749F59
:10DBE000900D112443E0969587954A95E1F7281BFF
:10DBF000390B2436310590F48AE1E82E83E0F82EC3
:10DC0000D7018D917D01882319F00E949238F8CFB9
:10DC10008D819E810E94BCBA24E630E08091B303DE
:10DC2000882301F1C901293BBBE03B07E0F068EB29
:10DC30007BE00E944AF3883EE3E09E0718F4885494
:10DC4000944F02C088EB9BE0A901481B590B60E090
:10DC500070E04093D9105093DA106093DB1070930A
:10DC6000DC1001C0C90190938900809388008981EC
:10DC70009A81AB81BC81820F931FA11DB11D80933E
:10DC8000D5109093D610A093D710B093D81030C071
:10DC90002091D2103091D3108091B303882301F1E9
:10DCA000293BFBE03F07E0F0C90168EB7BE00E9405
:10DCB0004AF3883E03E0900718F48854944F02C05A
:10DCC00088EB9BE0A901481B590B60E070E0409392
:10DCD000D9105093DA106093DB107093DC109C0124
:10DCE00030938900209388008091D1108093D410C4
:10DCF0002091880030918900809184009091850066
:10DD000040962817390748F4809184009091850047
:10DD100040969093890080938800BB2031F0109248
:10DD2000AA101092A9100E94BF67F8948091A211C6
:10DD3000882321F080916E008B7F03C080916E005C
:10DD4000846080936E0080916F00826080936F008A
:10DD500026960FB6F894DEBF0FBECDBFDF91CF91F0
:10DD6000FF91EF91BF91AF919F918F917F916F91B3
:10DD70005F914F913F912F911F910F91FF90EF90E5
:10DD8000DF90CF90BF900F900BBE0F900FBE0F9003
:10DD90001F9018951F93CF93DF931092E2118091FB
:10DDA000FB159091FC15A091FD15B091FE158130E9
:10DDB0009048A105B10540F01092FB151092FC159A
:10DDC0001092FD151092FE15C091FB158091141153
:10DDD0001816DCF4282F082E000C330B21503109C3
:10DDE0004C2F0C2E000C550B4217530774F0CFEF3D
:10DDF000C80F8C2F90E0A0E0B0E08093FB159093CB
:10DE0000FC15A093FD15B093FE151092851180911D
:10DE10008611C81714F4C093861180918611082EBC
:10DE2000000C990B04962C2F0C2E000C330B821730
:10DE3000930724F48CEF8C0F809386111091861138
:10DE4000D0E011111AC08091E411811106C08091B7
:10DE50008F01882309F462C009C0C111F8CF0E9464
:10DE6000045080918511882391F389C081E0C1110C
:10DE700080E024E046EC5EE14EC01130E9F4809190
:10DE8000E411811106C080918F01882309F446C0F6
:10DE90000BC0C130C1F78AE491E70E94AFBA80910C
:10DEA0008511882381F36BC081E0C13009F080E0E7
:10DEB00023E04FEB5EE12FC01230E1F48091E411DA
:10DEC000811105C080918F01882341F10BC0C230C0
:10DED000C9F780E591E70E94AFBA80918511882348
:10DEE00089F34DC081E0C23009F080E023E048EBC7
:10DEF0005EE111C0133029F58091E411811116C043
:10DF000080918F01882351F081E0C33009F080E0D7
:10DF100023E041EB5EE16D2F0E9445B2DF5F1F5FA2
:10DF2000D53009F08ECFD093141129C0C33041F7FA
:10DF300086E591E70E94AFBA80918511882301F3AD
:10DF40001EC0143059F78091E411811105C08091F1
:10DF50008F01882319F30BC0C430C9F78CE591E712
:10DF60000E94AFBA80918511882389F308C081E0AF
:10DF7000C43009F080E023E048EA5EE1CCCFDF91D5
:10DF8000CF911F910895EF92FF921F93CF93DF934C
:10DF90007C0170931311609312111092E211809121
:10DFA000FB159091FC15A091FD15B091FE158130E7
:10DFB0009048A105B10540F01092FB151092FC1598
:10DFC0001092FD151092FE15C091FB158091111154
:10DFD0001816DCF4282F082E000C330B21503109C1
:10DFE0004C2F0C2E000C550B4217530774F0CFEF3B
:10DFF000C80F8C2F90E0A0E0B0E08093FB159093C9
:10E00000FC15A093FD15B093FE151092851180911B
:10E010008611C81714F4C093861180918611082EBA
:10E02000000C990B04962C2F0C2E000C330B82172E
:10E03000930724F48CEF8C0F809386111091861136
:10E04000D0E081E091E0E916F10469F122E0E21606
:10E05000F10409F44CC0E114F10409F06CC0111191
:10E0600091C08823B1F01C16A4F08091FB1590910B
:10E07000FC15A091FD15B091FE150196A11DB11DD5
:10E080008093FB159093FC15A093FD15B093FE159E
:10E09000CF5F80918F01882309F4EEC021E041E039
:10E0A00061EA7EE16BC011116DC08823B1F01C16CE
:10E0B000A4F08091FB159091FC15A091FD15B091F5
:10E0C000FE150196A11DB11D8093FB159093FC15C3
:10E0D000A093FD15B093FE15CF5F80918F0188232B
:10E0E00009F4CAC021E041E06AE97EE147C01111AC
:10E0F00049C08823B1F01C16A4F08091FB159091C3
:10E10000FC15A091FD15B091FE150196A11DB11D44
:10E110008093FB159093FC15A093FD15B093FE150D
:10E12000CF5F80918F01882309F4A6C021E041E0F0
:10E1300063E97EE123C0111125C08823B1F01C16CC
:10E14000A4F08091FB159091FC15A091FD15B09164
:10E15000FE150196A11DB11D8093FB159093FC1532
:10E16000A093FD15B093FE15CF5F80918F0188239A
:10E1700009F482C021E041E06AE87EE18D2F0E942F
:10E18000A2E27AC01130D9F48091E411811106C065
:10E1900080918F01882309F46FC009C0C130C1F795
:10E1A0000E94045080918511882391F36DC081E015
:10E1B000C13009F080E024E040E85EE15AC012304E
:10E1C000E9F48091E411811106C080918F018823C8
:10E1D00009F452C00BC0C230C1F786E791E70E9434
:10E1E000AFBA80918511882381F34EC081E0C2309F
:10E1F00009F080E023E046E75EE13BC01330E1F444
:10E200008091E411811105C080918F018823A1F1D3
:10E210000BC0C330C9F78CE791E70E94AFBA809179
:10E220008511882389F330C081E0C33009F080E094
:10E2300023E04DE65EE11DC01430F1F48091E4115D
:10E24000811105C080918F018823B1F00BC0C430CB
:10E25000C9F782E891E70E94AFBA809185118823BF
:10E2600089F312C081E0C43009F080E023E042E687
:10E270005EE16D2F0E9445B2DF5F1F5F80E0D53009
:10E2800009F0E0CED0931111DF91CF911F91FF9053
:10E29000EF90089564E273E780E090E00C94C36F20
:10E2A0006EE173E781E090E00C94C36F68E173E77F
:10E2B00082E090E00C94C36F6EEB71E783E090E036
:10E2C0000C94C36F21E02093DD1160930D117093C6
:10E2D0000E1180930F119093101140E050E0BA019D
:10E2E00080911211909113110C94DA4F60E070E05C
:10E2F00080E291E40C94627160E070E080E89FE35A
:10E300000C9462716DEC7CEC8CEC9DE30C9462716E
:10E31000CF92DF92EF92FF92CF93C82F0E944BAE25
:10E320006B017C0124EA30E74DE75FE360910D115A
:10E3300070910E1180910F11909110110E9483E93C
:10E3400087FD05C08AEF90E0A0E0B0E003C080E068
:10E3500090E0DC01C80ED91EEA1EFB1EC092D5114A
:10E36000D092D611E092D711F092D811C093350116
:10E37000CF91FF90EF90DF90CF9008958091E411BE
:10E3800081110C9404506091FB157091FC158091E3
:10E39000FD159091FE15611571058105910569F1D5
:10E3A0000E948AE920910D1130910E1140910F11B8
:10E3B000509110110E94E9E9209187183091881836
:10E3C0004091891850918A180E943DF060938718F7
:10E3D000709388188093891890938A1883E090E04E
:10E3E0000E94887181E080938F011092FB1510923A
:10E3F000FC151092FD151092FE1580918F01882357
:10E4000049F087E898E10E94EDB0BC0189E59EE102
:10E410000C94DE5508952F923F924F925F926F9227
:10E420007F928F929F92AF92BF92CF92DF92EF92A4
:10E43000FF920F931F93CF93DF93CDB7DEB72A9749
:10E440000FB6F894DEBF0FBECDBF9A8789871B0138
:10E450008091E411882319F00E940450D0C080916B
:10E46000FB159091FC15A091FD15B091FE15892B1F
:10E470008A2B8B2B09F492C00E9487388101000FF0
:10E48000111F000F111FF801E558F74E4080518011
:10E490006280738080912E01811115C020E030E0F0
:10E4A0004AE754E4C301B2010E943CF04B015C0115
:10E4B00020E030E04AE754E4C301B2010E943DF09D
:10E4C0006B017C010EC0F801E250FF4E808091800C
:10E4D000A280B380F801EE5DFE4FC080D180E28063
:10E4E000F3808091FB159091FC15A091FD15B091E2
:10E4F000FE158D839E83AF83B887BC01CD010E943A
:10E500008AE920910D1130910E1140910F11509117
:10E5100010110E94E9E9A30192010E943DF09B01C4
:10E52000AC010558174ED8016D937D938D939C9344
:10E5300013978D819E81AF81B885B7FF0DC0C5014E
:10E54000B4010E949DF21816DCF4D8018D929D92C0
:10E55000AD92BC92139714C08D819E81AF81B88516
:10E56000892B8A2B8B2B61F0C701B6010E9483E9AE
:10E5700087FF06C0D801CD92DD92ED92FC921397F1
:10E580001092FB151092FC151092FD151092FE15BD
:10E59000C1010E94887181E080938F0180918F0179
:10E5A000882369F1F101EE0FFF1FEE0FFF1FE55801
:10E5B000F74E80819181A281B38189839A83AB8355
:10E5C000BC832DEC3CEC4CEC5DE360910D11709143
:10E5D0000E1180910F11909110110E949DF287FDF4
:10E5E00005C0CE0101960E94EDB004C0CE01019697
:10E5F0000E9487CDBC0189859A850E94DE552A96A6
:10E600000FB6F894DEBF0FBECDBFDF91CF911F9143
:10E610000F91FF90EF90DF90CF90BF90AF909F90C1
:10E620008F907F906F905F904F903F902F900895C4
:10E6300062E070E082E59EE10C940B7261E070E0B4
:10E640008BE49EE10C940B7260E070E084E49EE148
:10E650000C940B72AF92BF92CF92DF92EF92FF9227
:10E660000F931F93CF93DF931092E2118091FB15CC
:10E670009091FC15A091FD15B091FE158130904848
:10E68000A105B10540F01092FB151092FC151092F7
:10E69000FD151092FE15C091FB1580910C111816F6
:10E6A000DCF4282F082E000C330B215031094C2F9D
:10E6B0000C2E000C550B4217530774F0CFEFC80F08
:10E6C0008C2F90E0A0E0B0E08093FB159093FC15B8
:10E6D000A093FD15B093FE151092851180918611BF
:10E6E000C81714F4C093861180918611082E000C6F
:10E6F000990B04962C2F0C2E000C330B82179307CA
:10E7000024F48CEF8C0F80938611D091861100E059
:10E710008AE0E82E8EE1F82E9FECC92E9DE1D92EDD
:10E720002BECA22E2DE1B22ED1111AC08091E41152
:10E73000811106C080918F01882309F46BC009C044
:10E74000C111F8CF0E94045080918511882391F364
:10E7500037C181E0C11180E024E04FE35EE157C0A2
:10E76000D130E9F48091E411811106C080918F01CC
:10E77000882309F44FC00BC0C130C1F78AEC9EE674
:10E780000E94AFBA80918511882381F319C181E07D
:10E79000C13009F080E023E045E35EE138C0D230CB
:10E7A00021F58091E411811105C080918F018823AA
:10E7B00089F113C0C230C9F7B092D50BA092D40B27
:10E7C0000E949B365E9A1092B4035E9A1092B50333
:10E7D00080918511882349F3F3C081E0C23009F0AC
:10E7E00080E020E24BE25EE112C0D33009F0A6C027
:10E7F0008091E411811191C080918F01882351F0A3
:10E8000081E0C33009F080E020E24EE05EE1602F5D
:10E810000E9445B20E9493B2811105C080915A14A2
:10E82000882309F4ADC015E080910E1690910F1663
:10E83000892B31F480912E0790912F07892B21F19C
:10E840001D1321C08091E411811105C080918F01B9
:10E850008823C9F00FC0C113F9CF1092111610927E
:10E8600010160E9427A40E94FD4F809185118823D5
:10E8700069F3A6C081E0CD1380E020E240EE5DE1C7
:10E88000602F0E9445B21F5F1D131DC08091E411CF
:10E89000811105C080918F018823A9F00BC0C1139D
:10E8A000F9CF80EE95E70E94AFBA80918511882359
:10E8B00089F386C081E0CD1380E023E044ED5DE183
:10E8C000602F0E9445B281E0810FD8131DC0809156
:10E8D000E411811105C080918F018823A9F00BC03C
:10E8E000CD13F9CF8BEE94E70E94AFBA80918511DA
:10E8F000882389F365C081E0CD1380E023E04FE1F8
:10E900005EE1602F0E9445B20F5FDF5F053009F0C6
:10E910000BCF1E5F10930C1153C0C33009F06CCFA6
:10E92000D092D50BC092D40B0E949B360E94FD4F13
:10E9300080918511882309F45FCF42C0D43009F05B
:10E9400069CF8091E411811106C080918F018823E5
:10E9500009F460CF0DC0C430C1F7F092D50BE0923E
:10E96000D40B0E949B3680918511882371F328C0B7
:10E9700081E0C43009F080E020E249EF5DE147CF5B
:10E98000D530E1F48091E411811105C080918F01AF
:10E990008823A1F009C0C530C9F70E9457E08091D3
:10E9A0008511882399F30CC081E0C53009F080E01F
:10E9B00020E249EE5DE1602F0E9445B216E034CFBF
:10E9C000DF91CF911F910F91FF90EF90DF90CF904B
:10E9D000BF90AF9008951F93CF93DF931092E211F1
:10E9E0008091FB159091FC15A091FD15B091FE153D
:10E9F00081309048A105B10540F01092FB151092AE
:10EA0000FC151092FD151092FE15C091FB1580911A
:10EA10000B111816DCF4282F082E000C330B215094
:10EA200031094C2F0C2E000C550B4217530774F074
:10EA3000CFEFC80F8C2F90E0A0E0B0E08093FB15E3
:10EA40009093FC15A093FD15B093FE1510928511BF
:10EA500080918611C81714F4C09386118091861195
:10EA6000082E000C990B04962C2F0C2E000C330B47
:10EA70008217930724F48CEF8C0F809386111091EA
:10EA80008611D0E011111AC08091E411811106C0E5
:10EA900080918F01882309F474C009C0C111F8CF97
:10EAA0000E94045080918511882391F385C081E0F4
:10EAB000C11180E024E043EC5DE160C0113039F524
:10EAC0008091E411811106C080918F01882309F49F
:10EAD00058C015C0C130C1F7409122115091231187
:10EAE00060911A1170911B1180911E1190911F114C
:10EAF0000E94FCCD80918511882331F35DC081E0B7
:10EB0000C13009F080E020E247EB5DE137C0123010
:10EB100021F58091E411811105C080918F01882336
:10EB200081F113C0C230C9F74091221150912311D5
:10EB30006FEF7FEF80911E1190911F110E94FCCD0D
:10EB400080918511882349F337C081E0C23009F0F4
:10EB500080E020E247E95DE111C0133091F480913B
:10EB6000E411811117C080918F01882351F081E059
:10EB7000C33009F080E020E247EA5DE16D2F0E949A
:10EB800045B2DF5F1F5FD53009F07CCF84E0809312
:10EB90000B1112C0C33039F740912211509123114B
:10EBA00060911A1170911B1180E090E00E94FCCDE1
:10EBB000809185118823B9F2DF91CF911F9108953B
:10EBC0001F93CF93DF931092E2118091FB159091E8
:10EBD000FC15A091FD15B091FE1581309048A1055E
:10EBE000B10540F01092FB151092FC151092FD1526
:10EBF0001092FE15C091FB1580910A111816DCF4D5
:10EC0000282F082E000C330B215031094C2F0C2ECD
:10EC1000000C550B4217530774F0CFEFC80F8C2F21
:10EC200090E0A0E0B0E08093FB159093FC15A093DA
:10EC3000FD15B093FE151092851180918611C817AD
:10EC400014F4C093861180918611082E000C990B44
:10EC500004962C2F0C2E000C330B8217930724F4F0
:10EC60008CEF8C0F8093861110918611D0E01111DA
:10EC70001AC08091E411811106C080918F01882310
:10EC800009F474C009C0C111F8CF0E9404508091EA
:10EC90008511882391F385C081E0C11180E024E0D3
:10ECA0004FE85DE160C0113039F58091E4118111C8
:10ECB00006C080918F01882309F458C015C0C13067
:10ECC000C1F740912011509121116091181170915C
:10ECD000191180911C1190911D110E94FCCD809101
:10ECE0008511882331F35DC081E0C13009F080E0F7
:10ECF00020E243E85DE137C0123021F58091E41154
:10ED0000811105C080918F01882381F113C0C23029
:10ED1000C9F740912011509121116FEF7FEF809141
:10ED20001C1190911D110E94FCCD809185118823AA
:10ED300049F337C081E0C23009F080E020E243E6C9
:10ED40005DE111C0133091F48091E411811117C07D
:10ED500080918F01882351F081E0C33009F080E079
:10ED600020E243E75DE16D2F0E9445B2DF5F1F5F48
:10ED7000D53009F07CCF84E080930A1112C0C330F3
:10ED800039F7409120115091211160911811709123
:10ED9000191180E090E00E94FCCD809185118823BC
:10EDA000B9F2DF91CF911F9108954F925F926F92C8
:10EDB0007F928F929F92AF92BF92CF92DF92EF920B
:10EDC000FF920F931F93CF93DF93CDB7DEB76A9770
:10EDD0000FB6F894DEBF0FBECDBF9A8F898F5B014F
:10EDE0008A01DC01D7966D917D918D919C91DA9786
:10EDF0000E9488E96B017C01F5012081318142810B
:10EE000053810E94E9E90E941BF10E94B0F16987D9
:10EE10007A878B879C87D8012D913D914D915C918C
:10EE2000C701B6010E94E9E90E941BF10E94B0F1FE
:10EE30006D877E878F87988B29853A854B855C8582
:10EE4000283731054105510540F488E790E0A0E0FE
:10EE5000B0E089879A87AB87BC872D853E854F8533
:10EE60005889283731054105510540F488E790E07D
:10EE7000A0E0B0E08D879E87AF87B88BE98DFA8DD3
:10EE8000ED5BFF4F20813181428153812D833E8391
:10EE90004F835887CA01B9010E948AE969837A833E
:10EEA0008B839C8369857A858B859C850E9488E904
:10EEB000698B7A8B8B8B9C8B20E030E0A901698178
:10EEC0007A818B819C810E9483E9882339F1A70193
:10EED0009601C701B6010E94E9E94B015C0129894D
:10EEE0003A894B895C89CA01B9010E94E9E99B0111
:10EEF000AC01C501B4010E943CF04B015C012981C9
:10EF00003A814B815C81CA01B9010E943DF09B01AD
:10EF1000AC01C501B4010E9437F103C060E070E0AC
:10EF2000CB010E941BF10E94A9F12B013C016D81D4
:10EF30007E818F81988590958095709561957F4FA2
:10EF40008F4F9F4F0E948AE94B015C016D857E8542
:10EF50008F8598890E9488E96D837E838F83988747
:10EF600020E030E0A901C501B4010E9483E98823B3
:10EF700049F12D813E814F815885CA01B9010E9416
:10EF8000E9E96D8B7E8B8F8B988FA7019601C70166
:10EF9000B6010E94E9E99B01AC016D897E898F89E8
:10EFA000988D0E943CF06B017C01A5019401C50184
:10EFB000B4010E943DF09B01AC01C701B6010E9463
:10EFC00037F103C060E070E0CB010E94DFF1A98D52
:10EFD000BA8D52968D909D90AD90BC9055977501CD
:10EFE0006401C418D508E608F7080E94A9F1C61AFA
:10EFF000D70AE80AF90AF7FE6BC020E030E0A90161
:10F0000069817A818B819C810E9483E9882309F43C
:10F0100047C0C501B4010E9488E96B017C012981C8
:10F020003A814B815C81CA01B9010E943DF09B018C
:10F03000AC01C701B6010E94E9E96B017C01298995
:10F040003A894B895C89CA01B9010E94E9E99B01AF
:10F05000AC01C701B6010E943CF06B017C012D811F
:10F060003E814F815885CA01B9010E94E9E99B019F
:10F07000AC01C701B6010E943DF06B017C0120E0AC
:10F0800030E040E850E469817A818B819C810E9464
:10F09000E9E99B01AC01C701B6010E9437F103C049
:10F0A00060E070E0CB010E941BF10E94A9F12B01EE
:10F0B0003C0197FF03C0412C512C320148145904E4
:10F0C0006A047B0410F024013501C12CD12C760197
:10F0D0008FB7F894E98DFA8D908193FD1DC0468A13
:10F0E000578A608E718EC40CD51CE61CF71CC28E2C
:10F0F000D38EE48EF58E29853A854B855C8523AFCA
:10F1000034AF45AF56AFFF962D853E854F85588964
:10F1100020833183428353838FBF6A960FB6F8945E
:10F12000DEBF0FBECDBFDF91CF911F910F91FF903A
:10F13000EF90DF90CF90BF90AF909F908F907F9097
:10F140006F905F904F9008950F931F93CF93DF932D
:10F15000E091A910F091AA1082819381A481B581D8
:10F16000181619061A061B06E4F48091A61080FFF3
:10F1700018C096B18091171192FB992790F98E7F54
:10F18000892780931711909116119170892349F066
:10F1900080914C07816080934C0780E090E00E9452
:10F1A0004567E091A910F091AA1086819781A0850A
:10F1B000B185181619061A061B0614F58091A610BB
:10F1C00081FF1EC096B18091171193FB002700F9B3
:10F1D00010E01195019511090827027011270827E1
:10F1E00000931711809116118270082349F08091C5
:10F1F0004C07826080934C0781E090E00E94456755
:10F20000E091A910F091AA1082859385A485B58517
:10F21000181619061A061B061CF58091A61082FF07
:10F220001FC096B18091171192959170C92F90E0EF
:10F23000D92FD195C195D109C827C470DD27C8271A
:10F24000C0931711809116118470C82349F08091E2
:10F250004C07846080934C0782E090E00E944567F1
:10F260008091171180931611DF91CF911F910F910B
:10F270000895CF93DF93E5E5F1E28491EF012196C4
:10F28000882321F00E949238FE01F7CFEDE4F1E2ED
:10F290008491EF012196882321F00E949238FE018B
:10F2A000F7CF329903C0CEE2D3E002C0C3E3D3E08C
:10F2B0008991882319F00E949238FACF8AE00E943F
:10F2C0009238E5E4F1E28491EF012196882321F060
:10F2D0000E949238FE01F7CF339903C0CEE2D3E00B
:10F2E00002C0C3E3D3E08991882319F00E949238C9
:10F2F000FACF8AE00E949238EDE3F1E28491EF01C7
:10F300002196882321F00E949238FE01F7CF34998C
:10F3100003C0CEE2D3E002C0C3E3D3E089918823E7
:10F3200019F00E949238FACF8AE0DF91CF910C94C5
:10F330009238CF93DF932BE838E1CCE2D1E1ACE314
:10F34000B1E180E090E0FC01E251F14E4591559130
:10F3500065917491F90141935193619371939F0168
:10F36000FC01E252F14E459155916591749149939A
:10F37000599369937993FC01E253F14E459155916C
:10F38000659174914D935D936D937D930496803157
:10F390009105C9F680E090E0AAEFB3E480935411A0
:10F3A00090935511A0935611B0935711809350111B
:10F3B00090935111A0935211B093531180E090E0BB
:10F3C000AAE7B4E480934C1190934D11A0934E1191
:10F3D000B0934F11109228111092291110922A11F6
:10F3E00010922B1180E29EE4A0E0B0E080935209DD
:10F3F00090935309A0935409B09355091092241186
:10F4000010922511109226111092271180E090E0A1
:10F41000A0E2B1E48093691190936A11A0936B11FB
:10F42000B0936C1180936D1190936E11A0936F1136
:10F43000B09370118DEC9CECACECBEE38093711139
:10F4400090937211A0937311B093741180E090E0C7
:10F45000A0EAB0E48093751190937611A093771190
:10F46000B09378118CE0E9E1F7E0DF011D928A9515
:10F47000E9F789EB90E090931D1180931C1180EFC8
:10F4800090E090931F1180931E118DE290E0909375
:10F4900019118093181186E490E090931B118093CA
:10F4A0001A118FEF90E09093211180932011909387
:10F4B00023118093221182E598EBA6EAB1E48093B0
:10F4C000AF109093B010A093B110B093B2108EEA29
:10F4D0009AE6A4EABEE38093AB109093AC10A0939D
:10F4E000AD10B093AE1081EF97E4A9EAB3E4809336
:10F4F000B3109093B410A093B510B093B6101092BF
:10F500007D1180E090E0A0EEBFE3809379119093AD
:10F510007A11A0937B11B0937C111092B3031092D7
:10F520001511DF91CF910C94CACEAF92BF92CF92BA
:10F53000DF92EF92FF920F931F93CF93C82F8823F0
:10F5400019F0E5E2F1E20CC0E8E0F5E384918F0107
:10F550000F5F1F4F8823A9F30E949238F801F6CF5E
:10F5600084918F010F5F1F4F882321F00E949238F2
:10F57000F801F6CFCC2319F0E8E0F1E20CC0E8E0A6
:10F58000F5E384918F010F5F1F4F8823A9F30E9439
:10F590009238F801F6CF84918F010F5F1F4F8823B7
:10F5A00021F00E949238F801F6CF8AE00E9492384A
:10F5B000C1112CC0E8E0F5E384918F010F5F1F4F6C
:10F5C000882321F00E949238F801F6CFE5EFF0E2AF
:10F5D00084918F010F5F1F4F882321F00E94923882
:10F5E000F801F6CF80917D11882321F08AE00E94F6
:10F5F00092383AC0EAEEF0E284918F010F5F1F4F1C
:10F60000882391F10E949238F801F6CF4091791148
:10F6100050917A1160917B1170917C1181EE90E292
:10F620000E9417418AE00E94923880917D118111D9
:10F6300027C0CC2319F0E6EDF0E20CC0E8E0F5E3DA
:10F6400084918F010F5F1F4F8823A9F30E94923886
:10F65000F801F6CF84918F010F5F1F4F882381F04F
:10F660000E949238F801F6CFE8E0F5E384918F012B
:10F670000F5F1F4F882351F20E949238F801F6CF96
:10F68000C11124C0E8E0F5E384918F010F5F1F4FA3
:10F69000882321F00E949238F801F6CFE5ECF0E2E1
:10F6A00084918F010F5F1F4F882321F00E949238B1
:10F6B000F801F6CFE8E0F5E384918F010F5F1F4F6B
:10F6C000882321F00E949238F801F6CF40918B18E0
:10F6D00050918C1860918D1870918E188DEB90E27E
:10F6E0000E94174140918F18509190186091911885
:10F6F000709192188AEB90E20E9417414091931802
:10F7000050919418609195187091961887EB90E23B
:10F710000E9417414091971850919818609199183C
:10F7200070919A1884EB90E20E9417418AE00E943F
:10F730009238C11124C0E8E0F5E384918F010F5F96
:10F740001F4F882321F00E949238F801F6CFE6E996
:10F75000F0E284918F010F5F1F4F882321F00E94F8
:10F760009238F801F6CFE8E0F5E384918F010F5F5E
:10F770001F4F882321F00E949238F801F6CF409164
:10F780002C1150912D1160912E1170912F118DE837
:10F7900090E20E94174140913011509131116091D7
:10F7A0003211709133118AE890E20E941741409122
:10F7B000341150913511609136117091371187E8ED
:10F7C00090E20E9417414091381150913911609197
:10F7D0003A1170913B1184E890E20E9417418AE04F
:10F7E0000E949238C11124C0E8E0F5E384918F01B2
:10F7F0000F5F1F4F882321F00E949238F801F6CF47
:10F80000E2E6F0E284918F010F5F1F4F882321F021
:10F810000E949238F801F6CFE8E0F5E384918F0179
:10F820000F5F1F4F882321F00E949238F801F6CF16
:10F8300040913C1150913D1160913E1170913F11EA
:10F8400089E590E20E94FA404091401150914111A7
:10F85000609142117091431186E590E20E94FA4056
:10F86000409144115091451160914611709147119A
:10F8700083E590E20E94FA4040914811509149116D
:10F8800060914A1170914B1180E590E20E94FA401C
:10F890008AE00E949238C11124C0E8E0F5E3849127
:10F8A0008F010F5F1F4F882321F00E949238F801CB
:10F8B000F6CFE6E0F0E284918F010F5F1F4F8823BF
:10F8C00021F00E949238F801F6CFE8E0F5E3849148
:10F8D0008F010F5F1F4F882321F00E949238F8019B
:10F8E000F6CF40915411509155116091561170917D
:10F8F00057118DEF9FE10E94174140915011509197
:10F90000511160915211709153118AEF9FE10E9441
:10F91000174140914C1150914D1160914E117091D1
:10F920004F1187EF9FE10E9417418AE00E949238B1
:10F93000C11124C0E8E0F5E384918F010F5F1F4FF0
:10F94000882321F00E949238F801F6CFE3E8FFE126
:10F9500084918F010F5F1F4F882321F00E949238FE
:10F96000F801F6CFE8E0F5E384918F010F5F1F4FB8
:10F97000882321F00E949238F801F6CF4091281197
:10F980005091291160912A1170912B118AE79FE102
:10F990000E94174140912411509125116091261128
:10F9A0007091271187E79FE10E941741409152090A
:10F9B00050915309609154097091550984E79FE172
:10F9C0000E94FA404091691150916A1160916B1147
:10F9D00070916C1181E79FE10E94174140916D1178
:10F9E00050916E1160916F11709170118EE69FE1D0
:10F9F0000E941741409171115091721160917311E1
:10FA0000709174118BE69FE10E941741409175112E
:10FA100050917611609177117091781188E69FE18D
:10FA20000E9417418AE00E949238C11124C0E8E088
:10FA3000F5E384918F010F5F1F4F882321F00E940F
:10FA40009238F801F6CFEAE5FFE184918F010F5F6C
:10FA50001F4F882321F00E949238F801F6CFE8E08A
:10FA6000F5E384918F010F5F1F4F882321F00E94DF
:10FA70009238F801F6CF4091190750911A0760911A
:10FA80001B0770911C0781E59FE10E94174140917F
:10FA90001D0750911E0760911F07709120078EE48B
:10FAA0009FE10E94174140912107509122076091E8
:10FAB0002307709124078BE49FE10E9417418AE09D
:10FAC0000E949238CC2379F08CE1A82E81E1B82EE7
:10FAD00098E1C92E91E1D92E20E2E22E21E1F22E09
:10FAE00000E010E024C0E8E0F5E384918F010F5FAF
:10FAF0001F4F882321F00E949238F801F6CFEEE2E2
:10FB0000FFE184918F010F5F1F4F882321F00E9436
:10FB10009238F801F6CFE8E0F5E384918F010F5FAA
:10FB20001F4F882389F20E949238F801F6CFB8015E
:10FB300085E29FE10E943441F501619171915F017D
:10FB400082E29FE10E943441F601619171916F015F
:10FB50008FE19FE10E943441F701619171917F0132
:10FB60008CE19FE10E9434418AE00E9492380F5F4D
:10FB70001F4F02301105D9F6C11124C0E8E0F5E3AA
:10FB800084918F010F5F1F4F882321F00E949238CC
:10FB9000F801F6CFEDE0FFE184918F010F5F1F4F79
:10FBA000882321F00E949238F801F6CFE8E0F5E3CF
:10FBB00084918F010F5F1F4F882321F00E9492389C
:10FBC000F801F6CF4091AF105091B0106091B11094
:10FBD0007091B21084E09FE10E9417412CEA35EC4D
:10FBE00047E25EE36091AB107091AC108091AD1074
:10FBF0009091AE100E9437F1AB01BC0181E09FE112
:10FC00000E9417412CEA35EC47E25EE36091B310A5
:10FC10007091B4108091B5109091B6100E94E9E9EE
:10FC2000AB01BC018EEF9EE10E9417418AE0CF91AB
:10FC30001F910F91FF90EF90DF90CF90BF90AF900A
:10FC40000C949238EF92FF920F931F93CF93DF9310
:10FC500000D000D0CDB7DEB71092E2118091FB1535
:10FC60009091FC15A091FD15B091FE158130904842
:10FC7000A105B10540F01092FB151092FC151092F1
:10FC8000FD151092FE151091FB1580915C11181650
:10FC9000DCF4282F082E000C330B21503109412FA2
:10FCA000012E000C550B4217530774F01FEF180F6D
:10FCB000812F90E0A0E0B0E08093FB159093FC15BD
:10FCC000A093FD15B093FE151092851180918611B9
:10FCD000181714F41093861180918611082E000CC9
:10FCE000990B0496212F012E000C330B82179307DA
:10FCF00024F48CEF810F80938611E0908611F12C13
:10FD0000E1101DC08091E411811106C080918F0126
:10FD1000882309F483C009C01111F8CF0E94045050
:10FD200080918511882391F376C181E0111180E0E3
:10FD300024E044E753E26F2D0E9445B26FC081E09A
:10FD4000E81228C08091E411811106C080918F01D2
:10FD5000882309F463C011C01130C1F720E030E0FE
:10FD600040E251E464E571E18EE693E20E9444E3EF
:10FD700080918511882351F34EC184E591E10E9461
:10FD80004BB09C0181E0113009F080E000E048E6D2
:10FD900053E241C022E0E21227C08091E4118111B8
:10FDA00005C080918F018823C9F111C01230C9F7B5
:10FDB00020E030E048EC52E460E571E18EE593E24A
:10FDC0000E9444E380918511882359F324C180E582
:10FDD00091E10E944BB09C0181E0123009F080E07B
:10FDE00000E044E553E217C023E0E21231C0809105
:10FDF000E41181111CC080918F01882379F08CE47B
:10FE000091E10E944BB09C0181E0133009F080E049
:10FE100000E042E453E26F2D0E945FDEF394E3942E
:10FE200085E0F8126DCF88E080935C11F4C0133048
:10FE300011F720E030E048EC52E46CE471E18BE42F
:10FE400093E20E9444E3809185118823A1F2E3C0EC
:10FE500084E0E81235C08091E411811105C08091E1
:10FE60008F018823D9F211C01430C9F724E630E09D
:10FE700040E050E06CE371E18BE393E20E9404E424
:10FE800080918511882359F3C6C060913C1170910F
:10FE90003D1180913E1190913F110E9488E9698344
:10FEA0007A838B839C83CE0101960E944BB09C0188
:10FEB00081E0143009F080E000E044E353E2ABCF8E
:10FEC00025E0E21236C08091E411811106C08091D4
:10FED0008F01882309F4A2CF11C01530C1F724E6A1
:10FEE00030E040E050E060E471E18DE293E20E9496
:10FEF00004E480918511882351F38DC060914011F5
:10FF00007091411180914211909143110E9488E9B2
:10FF100069837A838B839C83CE0101960E944BB0C8
:10FF20009C0181E0153009F080E000E046E253E2F8
:10FF300072CF86E0E81236C08091E411811106C0CC
:10FF400080918F01882309F469CF11C01630C1F761
:10FF50002AE030E040E050E064E471E18FE193E2B8
:10FF60000E9404E480918511882351F354C060916C
:10FF700044117091451180914611909147110E9452
:10FF800088E969837A838B839C83CE0101960E94E2
:10FF90004BB09C0181E0163009F080E000E048E1C0
:10FFA00053E239CF27E0E21239CF8091E411811179
:10FFB00006C080918F01882309F430CF11C017301B
:10FFC000C1F724E630E040E050E068E471E181E10F
:10FFD00093E20E9404E480918511882351F31BC0B1
:10FFE000609148117091491180914A1190914B1183
:10FFF0000E9488E969837A838B839C83CE01019672
:020000021000EC
:100000000E944BB09C0181E0173009F080E000E0D5
:100010004AE053E200CF0F900F900F900F90DF91C6
:10002000CF911F910F91FF90EF9008950C94B841DC
:100030002F924F926F927F928F929F92AF92BF9228
:10004000CF92DF92EF92FF920F931F93CF93DF93A4
:100050001092E2118091FB159091FC15A091FD1575
:10006000B091FE1581309048A105B10540F0109285
:10007000FB151092FC151092FD151092FE15C09103
:10008000FB1580915B111816DCF4282F082E000C4C
:10009000330B215031094C2F0C2E000C550B4217FD
:1000A000530774F0CFEFC80F8C2F90E0A0E0B0E0C2
:1000B0008093FB159093FC15A093FD15B093FE154E
:1000C0001092851180918611C81714F4C09386117F
:1000D00080918611082E000C990B04962C2F0C2E63
:1000E000000C330B8217930724F48CEF8C0F809352
:1000F0008611D0918611412C63E0262E7BEC672E71
:1001000072E2772EE0EECE2EE2E2DE2EFEEEAF2E93
:10011000F2E2BF2EA5EF8A2EA2E29A2ED1111DC0C7
:100120008091E411811106C080918F01882309F428
:10013000A5C009C0C111F8CF0E940450809185115B
:10014000882391F3A9C181E0C11180E024E043E05C
:1001500053E2642D0E9445B291C0D13009F03FC0F6
:100160008091E411811106C080918F01882309F4E8
:1001700085C016C0C130C1F7E12C10ECF12E09E7A3
:1001800014E420E030E040E85FE36CE271E18CEFE2
:1001900092E20E9485E080918511882329F37CC139
:1001A0002F9287EE8F931F9281E08F938CE291E1E3
:1001B0009F938F93BF92AF929F928F924F9281E0C5
:1001C000C13009F080E08F930E94CFDE8DB79EB7DB
:1001D0000C960FB6F8949EBF0FBE8DBF4FC0D230A5
:1001E00009F041C08091E411811106C080918F0116
:1001F000882309F443C016C0C230C1F7E12C10ECCB
:10020000F12E09E714E420E030E040E85FE360E32A
:1002100071E187EE92E20E9485E08091851188234A
:1002200029F33AC12F9287EE8F931F9281E08F932B
:1002300080E391E19F938F9389ED92E29F938F9357
:10024000DF92CF924F9281E0C23009F080E08F932D
:100250000E94CFDE8DB79EB70C960FB6F8949EBF66
:100260000FBE8DBF0BC0D33009F048C08091E411A0
:1002700081110DC080918F0181111FC04394DF5FF8
:1002800095E049124BCF87E080935B1105C1C330E5
:1002900089F7E12C10ECF12E09E714E420E030E0BE
:1002A00040E85FE364E371E182ED92E20E9485E061
:1002B000809185118823F1F2EFC02F9287EE8F9302
:1002C0001F9281E08F9384E391E19F938F9384EC5D
:1002D00092E29F938F937F926F924F9281E0C3300F
:1002E00009F080E08F930E94CFDE8DB79EB70C9609
:1002F0000FB6F8949EBF0FBE8DBFC0CFD43009F0AB
:1003000043C08091E411811106C080918F01882340
:1003100009F4B4CF16C0C430C1F7E12C10ECF12EB3
:1003200009E714E420E030E040E85FE368E371E1CE
:100330008DEB92E20E9485E080918511882329F35C
:10034000ABC02F9287EE8F931F9281E08F9388E34B
:1003500091E19F938F938FEA92E29F938F9386EB25
:1003600092E29F938F934F9281E0C43009F080E036
:100370008F930E94CFDE8DB79EB70C960FB6F89480
:100380009EBF0FBE8DBF7ACFD53009F041C080919E
:10039000E411811106C080918F01882309F46ECF8A
:1003A00015C0C530C1F7E12C10ECF12E09E714E4BB
:1003B00020E030E0A90168E271E18AEA92E20E945D
:1003C00085E080918511882331F366C02F9287EEF6
:1003D0008F931F921F9288E291E19F938F9380EAFF
:1003E00092E29F938F9385EA92E29F938F934F922D
:1003F00081E0C53009F080E08F930E94CFDE8DB799
:100400009EB70C960FB6F8949EBF0FBE8DBF36CF29
:10041000D63009F033CF8091E411811106C080916C
:100420008F01882309F42ACF15C0C630C1F7E12C0B
:1004300010ECF12E09E714E420E030E0A90164E2B9
:1004400071E186E992E20E9485E08091851188231E
:1004500031F322C02F9287EE8F931F921F9284E276
:1004600091E19F938F9382E892E29F938F938CE820
:1004700092E29F938F934F9281E0C63009F080E023
:100480008F930E94CFDE8DB79EB70C960FB6F8946F
:100490009EBF0FBE8DBFF2CEDF91CF911F910F9106
:1004A000FF90EF90DF90CF90BF90AF909F908F9094
:1004B0007F906F904F902F9008950C94D6421F9389
:1004C000CF93DF931092E2118091FB159091FC1570
:1004D000A091FD15B091FE1581309048A105B105A0
:1004E00040F01092FB151092FC151092FD15109221
:1004F000FE15C091FB15809158111816DCF4282FB9
:10050000082E000C330B215031094C2F0C2E000CFF
:10051000550B4217530774F0CFEFC80F8C2F90E0A4
:10052000A0E0B0E08093FB159093FC15A093FD151F
:10053000B093FE151092851180918611C81714F49E
:10054000C093861180918611082E000C990B049699
:100550002C2F0C2E000C330B8217930724F48CEFF6
:100560008C0F8093861110918611D0E011111AC062
:100570008091E411811106C080918F01882309F4D4
:1005800062C009C0C111F8CF0E940450809185114A
:10059000882391F3C8C081E0C11180E024E04AEBD8
:1005A00051E24EC01130E9F48091E411811106C08E
:1005B00080918F01882309F446C00BC0C130C1F778
:1005C00080E395E80E94AFBA80918511882381F37A
:1005D000AAC081E0C13009F080E023E04EEA51E298
:1005E0002FC01230E1F48091E411811105C0809197
:1005F0008F01882341F10BC0C230C9F78AE791E926
:100600000E94AFBA80918511882389F38CC081E064
:10061000C23009F080E023E047EA51E211C0133014
:1006200031F58091E411811117C080918F018823E9
:1006300051F081E0C33009F080E023E04EE951E25F
:100640006D2F0E9445B2DF5F1F5FD53009F08ECF5E
:1006500087E08093581167C0C33039F786E190E98D
:100660000E94AFBA809185118823F9F25CC01430E2
:10067000E1F48091E411811105C080918F018823FC
:1006800011F30BC0C430C9F70E94CEC10E94994F2C
:1006900080918511882389F346C081E0C43009F038
:1006A00080E020E24FE851E2CBCF1530E1F48091B9
:1006B000E411811105C080918F01882321F20BC0C4
:1006C000C530C9F70E94A9BD0E94994F809185113C
:1006D000882389F328C081E0C53009F080E020E25A
:1006E0004FE651E2ADCF163009F0ADCF8091E41165
:1006F000811106C080918F01882309F4A4CF0BC01B
:10070000C630C1F787E993E80E94AFBA809185119E
:10071000882381F308C081E0C63009F080E023E03F
:100720004DE751E28DCFDF91CF911F9108950E9447
:1007300099790E9410B20E94CEC10C9404502F925D
:100740003F924F925F926F927F928F929F92AF9261
:10075000BF92CF92DF92EF92FF920F931F93CF93AE
:10076000DF931092E2114091FB155091FC156091BE
:10077000FD157091FE15413050486105710540F03E
:100780001092FB151092FC151092FD151092FE159B
:100790001091FB1590915A111916DCF4292F092E8E
:1007A000000C330B21503109412F012E000C550B49
:1007B0004217530774F01FEF190F412F50E060E00C
:1007C00070E04093FB155093FC156093FD157093FA
:1007D000FE151092851190918611191714F410933B
:1007E000861120918611022E000C330B2C5F3F4F97
:1007F000412F012E000C550B2417350724F49CEFD4
:10080000910F9093861100918611412C5524539499
:10081000C82FD0E0CC0FDD1FCE01885E9E4E1C019C
:10082000CE01845E9E4E7C0193E4692E92E2792E85
:100830002AE4C22E22E2D22EC05EDE4E38E5A32E7E
:1008400032E2B32E42E6842E42E2942E01111AC007
:100850008091E411811106C080918F01882309F4F1
:1008600098C009C01111F8CF0E94045080918511E1
:10087000882391F3DCC081E0111180E024E046E799
:1008800052E284C00130B1F58091E411811106C0BB
:1008900080918F01882309F47CC010C01130C1F70A
:1008A0002FEF30E040E050E0BE018CE692E20E9483
:1008B000F1E080918511882359F3B9C01F928FEF21
:1008C0008F931F921F92DF93CF93BF92AF929F920D
:1008D0008F924F9281E0113009F080E08F930E9457
:1008E000EBDE8DB79EB70C960FB6F8949EBF0FBE89
:1008F0008DBF4FC00230B9F58091E411811106C05F
:1009000080918F01882309F444C010C01230C1F7D0
:1009100024E031E045E050E0B70181E592E20E9439
:10092000F1E080918511882359F381C05F9284E0C2
:100930008F931F9285E08F93FF92EF927F926F9239
:10094000DF92CF924F9281E0123009F080E08F93D6
:100950000E94EBDE8DB79EB70C960FB6F8949EBF43
:100960000FBE8DBF16C00330E1F0043091F48091CA
:10097000E411811150C080918F01882351F081E0F2
:10098000143009F080E020E248E252E2642D0E9437
:1009900045B243940F5F95E0491258CF40925A11E7
:1009A00046C08091E411811105C080918F01882398
:1009B00081F310C01330C9F727E830E045E050E07C
:1009C000B1018FE392E20E94F1E0809185118823CA
:1009D00061F32DC01F9287E88F931F9285E08F935C
:1009E0003F922F9287E392E29F938F938BE392E261
:1009F0009F938F934F9281E0133009F080E08F93A3
:100A00000E94EBDE8DB79EB70C960FB6F8949EBF92
:100A10000FBE8DBFBECF143009F0ADCF0E94CEC146
:100A20000E94994F80918511882309F4A4CFDF910A
:100A3000CF911F910F91FF90EF90DF90CF90BF90DB
:100A4000AF909F908F907F906F905F904F903F906E
:100A50002F90089581E00C949F8380E00C949F83F5
:100A60002F923F924F925F926F927F928F929F92BE
:100A7000AF92BF92CF92DF92EF92FF920F931F93AC
:100A8000CF93DF931092E2118091FB159091FC15AA
:100A9000A091FD15B091FE1581309048A105B105DA
:100AA00040F01092FB151092FC151092FD1510925B
:100AB000FE15C091FB15809159111816DCF4282FF2
:100AC000082E000C330B215031094C2F0C2E000C3A
:100AD000550B4217530774F0CFEFC80F8C2F90E0DF
:100AE000A0E0B0E08093FB159093FC15A093FD155A
:100AF000B093FE151092851180918611C81714F4D9
:100B0000C093861180918611082E000C990B0496D3
:100B10002C2F0C2E000C330B8217930724F48CEF30
:100B20008C0F80938611D0918611612C44244394BC
:100B300077247A9481EE282E81E2382E0BEE11E292
:100B400097E8592E2FEFE22E21E2F22E33E0C32E4A
:100B500032E2D32E4BE0A42E42E2B42E52E1852E97
:100B600052E2952ED1111AC08091E411811106C074
:100B700080918F01882309F4BBC009C0C111F8CF4F
:100B80000E94045080918511882391F328C181E04F
:100B9000C11180E024E040E252E2A7C0D13009F068
:100BA00047C08091E411811106C080918F01882394
:100BB00009F49EC01BC0C130C1F7C093E21110926E
:100BC000DE111092DF111092E0111092E11122E675
:100BD00036E544E051E06EE277E089E192E20E947E
:100BE000F3E280918511882301F3F9C082E696E54E
:100BF0009F938F934F9284E08F931F921F928EE268
:100C000097E09F938F93BF92AF929F928F926F9234
:100C100081E0C13009F080E08F930E94EBDE8DB758
:100C20009EB70E960FB6F8949EBF0FBE8DBF60C0E4
:100C3000D23009F046C08091E411811106C0809144
:100C40008F01882309F454C01BC0C230C1F7409201
:100C5000E2111092DE111092DF111092E011109249
:100C6000E11125E636E547E850E06EE076E187E001
:100C700092E20E94F3E280918511882301F3AFC0D4
:100C800085E696E59F938F931F925F921F921F9226
:100C90008EE096E19F938F93FF92EF92DF92CF9237
:100CA0006F9281E0C23009F080E08F930E94EBDE0A
:100CB0008DB79EB70E960FB6F8949EBF0FBE8DBF30
:100CC00017C0D330F1F0D43009F069C08091E4113D
:100CD000811158C080918F01882351F081E0C43088
:100CE00009F080E023E040ED51E2662D0E9445B21C
:100CF0006394DF5F95E0691235CF86E080935911E8
:100D00006EC08091E411811105C080918F0188230C
:100D100079F31BC0C330C9F74092E2111092DE1183
:100D20001092DF111092E0111092E1112FEF30E0DC
:100D300040E050E060E176E185EF91E20E94F1E071
:100D400080918511882309F34AC01F927F921F92D8
:100D50001F9280E196E19F938F933F922F921F9372
:100D60000F936F9281E0C33009F080E08F930E946F
:100D7000EBDE8DB79EB70C960FB6F8949EBF0FBEF4
:100D80008DBFB6CFC43009F0A5CF8DE295E80E94A3
:100D9000AFBA80918511882309F49CCF20C0D5304B
:100DA00009F0A6CF8091E411811106C080918F01D6
:100DB000882309F49DCF0BC0C530C1F78AE295E8BE
:100DC0000E94AFBA80918511882381F308C081E029
:100DD000C53009F080E023E04FEB51E286CFDF9190
:100DE000CF911F910F91FF90EF90DF90CF90BF9028
:100DF000AF909F908F907F906F905F904F903F90BB
:100E00002F900895FF920F931F93CF93DF938C0140
:100E1000EB01F42E80E20E9492388FEFF81611F069
:100E200084E501C082E40E9492388AE30E949238ED
:100E3000F801608171818281938142E00E949F3C30
:100E4000488159816A817B818BE793E2DF91CF9161
:100E50001F910F91FF900C94174188E893E19093B4
:100E6000A8108093A71080916F008D7F80936F00F2
:100E700090915C1280915D12981719F00E94BF67E3
:100E8000F7CF1092AA101092A91080916F00826083
:100E900080936F008FB7F8941092D9111092DA11E5
:100EA0001092DB111092DC118FBF0E94876780E0E7
:100EB00090E00E94686760935D1170935E1180936B
:100EC0005F119093601181E090E00E9468676093E9
:100ED000611170936211809363119093641182E0A9
:100EE00090E00E946867609365117093661180932B
:100EF0006711909368118CE0EDE5F1E1ABE7B8E1A3
:100F000001900D928A95E1F70C94F4364F925F921E
:100F10006F927F928F929F92AF92BF92CF92DF9209
:100F2000EF92FF92CF93DF93EDEEF3E28491EF0126
:100F30002196882321F00E949238FE01F7CF60911C
:100F40007B1870917C1880917D1890917E1842E0FA
:100F50000E949F3CE9EEF3E28491EF012196882301
:100F600021F00E949238FE01F7CF60917F187091B6
:100F70008018809181189091821842E00E949F3CD5
:100F8000E5EEF3E28491EF012196882321F00E949F
:100F90009238FE01F7CF6091831870918418809188
:100FA00085189091861842E00E949F3CE1EEF3E2A2
:100FB0008491EF012196882321F00E949238FE014E
:100FC000F7CF609187187091881880918918909157
:100FD0008A1842E00E949F3C8FB7F89440906B18AB
:100FE00050906C1860906D1870906E1880906F180B
:100FF00090907018A0907118B0907218C0907318EB
:10100000D0907418E0907518F09076188FBFE7EDC7
:10101000F3E28491EF012196882321F00E94923817
:10102000FE01F7CFC301B2010E944839E3EDF3E2BC
:101030008491EF012196882321F00E949238FE01CD
:10104000F7CFC501B4010E944839EFECF3E2849177
:10105000EF012196882321F00E949238FE01F7CFFC
:10106000C701B6010E9448398AE0DF91CF91FF9015
:10107000EF90DF90CF90BF90AF909F908F907F9038
:101080006F905F904F900C9492380F931F93CF9373
:10109000DF93CDB7DEB728970FB6F894DEBF0FBE4B
:1010A000CDBF60912E0770912F07072E000C880B83
:1010B000990B0E948AE96D837E838F839887809144
:1010C000C5119091C611A091C711B091C811898323
:1010D0009A83AB83BC834EEFBE016B5F7F4FCE0123
:1010E00001960E94028760910E1670910F16072ECE
:1010F000000C880B990B0E948AE96D837E838F8395
:1011000098878091770990917809A0917909B09199
:101110007A0989839A83AB83BC834FEFBE016B5FEF
:101120007F4FCE0101960E940287E3E8F3E28491AB
:101130008F010F5F1F4F882321F00E949238F80122
:10114000F6CFE0919C03F0E0EF55FE4E608170E039
:1011500080E090E00E944839EEE7F3E284918F014D
:101160000F5F1F4F882321F00E949238F801F6CFBD
:101170006091A01170E080E090E00E9448392896CC
:101180000FB6F894DEBF0FBECDBFDF91CF911F9198
:101190000F9108952F923F924F925F926F927F929C
:1011A0008F929F92AF92BF92CF92DF92EF92FF9277
:1011B0000F931F93CF93DF93CDB7DEB7E0970FB6B2
:1011C000F894DEBF0FBECDBF85E40E9402388823AD
:1011D00029F00E946C377A83698302C01A821982CF
:1011E00083E40E940238882329F00E946C3779A793
:1011F00068A704C025E030E039A728A785E50E944C
:10120000D3378F8F882319F00E9490378F8F4981B1
:101210005A8157FD07C0C12CD12CB6E1EB2EB3E4A7
:10122000FB2E06C0C12CD12CACE8EA2EA2E4FA2E8B
:1012300083E50E940238882321F00E94A0376B01C9
:101240007C0189819A81892B11F410929C030E9460
:101250004BAE4B015C01A981BA81AB2B49F1EDE3A7
:10126000F3E0FA83E983A981BA818D91BA83A983D6
:10127000882319F00E949238F6CF8AE0E0960FB6E4
:10128000F894DEBF0FBECDBFDF91CF911F910F91BC
:10129000FF90EF90DF90CF90BF90AF909F908F9096
:1012A0007F906F905F904F903F902F900C9492386A
:1012B000E6E6F3E0FA83E983A981BA818D91BA83E6
:1012C000A983882319F00E949238F6CFC701B6018E
:1012D0000E94A9F1072E000C880B990B0E948AE945
:1012E0006B877C878D879E878AE00E9492380E9458
:1012F00027A48FE78093A11181E08093170188A232
:1013000099A2AAA2BBA28AA69BA6ACA6BDA61F862E
:10131000B0E4B88BECE1E98BF6E4FA8B1B8A1C8A0B
:101320001D8A1E8A1B8E1C8E1D8E1E8E1F8A188E75
:10133000198E1A8E412C512C3201FFE7CF2ED12C61
:10134000E12CF12C2FE730E040E050E02D833E838C
:101350004F8358871CA21DA21EA21FA231E03EA7E8
:101360001A861986212C312C00E010E0809117019B
:10137000882309F465C10E944BAE69837A838B830D
:101380009C8380919F11882309F484C00E942AA520
:101390002090C5113090C6110091C7111091C8114D
:1013A0002B893C894D895E89B101C8010E949DF25B
:1013B000181624F42B8A3C8A0D8B1E8B2F853889B6
:1013C00049895A89B101C8010E9483E987FF04C095
:1013D0002F86388A098B1A8B4EA591014423E9F197
:1013E000A8016B857C858D859E850E9483E987FF9A
:1013F00051C049815A816B817C81481959096A0918
:101400007B09DB01CA0188589341A109B109B7FDE5
:1014100041C08D819E81AF81B8858C199D09AE092F
:10142000BF09B595A795979587958093A1114CA372
:101430005DA36EA37FA35B855B8B8C858C8B9D8569
:101440009D8BAE85AE8B29813A814B815C8128A32F
:1014500039A34AA35BA31EA61DC0A8016B857C858A
:101460008D859E850E949DF21816A4F489819A812B
:10147000AB81BC8128A139A14AA15BA1821B930B3E
:10148000A40BB50BAC01BD0148585341610971096A
:1014900077FFF4C020E030E040EA51E46B857C85C2
:1014A0008D859E850E943DF09101A8010E9483E9EF
:1014B00087FF10C0EAEAF4E284919F012F5F3F4F5B
:1014C0003A832983882309F425C20E949238E9814E
:1014D000FA81F2CF80E398EFAFEFBFEF2AA53BA5EB
:1014E0004CA55DA5821B930BA40BB50B29813A81FA
:1014F0004B815C81820F931FA41FB51FB7FD0DC0E8
:101500000E9445888AE00E94923889819A81AB8145
:10151000BC818AA79BA7ACA7BDA789819A81AB8113
:10152000BC81880F991FAA1FBB1F28A139A14AA1FE
:101530005BA1821B930BA40BB50B88199909AA090F
:10154000BB0981389F44A241B10580F0ECE8F4E288
:101550008491AF014F5F5F4F5A834983882309F419
:10156000D9C10E949238E981FA81F2CF88A599A564
:10157000A985BA858A179B070CF05FC0EFE2F4E2F9
:1015800084919F012F5F3F4F3A832983882329F05D
:101590000E949238E981FA81F3CFB301A2018AE176
:1015A00094E20E9417418AE00E9492384F89588D38
:1015B000698D7A8D85E094E20E9417418AE00E944D
:1015C00092384B8D5C8D6D8D7E8D80EF93E20E9405
:1015D00017418AE00E9492383F8D332309F49AC163
:1015E0004092AF105092B0106092B1107092B21051
:1015F0002CEA35EC47E25EE36F89788D898D9A8D10
:101600000E94E9E96093AB107093AC108093AD1029
:101610009093AE102CEA35EC47E25EE36B8D7C8D47
:101620008D8D9E8D0E9437F16093B3107093B4102E
:101630008093B5109093B6106DC10E94C0B796CE3E
:1016400080911701811166C1E0960FB6F894DEBF54
:101650000FBECDBFDF91CF911F910F91FF90EF9003
:10166000DF90CF90BF90AF909F908F907F906F90C2
:101670005F904F903F902F900C9427A449855A85F6
:10168000141615060CF024C18CA09DA0AEA0BFA01E
:10169000880E991EAA1EBB1E2CA13DA14EA15FA1C2
:1016A000281B390B4A0B5B0BC701B6010E94C9EF1F
:1016B000A50194010E94FBEFCD80DE80EF80F884CD
:1016C000C20ED31EE41EF51E54E1C516D104E1047A
:1016D000F1040CF18CEEC816D104E104F1043CF4E1
:1016E00090E8C916D104E104F10434F422C05BEEA1
:1016F000C52ED12CE12CF12CCD82DE82EF82F88632
:101700002EEF30E040E050E02C193D094E095F0912
:1017100069017A0112C084E190E0A0E0B0E08D831D
:101720009E83AF83B88744E1C42ED12CE12CF12CE9
:1017300004C0CD82DE82EF82F886E6E1F5E2849194
:10174000DF011196B8ABAFA7882329F00E94923829
:10175000EFA5F8A9F4CF6D817E818F8198850E94D5
:101760004839E1E1F5E284919F012F5F3F4F38ABAB
:101770002FA7882329F00E949238EFA5F8A9F3CF6C
:10178000C701B6010E9448394F85588969897A890D
:101790008AE095E20E9417414B895C896D897E89B8
:1017A00083E095E20E94174149855A8543305105EF
:1017B0000CF48EC0C701B6010E948AE920E030E037
:1017C00040E850E40E94E9E92B013C012F8538896B
:1017D00049895A896B897C898D899E890E943CF050
:1017E0002BED3FE049E450E40E94E9E920E030E0DD
:1017F00040E05FE30E94E9E99B01AC01C301B20153
:101800000E9437F12B013C01C501B4010E948AE915
:101810002FE632E143E85AE30E94E9E94B015C011B
:10182000B301A2018DEF94E20E941741B501A4011A
:1018300087EF94E20E9417412AE939E949E15FE321
:10184000C301B2010E94E9E92B013C019B01AC01FB
:101850000E943DF0A50194010E9437F16F8B788FB3
:10186000898F9A8FA3019201C501B4010E94E9E911
:1018700020E030E040E05EE30E94E9E96B8F7C8F7E
:101880008D8F9E8FE7EEF4E284915F015FEFA51AE2
:10189000B50A882321F00E949238F501F5CFB301F3
:1018A000A20181EE94E20E9417414F89588D698D03
:1018B0007A8D8BED94E20E9417414B8D5C8D6D8D7E
:1018C0007E8D85ED94E20E9417418AE00E94923855
:1018D0008D819E81AF81B8858C0D9D1DAE1DBF1D74
:1018E000B595A795979587958093A11189859A8538
:1018F00001969A8789879B859F87AC85A88BBD8534
:10190000B98BEE85EA8B89809A80AB80BC80F1E050
:10191000FEA7C0CDE0960FB6F894DEBF0FBECDBFD8
:10192000DF91CF911F910F91FF90EF90DF90CF90BB
:10193000BF90AF909F908F907F906F905F904F90EF
:101940003F902F9008952F923F924F925F926F9207
:101950007F928F929F92AF92BF92CF92DF92EF923F
:10196000FF920F931F93CF93DF93CDB7DEB72F97DF
:101970000FB6F894DEBF0FBECDBF8091C10983FDC5
:1019800070C160E082EC93E20E9407B383E50E949D
:1019900002388887811106C082E50E9402388823B8
:1019A00009F45FC10E94A0370E94A9F1673971054F
:1019B00014F066E970E070930F1660930E160E94A3
:1019C000DBA30E94A03720E030E040EA50E40E9410
:1019D0009DF2181614F40E9463CC81E080931701E5
:1019E0008091730980939C03412C512C32011C82FD
:1019F0001D821E821F821B8219862CE32A873CE1EE
:101A00003B8746E44C8710E000E050E859838FEBB9
:101A10008A83812C912C540160910E1670910F16BF
:101A2000072E000C880B990B0E948AE97B018F8797
:101A30009D879B01AC01612F702F89819A810E9443
:101A400083E9882309F449C0209177093091780906
:101A50004091790950917A099885B7018F85911144
:101A60000EC09D850E9483E9881F8827881F8B836D
:101A70001E2D0F2DAF85A983BD85BA832EC09D85F0
:101A80000E9483E987FF22C080911701882309F40F
:101A9000E8C060E084EB93E22F960FB6F894DEBFC7
:101AA0000FBECDBFDF91CF911F910F91FF90EF90AF
:101AB000DF90CF90BF90AF909F908F907F906F906E
:101AC0005F904F903F902F900C9407B31E2D0F2DD9
:101AD0002F8529833D853A831B820E944BAE6B0183
:101AE0007C01DC01CB012C813D814E815F81821B19
:101AF000930BA40BB50BB7FD3CC0D701C6018851B1
:101B00009C4FAF4FBF4F8C839D83AE83BF830E949A
:101B10004588EEEBF3E28491DF011196BE87AD8735
:101B2000882329F00E949238ED85FE85F4CF811438
:101B30009104A104B104B9F0D501C401805F984DAE
:101B4000AF4FBF4FBC01CD016C197D098E099F09B4
:101B500028EE33E040E050E00E94D9EFCA01B9011D
:101B60000E94483903C08FE30E9492388AE00E94A5
:101B7000923880E00E9444C80E94873820907709FC
:101B800030907809B0917909BF8720917A092D8723
:101B900091014B2F5D85612F702F89819A810E9461
:101BA0003CF09F7781149104A104B10449F420E032
:101BB00030E040E85FE30E9483E987FF0BC008C084
:101BC00020E030E040E450E40E949DF2181614F446
:101BD000460157013B81332361F1411451046104F3
:101BE000710441F0D701C60184199509A609B70906
:101BF000B7FD1FC091014F855D8569857A858B850D
:101C00009C850E943CF020E030E040EC5FE30E94C5
